:020000040800F2
:10000000000001206DAD050809AE0508A532040801
:100010000933040809AE050809AE05080000000010
:1000200000000000000000000000000009AE05080C
:1000300009AE05080000000009AE050851DA030802
:1000400009AE050809AE050809AE050809AE0508A0
:1000500009AE050809AE05086934040861340408CE
:100060005934040851340408493404087D9D0508B6
:100070006D9D05085D9D05084D9D0508399D050888
:10008000259D0508119D050809AE050809AE05085E
:1000900009AE050809AE050809AE05084134040893
:1000A000BD7F0508B5800508AD7F0508DD80050822
:1000B000A58005089580050885800508FDA0050830
:1000C00009A10508E5A00508F1A0050809AE050885
:1000D00009AE0508E9DA0308D9DA0308C9DA030822
:1000E0003934040809AE050809AE05089D7F0508E6
:1000F000CD7F050809AE0508F57F0508FD9C0508BC
:1001000009AE0508216F05087580050809AE0508C8
:10011000B9DA0308A9DA030805800508EDDB000851
:10012000E99C0508D59C0508C19C0508AD9C0508FF
:10013000999C05080000000000000000000000007D
:1001400000000000000000000000000085E0000842
:10015000859C0508719C05085D9C050899DA0308D3
:10016000CDA00508D9A0050809AE050809AE050807
:1001700009AE050809AE05080000000000000000F7
:1001800009AE050809AE050809AE050809AE05085F
:1001900009AE050809AE05080000000009AE050813
:1001A00000000000000000000000000009AE05088B
:1001B00009AE050809AE05080000000000000000B7
:1001C000000000000000000000000000000000002F
:1001D00000000000000000000000000009AE05085B
:0801E000C4A8050001000000A5
:1001E8000E020100020000000453012064530120A4
:1001F80000000000F42F07081402010005000000A9
:100208002C2B01206853012000000000F62F07085E
:10021800031101000A000000B852012070530120A8
:1002280000000000550F0108232001001000000005
:10023800885201207C53012000000000316D020823
:100248000D10010070000000105201208C53012095
:100258000000000045580308FD01010024000000CB
:1002680094510120FC530120000000005BC20308E8
:10027800FB01010001000000505101202054012021
:100288000000000019BE0408FC010100090000007C
:100298001C500120245401200000000021BE040845
:1002A800F701010006000000F04F01203054012042
:1002B80000000000FC2F0708F901010004000000FD
:1002C800E04F01203854012000000000C9C2030893
:1002D80034000100100000000C4F01203C540120A4
:1002E80000000000E9740208110201000800000083
:1002F800E44E01204C5401200000000002300708A1
:100308001212010004000000DC4E012054540120A8
:10031800000000000A30070818300100380000000B
:10032800A44E012058540120000000008DC6040886
:10033800000201000B000000284B0120905401200E
:100348000000000061BE0408FF2101000500000054
:10035800CC4A01209C5401200000000009BE04087A
:100368000812040014000000D84A0120A4540120F7
:100378000000000091BE0408130201000400000000
:10038800242B0120B8540120000000000E3007087B
:10039800FA010100030000002C4A0120BC5401208E
:1003A8000000000039BE04082A020100080000000D
:1003B800204A0120C0540120000000001230070824
:1003C8002052010008000000D8490120C85401202B
:1003D800000000000D75020806100100240000004E
:1003E800B4490120D05401200000000011BF0408C6
:1003F8000C0201000400000050480120F4540120C0
:100408000000000081BE0408FE0101001400000085
:100418006C340120F85401200000000069BE040873
:100428000B3001001A0000003C8F0120449101208C
:10043800000000001C3007081F50010024000000C5
:10044800008F01206091012000000000383007086B
:100458000502010004000000B08F012084910120F2
:10046800000000005C3007081B2001000C000000A1
:100478009C9401203C9F012000000000CD740108DD
:1004880021020100F0000000CC920120489F0120C9
:1004980000000000798101083710010030000000D9
:1004A8005C9C012038A00120000000006030070893
:1004B80016100100060000005896012068A00120CF
:1004C80000000000903007082F10010022000000F3
:1004D800189F012070A00120000000009630070836
:1004E8002322010010000000BC95012094A00120E7
:1004F80000000000B83007081E00010009000000D5
:10050800A4950120A4A0012000000000C83007081D
:10051800052001000C0000002C960120B0A001204D
:1005280000000000D430070812300100100000005D
:100538008C950120BCA0012000000000E0300708D5
:10054800FD0701007C00000090910120CCA0012053
:10055800000000003D6E0108F59101006C000000EC
:100568005092012048A10120000000009D80010850
:10057800261001000E000000C4A10120B4A1012032
:1005880000000000416C0108140001000500000093
:1005980028B501204CB5012000000000F030070804
:1005A800012001000C00000014AA012054B501200C
:1005B80000000000F63007080C400600E4000000C8
:1005C800C8A8012060B501200000000085FE0208CF
:1005D8000A9001002400000084A8012044B60120EC
:1005E80000000000E96C02080E300300BC010000A6
:1005F800C0A6012068B60120000000002975020885
:100608001310010004000000B4B2012024B8012036
:100618000000000004310708010101000400000087
:10062800F8A5012028B80120000000000000000003
:100638000001010004000000F0A501202CB80120F1
:100648000000000008310708020101000300000053
:10065800ECA5012030B8012000000000C9FE020806
:10066800220201001C01000000B0012034B8012062
:1006780000000000E9C60408010201000B000000A8
:1006880004A6012050B901200000000051BE040852
:1006980002020100030000008CAA01205CB90120BD
:1006A80000000000000000001B0201001000000014
:1006B80068AA012060B9012000000000FDBE0408FE
:1006C800150010007000000038C60120F8C601208F
:1006D80000000000000000002A0008006000000080
:1006E80048C5012068C7012000000000C174020845
:1006F8002C00040010000000D8C70120C8C7012042
:10070800000000009D7302082920140078000000F2
:10071800C0C20120E8C7012000000000000000005E
:100728001A0001000E00000030C2012060C801203C
:10073800000000000C3107082B0012002400000004
:100748000CC2012070C8012000000000717302086B
:10075800190201001000000010C1012094C80120F6
:100768000000000041BE04081C0202001C0000003A
:1007780044BF0120A4C801200000000071C404087F
:10078800283001001600000060BF0120C0C8012009
:1007980000000000217602080A020100140000008F
:1007A80028D3012044D301200000000051FE020894
:1007B8001010010002000000DCCC012058D30120F9
:1007C800000000001A310708F83101000600000097
:1007D800B8CD01205CD30120000000001C310708BF
:1007E8000300010001000000C8CD012064D30120EE
:1007F80000000000000000001900010005000000D2
:1008080094CC012068D301200000000022310708A1
:10081800020001000C000000B0D4012004D7012020
:100828000000000000000000F62101000C0000009C
:100838004CD6012010D701200000000028310708FD
:1008480025201E002C010000BCD401201CD701204B
:100858000000000000000000290201004000000024
:10086800DCD3012048D801200000000034310708FB
:100878002C02010004000000CCD6012088D80120F9
:10088800000000007431070828020400040000007A
:1008980044E0012060E6012000000000F9BE0408E1
:1008A800270204000400000040E0012064E6012063
:1008B80000000000EDBE0408160215003F0000000D
:1008C80034D9012068E601200000000005BE0408B4
:1008D8001A0201003C000000F8D80120A8E6012017
:1008E8000000000031C70408031201003D000000A9
:1008F8008CE20120E4E601200000000078310708BE
:100908003820010003000000C4D8012024E701209A
:1009180000000000B631070804000800800000004D
:10092800E8E7012068E9012000000000000000005D
:100938000B2201003D0000004CED01203CF301209A
:1009480000000000BC3107080D120100140000006F
:1009580018F301207CF3012000000000FC31070897
:100968001E02010006000000ACED012090F30120FA
:1009780000000000103207081D02020006000000F7
:10098800B8F2012098F301200000000000000000E8
:100998000612040018000000C0F20120A0F3012094
:1009A8000000000001C504081F0208001000000034
:1009B800C8F30120B8F3012000000000BDBD040801
:1009C8002700010004000000C8ED0120D8F3012031
:1009D80000000000163207081002010001000000A4
:1009E800CC170220C8170220000000001A3207089E
:08280000082800080040000850
:10800000026C03463AB11A6CD20608D50022012050
:1080100083F83C207047426480F83C20F3E71A6CF8
:1080200049494A4811401A6841F00201F0B4196404
:108030004168474D21F44031416041685C6821430B
:1080400041605168186921F48071D3F808C0DF6875
:10805000516054689E6A44EA0024AE4254605468F9
:1080600024F040745460506840EA0C0050609068FE
:1080700020F400609060916841EA0701916054D05B
:108080009068DC6A20F07060906091680E439660A2
:10809000906820F040509060916821439160906812
:1080A0009C6920F002009060916841EA440191606F
:1080B00093F82010002941D05468596A44F40064B0
:1080C000481E5460516821F460415160516841EA92
:1080D00040315160D06A0025DC6920F470005E698F
:1080E000611ED0622846D46A44EA0154D46294687E
:1080F00024F400749460946893F8301044EA4124A6
:108100009460946824F480649460916841EA8621C4
:1081100091605D641A6C22F0030242F001021A645D
:10812000002283F83C20F0BC7047916821F0706118
:108130009160916821F040519160B0E7516821F45D
:1081400000615160C6E700BFFDEEFFFF0023014064
:108150000100000F0129F0B42A4C4FF000062A4D0F
:1081600094BF002701272368EE626662A6626763F8
:10817000676B47EA42076763EE63EC6B002A38D10E
:1081800044F49574EC631C6824F001041C601C68C2
:10819000E407FCD4490289085960D8601968EAB933
:1081A00021F04001196019498B421DD018494FF444
:1081B0007410C860196841F01E011960596941F0D6
:1081C00080015961196841F00101196022B90E4A14
:1081D000D36A43F00803D362F0BC704741F040011A
:1081E00019600A498B42E1D14FF0746041F8500C9C
:1081F000E0E744F01A04EC63EC6A44F00804EC6233
:10820000C1E700BF68190120002C014058640240FA
:108210000064024011480023024611780632032907
:1082200016D00133062BF8D10D49CA6D052A0ED0A0
:1082300002EB4203013200EB4303CA65032040F224
:10824000EB3140F2FF32187059809A8070477047C6
:1082500003EB430300EB4303F0E700BFA019012049
:1082600068190120124B30B41D6E6B6A28B943EABD
:1082700001430020AB6230BC7047AC6A013803EBAD
:1082800014440BD0002303F14002013305EB8202BA
:10829000DBB25268834204EB1244F4D3403044EA28
:1082A000014405EB80004460002030BC704700BFF3
:1082B00068190120037870B42BB30246C0F10105A0
:1082C000531912F8014FDBB2002CF9D101335B00D6
:1082D0000E4C03220B8084F8643484F86524017802
:1082E00079B1022300265A1CE518023354FA82F2AF
:1082F00085F86414DBB282F8646410F8011F002969
:10830000F1D170BC70470223E2E700BF6819012079
:10831000826D136A5B681B78FF2B08D090F8F030F1
:10832000013BDBB280F8F0301BB101207047002028
:108330007047126A0220526813707047F0B40F4BF6
:10834000C40800F0070700221E5D03EBD005BE4005
:10835000F6B2C7F1080300278B4228BF0B46C3F1D2
:1083600008049A40C91A46FA04F415F8016F42EA63
:108370000402EED11046F0BC704700BF0C1F012074
:1083800030B5EFF31181802383F312880A4AD2F8C3
:108390005836D2F85C46D2F85806D2F85C56CAB2C3
:1083A00082F31188013BA84294BF4FF40060002083
:1083B0001B1B184430BD00BF68190120012380F841
:1083C00051307047014BD3F860067047681901209F
:1083D00001207047024BC3F86426C3F86816704743
:1083E00068190120024BC3F86C26C3F87016704759
:1083F0006819012070477047212870B505D02228E0
:1084000029D0202810D0002070BD0029FBD0072AD9
:10841000F9D1184B18791C685A799B79087100209A
:108420000C604A718B7170BD0029ECD0072AEAD12B
:108430001148104B0C680E794D79D0F8682689796F
:108440001C601E715D719971002ADCD02146D0F844
:1084500064069047D7E70029D5D0022AD3D1064A2F
:10846000D2F87036002BCED00988D2F86C06984727
:10847000C9E700BF000001206819012000207047F3
:1084800003460A2201481A80704700BF08000120F5
:108490000346642201481A80704700BF140001207F
:1084A000012901D000207047014BD3F890301847C4
:1084B00000000120012901D008F0A4B9014BD3F834
:1084C0008C30184700000120014BD3F88830184742
:1084D0000000012010B40B780A46044603F00303A1
:1084E000012B05D0022B0BD000205DF8044B704708
:1084F0008B8843B9204611465DF8044B0BF09EBCB7
:108500008B88832BF6D0034B5DF8044BD3F8803077
:10851000184700BF0000012038B5054B04460D4642
:10852000DB6F98472946204608F026FF002038BD1B
:108530000000012038B5054B04460D469B6F984757
:108540002946204608F050FF002038BD00000120D9
:10855000F0B4002452004E1C2746030FB0F1204F08
:108560004FEA001003F1300503F1370334BF0D5516
:108570000B5537550234A242EFD1F0BC704700BF13
:10858000024808B5FFF796FE014808BDA45B06083F
:10859000CC1D0120024808B5FFF78CFE014808BD3C
:1085A000B45B0608CC1D01200B481A220B4B006857
:1085B0001B680A80C01801D109487047094B08227E
:1085C000094910B51C68FFF7C3FF0422074920467C
:1085D000FFF7BEFF024810BD107AF01F187AF01F97
:1085E000B0000120147AF01FB2000120C200012067
:1085F000024808B5FFF75EFE014808BDC05B0608EB
:10860000CC1D0120024808B5FFF754FE014808BD03
:10861000CC5B0608CC1D0120042301480B80704769
:10862000CC00012000487047F41E0120004870472C
:10863000F41E0120034B93F88805032894BF002003
:108640000120704768190120034B93F8880503281F
:1086500094BF00200120704768190120034B93F854
:108660008805003818BF0120704700BF6819012035
:10867000034B93F88805003818BF0120704700BFEE
:108680006819012098B182680C4B12B107229A70C8
:10869000704718780421DA6003281A611A750CBF34
:1086A00080224FF480729970C3E901227047034B16
:1086B000012241F2E4715A705A5470470C7501203E
:1086C0000378022B0FD0006908B9012070470E4BC8
:1086D0001B78032B12D080B24FF6F773984294BFE9
:1086E000002001207047084941F6500243688A582B
:1086F000B3EB422F2CBF012000207047034B984260
:1087000094BF0020012070470C750120F7FFFF0F78
:1087100030B40378022B13D0104A41F64801436865
:1087200041F63C04555802F5C25100692B400968D6
:10873000023812595B0A01FB003030BC104470470C
:10874000064B41F6300441F6340142681859595835
:1087500000EB410030BC00EB522070470C7501204B
:10876000826D0346126A52681278FF2A0AD190F885
:10877000F020002A02F1FF3214BF0120022083F80A
:10878000F02070470020704738B540F48062074CF5
:108790000B4640F2FF55012100F03F00A563A360A6
:1087A000E2604EF00FFAA56338BD00BF002C014017
:1087B0002DE9F843884600294FD04718461E284C1B
:1087C000802507F1FF39EFF3118185F31288D4F882
:1087D0005826C9B2D4F85C06D4F85836D4F85CC62A
:1087E00081F31188634594BF4FF400630023121A8C
:1087F0001344012B1AD1012035F020F9EFF3118138
:1088000085F31288D4F85826C9B2D4F85C06D4F897
:108810005836D4F85C7681F31188BB4294BF4FF48C
:1088200000630023121A1344012BE4D0EFF31182EA
:1088300085F31288D4F85C36D2B216F8011F2344AF
:1088400083F87416D4F85C360133C3F30A03C4F812
:108850005C3682F311884E45B5D14046BDE8F883B9
:1088600068190120F8B5002390F8505080F8503076
:10887000CDB10F4941F2E8028A5C032A15D10D4EB1
:1088800000F13C04B76A29462046FFF791FFB36A1E
:108890002D1A0444DB1B322B01D8002DF3D1B5FA7D
:1088A00085F04009F8BD0120FCE71846FAE700BF53
:1088B00068190120602A0120002280F85120D1E7A8
:1088C00090F85020531C0244DBB280F8503082F8FC
:1088D0003C1090F851200AB1132B00D9C2E7704721
:1088E000F8B5144641F2E803094A0D46D35C032B60
:1088F0000DD1084EB76A002C09DD21462846FFF746
:1089000057FFB36A241A0544DB1B322BF3D9F8BD99
:1089100068190120602A012010B5074C04F2BC50F0
:108920003BF074F90A2035F07DF8D4F8C405BDE8B1
:10893000104038F011B800BF6819012030B500238D
:108940008DB0124A082102930DF107058DF81430FD
:108950000124099302F2BC508DF828300B9382F861
:1089600054166944CDE90733094BCDE90354069306
:108970003AF00EFF07483BF049F99DF80700A0F1D7
:10898000FF00B0FA80F040090DB030BD6819012039
:1089900011830008241F0120F0B503798BB0284C07
:1089A000002B14BF0122002284F8B42503D184F8DF
:1089B00088350BB0F0BD04F2BC56054690F90010A6
:1089C00030463AF0EBFFAD7875BB01271D4B1E48D2
:1089D000C4F85036C4F8C45584F8C8753BF01CF888
:1089E00003464FF47A70A4F8C03535F027F8D4F870
:1089F000C40537F0B1FF28226846002154F0C4FABC
:108A00000A236946304602933AF0C2FE30463BF0F4
:108A1000FDF80E4B002284F888759B6A84F87C254B
:108A2000C4F878350BB0F0BD284637F0CBFD0546CD
:108A300008B11E23C3800D21284637F04DFEC4E740
:108A400068190120CC1E0120801A0600602A01202E
:108A500070B5952592B0044640F0400601AA080C76
:108A60008DF809500D0E8DF80810090A00238DF8B5
:108A700005508DF8060006250DF103008DF807104E
:108A800003920121174A8DF8046004938DF8183081
:108A90008DF82C300F938DF84030119305950C9282
:108AA000CDE90733CDE90D33CDE90901FFF746FFE5
:108AB00024B180F0010010F0FF0F10D10A4C082300
:108AC00003A904F2BC5084F854363AF061FE04F273
:108AD000BC503BF09BF89DF8030012B070BDFF2026
:108AE00012B070BD618700086819012030B50023FD
:108AF0008DB0104A014602930DF107058DF8143030
:108B00000124099302F2BC508DF828300B9382F8AF
:108B1000541602A9CDE90733074BCDE90354069358
:108B20003AF036FE05483BF071F89DF807000DB0AD
:108B300030BD00BF6819012061870008241F012093
:108B400070B590B01C4D0024FD220DF103030126E9
:108B500001A905F2BC508DF803200693C5F88445A1
:108B60008DF81040059407948DF824408DF8384016
:108B70000F9403960896CDE90144CDE90A44CDE966
:108B80000C443AF005FE05F2BC503BF03FF830468D
:108B9000FFF7ACFFFF2809D0084A20460923926A54
:108BA00085F88835C5F8782510B070BD04230220FB
:108BB00085F8883510B070BD68190120602A012041
:108BC00070B5064690B008200D46FFF78FFFFF28CE
:108BD00022D0FE2802D0022010B070BD0024022353
:108BE00001A90F48089301948DF8104007948DF85F
:108BF00024408DF838400F94CDE90265CDE9054455
:108C0000CDE90A44CDE90C443AF0C2FD04483AF0FB
:108C1000FDFF204610B070BD012010B070BD00BF38
:108C2000241F01202DE9F84F484B98420FD003F53F
:108C30006853083398424DD00023454A1846A2F89D
:108C40009430A2F8A030C2E92633BDE8F88F404C3A
:108C5000022300263F4F04F13005DFF80481E36270
:108C6000D7F8D0303146B34206F1010603D0D4F82C
:108C7000B00047F047FD94F8B4302846D4F8B0204F
:108C8000414685F82430303545F8102C47F04EFF2A
:108C9000E36A9E42E4DB002384F8A230E36A012009
:108CA000E16BA28EA56B12FB03F201FB03F3B4F898
:108CB0004060A4F89420C4F89C30E28E264BC4F89F
:108CC000C010C4F89850A4F8A060A4F89620C4F886
:108CD0009030BAE71E4C02224FF0000B1D4F04F1FA
:108CE00030054FF4806A4FF040094FF40068E262AB
:108CF000D7F8D020012659465A45B34403D0D4F8BA
:108D0000B00047F0FFFC4FF00062D4F8B0104FF411
:108D1000003094F8B4C0296285F824C0A5F804A0F6
:108D2000A5F81090A5F80680AE74C5E90202FFF719
:108D300071FA28466E7647F045FEE26A074B934586
:108D400045F8303BD4DB84F8A260A7E71971EF0047
:108D5000602A012000000120A4D2050878D205086D
:108D60001940EF0010B50C4647F0FCFA50B9074B1C
:108D700093F8C430012B4FF012030CBF0448054890
:108D8000238010BD12230448238010BD602A0120D7
:108D9000FC000120E8000120D40001202DE9F84367
:108DA0001C4C05468946904694F888651F46042E5B
:108DB00008D0082E02D00020BDE8F883FFF7C0FEDF
:108DC0000228F8D1D4F8C40537F0C0FD94F87E35F8
:108DD000B3B969021120FFF73BFEB8B90E4A05236B
:108DE0000120C4F86495926AC4F86855C4F8708587
:108DF000C4F87475C4F8782584F88835BDE8F8831C
:108E000029461120FFF724FE0028E7D0FFF784FD54
:108E1000D1E700BF68190120602A012010B50D4C70
:108E2000002394F85626C4F8843512B10A4AC2F8D1
:108E3000C8304EF0D3F820B10423022084F88835DE
:108E400010BD054A0923926A84F88835C4F878254C
:108E500010BD00BF68190120602A012070B50F4DB8
:108E600004460E4695F88835042B0BD0082B07D105
:108E7000D5F8803583420ED0FFF7D0FF022801D00D
:108E8000012070BD08230220C5F88465C5F880451F
:108E900085F8883570BD022070BD00BF68190120BB
:108EA00010B509F057FA104C58B194F88835032BD7
:108EB00013D894F87C350133DBB2072B84F87C356A
:108EC00003D9002384F8883510BD084B01229B6A22
:108ED00084F88825C4F8783510BD05483AF09CFD23
:108EE000A4F8C005E5E700BF68190120602A012049
:108EF000801A060070B51F4C06460D4694F888355A
:108F0000042B09D0082B25D1D4F8803583422FD0EB
:108F1000FFF716FE02281DD1D4F8C40537F016FD60
:108F200000213720FFF794FD29461720FFF790FD19
:108F3000C0B994F87E357BB971021920FFF788FD1E
:108F400080B908230220C4F88455C4F8806584F8E9
:108F5000883570BD012070BD31461920FFF778FDBE
:108F60000028EED0FFF7D8FCFFF79AFF032070BD72
:108F7000022070BD6819012070B50379234C002BC5
:108F800014BF0123002384F8B43503D1002384F8EF
:108F9000883570BD1E4D0021032095F9CF203AF091
:108FA00009FB0028F2D0466830463AF02FFB84F8DF
:108FB00055060028EAD095F8CD303046003B18BF62
:108FC000012384F856364DF0A1FB09F0C3F938B9F6
:108FD00094F87C3584F88805013384F87C3570BDBD
:108FE0004EF0D6F840B194F87C350022013384F875
:108FF000882584F87C3570BDAA6A012384F87C0535
:10900000C4F8782584F8883570BD00BF6819012040
:10901000602A012010B54EF0BBF858B10C4C94F802
:109020007C350133DBB2072B84F87C3503D9002370
:1090300084F8883510BD09F08DF90028F7D0054B6C
:1090400001229B6A84F88825C4F8783510BD00BFDA
:1090500068190120602A01202DE9F84F904C94F8FE
:10906000B455002D00F0028194F8882502278D4E1A
:10907000531E082B3ED8DFE803F03436A73D66497F
:10908000153D05004DF0AAFF002840F00181D4F8FD
:109090007835B26AFA33934229D2FFF7BBFF94F8CE
:1090A0008825E5E74DF09AFF0028F0D0D4F8843504
:1090B0000022012B84F87C2540F2EE80D4F8801544
:1090C000013B94F856560131C4F88435C4F8801534
:1090D00015B1744BC3F8C8200823054684F88835B9
:1090E00011E084F888754DF079FF00284DD194F88F
:1090F0008825531EDBB2022B3CD9082A18BF042A4C
:109100000CBF012500252846BDE8F88F236B002BF6
:1091100037D1644B0722D4F870559B6A84F88825B0
:10912000C4F87835002DEED0D4F874350120D4F889
:109130006425D4F86815A847D9E7D4F87835B26A19
:10914000643393421DD2D4F82C80B8F1000FF4D1CF
:109150004DF044FF0028A2D00423D4F8705584F8C1
:109160007C8584F88835002D00F090804046D4F846
:109170007435DCE74B4BD4F878259B6A9B1AC82BD7
:1091800079D800252846BDE8F88F4DF0B9FB0028B6
:10919000ADD196F8D130002BA3F10203B3FA83F3DB
:1091A00014BF022201225B0984F87D2584F87E35F4
:1091B0004DF0A6FB00287FF470AFD6F820210323E2
:1091C000C4F88C2584F888354DF09AFB00288ED1A0
:1091D000344A4FF0040EC4F88405032392F804B116
:1091E000B2F80611D2F8080184F892B5D2F80871E5
:1091F0004FEA106CD2F80861A4F890153F0CD2F831
:1092000008A1360A92F80C9192F80D5192F80D01CE
:10921000D2F8108125FA0EF5B2F816B100F00F0061
:10922000B2F81611B2F81621C1F30B1184F893C5E8
:1092300002F00F0C84F8947541EA1B21724684F801
:10924000956501F00F0184F896A584F8979501F5CE
:10925000FA6184F89C5584F89D05C4F89885A4F8B3
:109260009E1584F8A0C584F888E543E7284684F86D
:109270008855BDE8F88FFFF7CDFE94F88855082D86
:1092800018BF042D0CBF012500253CE705463AE731
:10929000042384F8883536E7FAD1FFF7BFFD26E7C7
:1092A00068190120602A01202DE9F8430546884607
:1092B00017461E462A4C94F88805042835D00828FD
:1092C00007D1D4F88035AB4206D0FFF739FC02282D
:1092D000F1D00120BDE8F883FC22224BDFF88C900E
:1092E000214883F83021C9F838813AF081FA002802
:1092F00009F588711C4814BF4FF400734FF4807354
:10930000C9F840313AF044FA012206230020C4F89B
:109310006485C4F86855C4F87075C4F8746584F839
:109320006C2584F88835BDE8F883D4F8C40537F097
:109330000DFB94F87E3553B969021820FFF788FBBE
:1093400038B994F88835082BC6D0FE22C5E72946DF
:10935000F3E7FFF7E1FAFFF7A3FD0320BAE700BF49
:1093600068190120602A0120241F0120000001202B
:109370002DE9F04FD84C95B094F8B465002E00F06C
:10938000998194F8882504F2BC57DFF8508304F2E1
:10939000A459531E082B00F2A080DFE813F034001C
:1093A0005E0029019E008C00AF001B009E0009009A
:1093B000FFF7C4FA002840F05482D4F87835D8F882
:1093C0002820FA33934280F08580FFF769FD94F8F6
:1093D0008825DEE7FFF7B2FA0028EED0D4F884350E
:1093E0000022012B84F87C2540F26082D4F880258D
:1093F000013B082106460132C4F8843584F88815FB
:10940000C4F8802552E1D4F8C40537F09FFA002152
:109410000846FFF71DFB0546FFF77EFA012D59D1DF
:109420004FF0000AD4F8C40584F87DA537F08EFA11
:1094300040F2AB110820FFF70BFB052800F09081EC
:10944000012800F05181FFF767FA94F87D35002B71
:1094500000F02882022384F88835D4F8C40537F058
:1094600075FA94F87D3500213720022B0CBF4FF0A0
:1094700080450D46FFF7ECFA29202946FFF7E8FA68
:109480000546FFF749FA2DBB94F87D35022B00F015
:10949000988184F87E55D4F8C40537F057FA002136
:1094A0000920FFF7D5FA002871D0FFF735FA94F8B4
:1094B0008825531E11E04FF40071D4F86405FFF7BE
:1094C0007FFB012800F03081022800F03581002860
:1094D00000F0618194F88825531EDBB2022B00F264
:1094E000DF807E4BD4F878259B6A9B1AC82B00F24C
:1094F000E7800026304615B0BDE8F08FD4F8BC35C3
:1095000077481D6A3AF074F9002800F02C81B5FA0A
:1095100085F56D09002DDDD004A800250DF10F03A0
:1095200002224FF0010A05A9059038460792ADF8CE
:10953000105006958DF820508DF834508DF8485015
:109540001395CDE90B3ACDE90955CDE90E55CDE995
:1095500010553AF01DF938463AF058FB9DF80F3097
:1095600003F01F03052B00F08581FFF799FCD4F869
:1095700070B5BBF1000F00F0F0802A465046D4F8D9
:109580007435D4F86815D84794F8882501E7102178
:109590004846FFF715FB8246002886D101217F202F
:1095A000FEF7CCFE012805467FF47FAF504602212E
:1095B000FEF7C4FE002800F0358101287FF475AF66
:1095C00016213A20FEF7BAFE01308002C4F88C055D
:1095D000FFF7A2F9D4F8C40537F0B8F900210A2042
:1095E000FFF736FA002840F01681032384F8883507
:1095F000102105A8FFF7E4FA00287FF46BAF9DF86F
:1096000021309DF822201B019DF815009DF8165071
:1096100002F00F01DBB245EA0025DDF81D0043EA48
:1096200012139DF81C2000BA84F8A01503F5FA6304
:109630009DF81710C4F89805A4F89E3513099DF8F5
:10964000140002F00F0284F89C35069BA4F8905594
:10965000C4F8943584F89D2584F8920584F8931510
:10966000FFF75AF994F87E3573B9D4F8C40537F08A
:109670006DF94FF400711020FFF7EAF90546FFF786
:109680004BF9002D7FF4A1AE16483AF0C5F900223F
:109690000423A4F8C005C4F884251A4684F8883544
:1096A000082A18BF042A0CBF01260026304615B030
:1096B000BDE8F08F304684F8886515B0BDE8F08FBE
:1096C000FFF7EEFB94F88865042E18BF082E0CBF38
:1096D00001260026EAE700BF68190120602A012060
:1096E000241F012040787D01042304AA05A977489E
:1096F00007930692CDF814A08DF820A08DF834A021
:10970000CDF838A0CDE909AACDE90BAA3AF040F886
:109710006E483AF07BFA9DF81330AB2B7FF493AE92
:10972000022384F87D358EE6D4F87835D8F82820E1
:1097300064339342BFF4CEAEFFF7EEF8FFF7B0FB11
:10974000D4F870554DB10022D4F87435D4F86815AA
:109750001046A84794F888251BE694F8882518E653
:1097600084F87D556FE694F86C550246D4F864157C
:109770004FF48073384601EB05213AF02DFA94F846
:109780006C250132D2B2A2F1020584F86C25B5FA3B
:1097900085F56D09BEE60190FFF7BEF80423019838
:1097A000D4F8705584F87C0584F88835002D3FF492
:1097B0007DAFD4F87435D4F86425D4F86815A8477B
:1097C00088E6D4F8C40537F0C1F829463A20FFF7F7
:1097D0003FF904AA0423824605A9384605958DF869
:1097E00020508DF834500E95CDE90955CDE90B5533
:1097F000CDE9062339F0CCFF38463AF007FABAF142
:10980000000F08D1FFF788F8049B1BBAC3F38073DD
:1098100084F87E353FE6FFF77FF8FFF741FB94F8C9
:109820008825B6E504212C20FEF788FD0321824619
:109830004E20FEF783FD83460C213620FEF77EFD89
:109840000BF1020B421C05FA0AF502FA0BF2A2FB1D
:109850000501420A42EAC152C4F88C25FFF75CF8C0
:10986000B8E60190FFF758F80423019884F888358A
:1098700006461BE7164B0722D4F870659B6A84F8EE
:109880008825C4F87835002E3FF410AFD4F874352D
:109890005046D4F86425D4F86815B04794F8882564
:1098A000531E1AE61E4684F88835FFE608D00423C6
:1098B00084F88835FFF730F894F88825531E0CE6B5
:1098C000FFF73EF902287FF405AEEEE5241F0120E4
:1098D000602A0120154BDB68C3F3022310B4C3F1E7
:1098E00007041A1D042C28BF0424062A4FF0FF3257
:1098F0008CBF033B0023A240002821EA020101FAA9
:1099000003F108DB09010A4BC9B2034483F80013D1
:109910005DF8044B704700F00F000901054BC9B218
:10992000034419765DF8044B704700BF00ED00E07A
:1099300000E100E0FCEC00E030B5264C00222648B7
:1099400041F28731D4F8743183B0244DA0FB030376
:1099500004F59A70C4F83451DB0C013BC4E9501291
:10996000C4E94E320CF080FA1D4B062137201A6CE8
:1099700042F020021A641B6C03F020030193019B48
:10998000FFF7A8FFD4F834314FF400001549164A08
:109990004860D96841F00101D96099680A40062AF7
:1099A00006D0B2F5803F03D01A6842F001021A6077
:1099B0000E4B41F2041200200D499A5803F27464D0
:1099C000C3F87006C2F81002C3F86806C2E9811431
:1099D00003B030BD602A012083DE1B430014004029
:1099E0000038024000E100E0070001006819012092
:1099F000D82B012038B50F4B0F4AD3F87431A2FB96
:109A000003239B09013BB3F1807F10D20B4A002452
:109A1000F0200B490725536081F82300214694600C
:109A20004FF0FF301560FFF755FF204638BD01208D
:109A300038BD00BF602A0120D34D621010E000E065
:109A400000ED00E04309012200F01F0084B0013B5B
:109A500002FA00F0032B0BD8DFE803F015021E0C0E
:109A6000124B5A6C02435A645A6C10400090009B8F
:109A700004B070470D4B1A6B02431A631A6B104007
:109A80000390039BF4E7094B5A6B02435A635A6BEA
:109A900010400290029BEBE7044B1A6C02431A64DD
:109AA0001A6C10400190019BE2E700BF00380240B1
:109AB0002DE9F041D0F800E00C46DFF8588084B082
:109AC000DEF804501746DFF850C0194605EA0805CD
:109AD000DDF82880064603932C43424644EA0C0CEA
:109AE000CEF804C009F000FB78B931680246039B48
:109AF00030468F624021CDF8008009F025FB003808
:109B000018BF012004B0BDE8F081012004B0BDE819
:109B1000F08100BF009800FC00200180F8B5134FD1
:109B200004460D460AE09B69DB0602D509F09CFA63
:109B3000D0B9D7F878395B1B0A2B08D823682A4696
:109B40000A2120469E69B606EDD50020F8BD636C5B
:109B50002021002201200B4384F84020636484F814
:109B6000411084F84220F8BD0120F8BD602A012090
:109B70002DE9F04788B0884615461F46064639F05D
:109B800051FC041E30DB224BDFF890901A19B1888B
:109B900009EB840492F858A0C4F87C895EB14FF0B8
:109BA0000042B1FA81F0C24005D01A48046824EAA4
:109BB00002040460426103EB870305F0030230688E
:109BC000C5F341149B6E0026C5F38105D1441343B0
:109BD000039103A907960695CDE9043408F0A8FD82
:109BE00099F8BC39F02B02D808B0BDE8F0870A4AD2
:109BF000F023032112F90A0089F8BC390190FFF71C
:109C000069FE019808F0B8FB08B0BDE8F08700BF16
:109C100078D20508003C0140345C0608602A012027
:109C200010B4B8B10D4CD4F8C439102B05D10521AE
:109C300000205DF8044B39F0C5BB03EB430222441E
:109C400082F8C919012182F8C8090B4482F8CA199F
:109C5000C4F8C4395DF8044B704700BF602A012086
:109C600020218078DCE700BF2DE9F04FC14C0023B4
:109C700087B004F6F81894F80C2AC4F8F839C8E943
:109C80000133C8E903331AB194F80D3A84F8F8396E
:109C900094F80E3A1BB194F80F3A84F8073A94F806
:109CA000123A1BB194F8133A84F8023A94F8103A35
:109CB0001BB194F8113A84F8FD3994F8143A013B39
:109CC0005FB2DBB2019702933B46013300F04F8154
:109CD000A94EB0220023A94802FB076106F5217AAC
:109CE000A0F128050093743106F53F7953F0DAF8B6
:109CF0000122009B2E4602FA07FB1F46307890B3E4
:109D00009F494FF0300C03E089452CD011F808CF63
:109D10006045F9D14A7812EA0B0FF5D036F052FCC3
:109D2000FB1DDBB210B100218371C171032136F03C
:109D3000D3FC30780023302101E01AF83310884238
:109D400000F0B2810133102BF7D14FF0000C009AD4
:109D50000121072086F801C0531CB270F170DBB2FC
:109D6000307100930B4601370536042FC6D194F8A5
:109D7000240A01270393FFF765FE4FF44031814E1B
:109D80000022009BC4F82C1A3046D4F8201AC4F8DC
:109D9000443AC4F8407AC4F8387A84F8587AC4F857
:109DA000302AC4F8502AC4F8542AC4F8342A84F853
:109DB000482AC4F84C2AC4F83C2AC4F8281AFEF7EA
:109DC0001FF9019B002B40F0EF80039B002B00F05C
:109DD000EB80A6F1080050F0E5F9012308F1140822
:109DE0004FF0000A9B46EA78002A40F017810535BB
:109DF0004545F8D1019B02200299234493F91C2A7E
:109E000039F0D8FB0546002800F0B180406839F0F1
:109E1000FDFB0022062139F009FC002800F0A78094
:109E20006868002739F0F2FBDFF874814FF004FF17
:109E3000009B6A68012B4FF40063A8684FF400553B
:109E40008CBF4FF480613946C4F8702A4FF4003259
:109E5000C4F8801A4FF48071C4F8843A0323C4F81C
:109E6000740A4046C4F8983AC4F8787AC4F87C7A00
:109E7000C4F8947AC4F89C7AC4F8A07AC4F8885AD2
:109E8000C4F88C1AC4F8902A0BF03CFE94F8643A9B
:109E9000C4F8608A012B0597C4F8A86A67D001232B
:109EA000D4F8285A84F8643AAB68DE0713D4D4F89F
:109EB00074313549AA68B3FBF1F342F0010203EBB8
:109EC0004303AA600593059B2BB1059B013B0593BA
:109ED000059B002BF9D1AB68D80748D5D4F8682A80
:109EE0002A4B134043F48073C4F8683A6B685905F1
:109EF00007D5D4F8683A23F4405343F48053C4F8A8
:109F0000683AD4F8683A13F4805300F03881D4F8F2
:109F10006C3A23F00603C4F86C3A1D4800231D492F
:109F20006FF02202C4F8B00A1B4884F8643AC4F8FF
:109F3000AC1A05F14C01C4F8BC0A2A606E68009B9B
:109F400046F08066154A16486E60AE6846F4807624
:109F5000AE600BF04BFD134B5A68D20640F0F88010
:109F6000D4F8283A9A6812F0405F00F0038107B0F5
:109F7000BDE8F08F602A012078D2050880340120E6
:109F8000FCD405088834012040420F00FEF8FFFF92
:109F9000890C01088D0C0108790C0108E4010020EE
:109FA000D034012000230140B02200217B48482703
:109FB00052F0EAFFB0220021784852F0E5FF784BDA
:109FC000384684F8D47AC4F8D03AFFF73BFD4FF412
:109FD000403000230121D4F8D02AC4F8DC0A7148AB
:109FE000C4F8F01AC4F8E81A84F8081BC4F8E03A78
:109FF000C4F8003BC4F8043BC4F8E43AC4F8F43AAB
:10A0000084F8F83AC4F8FC3AC4F8EC3AC4F8D82A10
:10A01000FDF7F6FF614850F0C5F8DEE694F8640AF3
:10A020005A1C69780128D2B22F79CDF810A039D006
:10A03000092984F864BA52D94FF0030E6FF01D005D
:10A04000D4F828CA4FF007091EFB0100DCF80CE029
:10A0500009FA00F907FA00F02EEA0907CCF80C70AB
:10A06000DCF80C703843CCF80C00062B4FF00500E0
:10A0700020D86FF0040710FB0373D4F8287A1F2050
:10A0800000FA03FC786B01FA03F320EA0C00786312
:10A09000786B03437B63D4F8283A4148834234D039
:10A0A00084F864AA1346A2E63F4A02EBC30393F87E
:10A0B00088C24CE60C2B32D86FF0220710FB0373DA
:10A0C000D4F8280A1F2707FA03FC076B01FA03F3E9
:10A0D00027EA0C070763076B3B430363DBE7D4F80E
:10A0E000280A01EB41094FF0070ED0F810C007FA1B
:10A0F00009F70EFA09FE2CEA0E0CC0F810C0D0F8D1
:10A1000010C047EA0C070761AFE712291AD01129DE
:10A11000C6D126494B6843F400034B60C0E76FF09B
:10A12000400710FB0373D4F8280A1F2707FA03FC23
:10A13000C76A01FA03F327EA0C07C762C76A3B4301
:10A14000C362A8E719494B6843F480034B60A7E753
:10A15000D4F8282A12498A4214D05B68DB063FF5FE
:10A1600006AF134B9A427FF402AF9A6812F0405F39
:10A170007FF4FDAE9A6842F080429A60F7E6C4F838
:10A180006C3ACAE6936813F0405F03D1936843F0DA
:10A1900080439360054B5B68E9E600BF30350120E2
:10A1A000002001403835012078D205080023014005
:10A1B000002201402DE9F041D0F800E00C46DFF824
:10A1C000588084B0DEF804501746DFF850C01946B6
:10A1D00005EA0805DDF82880064603932C4342462D
:10A1E00044EA0C0CCEF804C008F07EFF78B9316860
:10A1F0000246039B30468F628021CDF8008008F034
:10A20000A3FF003818BF012004B0BDE8F081012091
:10A2100004B0BDE8F08100BF009800FC002001817F
:10A22000034690F83C00012800F03E810220F0B483
:10A23000012483F83D0083F83C40142A45D8DFE828
:10A2400012F04D004400440044007B0044004400F0
:10A250004400DA00440044004400AA0044004400E2
:10A260004400060144004400440015001A688E684A
:10A27000156A0F6825F48015AB4C1562106A556895
:10A2800020F40010D2F854C040EA0650A74E0CEA61
:10A290000404B24244EA072400F0088106F580660F
:10A2A000B24200F003814E6855605465D665106275
:10A2B000506D0C6940F400605065506D20F4806072
:10A2C0005065516D41EA042151650022012110467B
:10A2D00083F83D1083F83C20F0BC70471A68D1F831
:10A2E00008C0156A0F6825F00105914C1562106AC7
:10A2F0005668956920F002002C408C4D40EA0C0015
:10A30000AA4244EA070400F0DD8005F58065AA4210
:10A3100000F0D8804D685660946155631062906972
:10A320000C6940F008009061906920F00400906191
:10A33000916921439161C8E71A68D1F808C0156A8C
:10A340000F6825F010057B4C1562106A56689569F8
:10A3500020F020002C40754D40EA0C10AA4244EA3F
:10A36000072400F0C38005F58065AA4200F0BE8096
:10A370004D68566094619563106290690C6940F471
:10A3800000609061906920F480609061916941EA79
:10A390000421916199E71A688E68156A0F6825F49F
:10A3A0008055644C1562106A556820F40050D2F84C
:10A3B0001CC040EA06305D4E0CEA0404B24244EA96
:10A3C000072400F08D8006F58066B24200F0888098
:10A3D0004E685560D46116641062D0690C6940F40F
:10A3E0000060D061D06920F48060D061D16941EA19
:10A3F0000421D16169E71A68D1F808C0156A0F68AD
:10A4000025F480754A4C1562106A5668D56920F4A7
:10A4100000702C40454D40EA0C20AA4244EA070453
:10A4200073D005F58065AA426FD04D685660D4613F
:10A43000D5631062D0690C6940F00800D061D06922
:10A4400020F00400D061D1692143D1613DE71A6851
:10A450008E68156A0F6825F48035374C1562106ACE
:10A46000556820F40030D2F854C040EA06402F4E20
:10A470000CEA0404B24244EA07041DD006F58066E3
:10A48000B24219D04E685560546596651062506DA1
:10A490000C6940F008005065506D20F004005065D4
:10A4A000516D2143516510E70220704725F4802546
:10A4B0004E6945EA8625F6E625F480354E6945EA7B
:10A4C0000625DFE726F4407C20F008008E69CF687F
:10A4D0004D693843354320F0040045EA0C0619E77E
:10A4E00025F480454E6945EA861571E726F4406CEF
:10A4F00020F080008E69CF684D6940EA071035432F
:10A5000020F040004CEA850632E726F4405C20F457
:10A5100000608E69CF684D6940EA0720354320F41A
:10A5200080604CEA051680E7FF8FFFFE00000140C7
:10A530008CFFFEFFFF8CFFFE8FFFFEFFF8B53D4E48
:10A5400096F8804B04EB4403670006EBC30393F8D3
:10A55000843B032B44D8DFE803F0461B0F023C4446
:10A5600006EBC404D4F8883B002B58D0013B0025EF
:10A57000C4F8883B2846F8BD3B1906EBC303D3F863
:10A58000882B7AB1013A0025C3F8882B2846F8BDFC
:10A590003B1906EBC303D3F8882B002AF2D1022221
:10A5A00083F8842B3C4406EBC40494F8903B013BB5
:10A5B000DBB284F8903B4BBB0323D4F88C0B84F8BC
:10A5C000843B52F03DFEC4F8880B064652F048FE2C
:10A5D00080F00100002E0CBF002500F0010525BB16
:10A5E00001252846F8BD3AF0F9FD05460028F7D0C8
:10A5F0003C44012342F2107006EBC40484F8843B0F
:10A6000052F01EFEC4F8880B2846F8BD01254FF411
:10A610007A7052F015FEC4F8880B2846F8BD52F047
:10A62000DBFD80F00100C5B2B0E7013EC4F8886BE5
:10A63000ACE700BF602A012003689B0AA3F58013E2
:10A64000522B00D970470E4A134470B593F8044357
:10A6500084B00D2C12D800294FF0000309494FF0A7
:10A66000010514BF1E460226427901EB841069469B
:10A67000CDE90065CDE902330BF0F6FA04B070BD08
:10A6800078D205084436012033492DE9F84F91F876
:10A69000D1101C46012507460229DFF8C4A0104648
:10A6A00019464FF00002DFF8BC9018BF7F02CAF8CD
:10A6B0002C50FDF74FFD294A630240F2FF5BC9F8B9
:10A6C00024204FF40075C9F828304FF48A62D9F875
:10A6D0002C30012110205E4643F09303C9F82C3042
:10A6E000C9F838B0C9F808504D46C9F80C204CF0EC
:10A6F00069FA012CC9F838B04FF00A048CBF4FF04A
:10A7000052084FF051084FF0000939464046FEF715
:10A710003BF8013C034640F2774201213720E4B286
:10A7200023B91846CAF82830BDE8F88FAE63C5F8DB
:10A730000890EA604CF046FAAE63034608B1002C7C
:10A74000E3D1002BEDD000221846CAF82C20CAF81D
:10A750002830BDE8F88F00BF602A012000E1F50530
:10A7600068190120002C01402DE9F843DFF87480BE
:10A7700004460F46914698F888551E46042D08D089
:10A78000082D02D00020BDE8F883FEF747FB022821
:10A79000F8D101233A4620460021FFF775FF68B142
:10A7A000FEF738FCD8F87045002CEBD00022D8F822
:10A7B0007435D8F868151046A047E3E7084A052322
:10A7C0000120C8F86475926AC8F86845C8F87095A1
:10A7D000C8F87465C8F8782588F88835BDE8F88326
:10A7E000602A0120681901202A492DE9F04F91F8CB
:10A7F000D1100124DFF8A8B00746022983B0CBF8B6
:10A8000030409A4618BF4702012B4FF00A04224DF0
:10A8100040F2FF568CBF4FF059084FF058084FF0E8
:10A820000009009239464046FDF7AEFF013C034661
:10A8300040F2774201213720E4B2BBB9009851467B
:10A8400001220193154CFDF785FC13494FEA4A227A
:10A850000020019B4C628A62CA6A42F09102CA627D
:10A86000CBF82800184603B0BDE8F08FAE63C5F8FA
:10A870000890EA604CF0A6F9AE63034608B1002CDC
:10A88000D0D1002BDAD000221846CBF8302003B00C
:10A89000BDE8F08F602A0120002C014000E1F505A1
:10A8A000681901202DE9F84F05460E4690461F46CF
:10A8B000394C94F8880504280CD0082807D1D4F81E
:10A8C0008035AB4206D0FEF7A9FA0228F1D001206C
:10A8D000BDE8F88FDFF8C8A0C4F86465DAF8C8905E
:10A8E000C4F86855C9F34F234FEA59220F2B2BD8D0
:10A8F000D4F884B5BBF1000F26D094F8561619B3DE
:10A90000B9F5005F41D025484FF400723146484404
:10A9100052F0C8FA09F50072C2F34F23CAF8C820F2
:10A92000520A102B31D0BBF1010F2ED0D4F8802564
:10A930000BF1FF33042102200132C4F8843584F87E
:10A940008815C4F88025C3E701234FF00109284684
:10A95000062532460021C4F87085C4F8747584F861
:10A960006C9584F88855FFF73FFF0028B0D0FEF7BC
:10A9700051FBD4F870556DB14846D4F87435D4F80D
:10A9800068150022A8470320A2E792B2034E013ABD
:10A99000AD1ADAE703209BE7681901200C55012066
:10A9A000602A012070B50D4C1346D4F8A45F2A78B4
:10A9B000022A07D00A46014604F6A470BDE870409A
:10A9C00039F086BF2A6A0AB1002070BD0A460146E6
:10A9D00004F6A47039F080F8012070BD602A0120CF
:10A9E00003681878012801D00020704793F90430DB
:10A9F000074A03EB430302EB431313F8332C202ADB
:10AA0000F3D153F8743C9869C0F3C030704700BF6D
:10AA1000583B0120036801221B78022B01D03AF039
:10AA200081B939F0B1B810B50B4CD4F8A43F1B78FC
:10AA3000022B10D1D4F8AC0F35F08EFFD4F8AC0F48
:10AA400008B12123C380012135F046FE034838F0C8
:10AA5000E3FFA4F8A80F10BD602A0120809698009B
:10AA600030B5044683B001230D460DF107020848B6
:10AA7000214639F02DFF9DF8072035EA020304D066
:10AA80002A43214602483AF001FA03B030BD00BF24
:10AA9000043A012038B505460A460C4606482946C0
:10AAA00039F04AF845F08001034838F0C9FF231A0D
:10AAB0005842584138BD00BF043A012013B53A4C02
:10AAC0000023D4F804218DF80730137803F0FD013A
:10AAD000012905D194F8081111B90C2184F8081145
:10AAE000022B1ED0032B2ED001220B212F484BF01E
:10AAF000E3FC042032F0A2FF01230DF10702002144
:10AB00002A484BF0FBFC002839D09DF80730482B31
:10AB100035D1274BC4F8F830264BC4F8FC3002B0CE
:10AB200010BDD4F80C0135F017FFD4F80C0108B1B2
:10AB30003523C380012135F0CFFD1F4838F06CFF6D
:10AB4000A4F80801D0E7D4F8B43546F2A81150684B
:10AB5000122219610023372180F888304BF07FFCE6
:10AB6000D4F804310D22242158684BF078FCD4F835
:10AB7000043130226A2158684BF071FCB4E7D4F8F4
:10AB800004311A78022A03D0032A07D00020C6E72E
:10AB9000D4F80C0138F0DCFD0020C0E7102237218A
:10ABA00058684BF05CFCF1E7583B01205C3C01200D
:10ABB0005B650508DD65050880969800F8B55E4C74
:10ABC00000234FF4F07206460F4604F63810202199
:10ABD00084F8343984F8353952F0D6F94FF4F072EC
:10ABE000202104F6183052F0CFF9322032F026FF3F
:10ABF00094F8F93C002B00F0948094F8FA1C04F6C9
:10AC0000FC4038F0CBFE002800F08B8094F8F90C63
:10AC100035F0D8FC0546C4F8040D35F09FFD00283A
:10AC20007FD00DB12323EB800D21284635F054FD54
:10AC3000D4F8040D35F090FE404838F0EDFE0346A0
:10AC4000FF213F48A4F8003D38F0A8FF8C213C4884
:10AC500038F0F6FE1B2867D10122D4F8043D84F8B1
:10AC600034290BB12322DA8040220A21344838F0FB
:10AC700063FF8A21324838F0E3FE94F8F83CC0F3D1
:10AC8000801584F8945D002B44D0022B3BD12D48D5
:10AC900038F0C2FE0346A4F8960D94F8982D182AB1
:10ACA00011D1294A2949D2F87421A4F89C7D52086F
:10ACB000A4F89E5DA4F8A03DB2FBF3F2A1FB021242
:10ACC000520BA4F8A22D1E4802220021A4F8003D38
:10ACD00038F032FFC8201A4D32F0A4FE80212846F9
:10ACE00038F0AEFE10F00200F8D17278B378317807
:10ACF000C2F12002C3F1100384F8A52D84F8A63D0B
:10AD000084F8A41DF8BD124838F086FE0346A4F866
:10AD1000960DC2E7094838F07FFE0346A4F8960D69
:10AD2000BBE76FF00100F8BDD4F8040D202135F029
:10AD3000D3FC4FF0FF30F8BD583B0120404B4C0096
:10AD400054480120002D3101602A01205917B7D144
:10AD5000809698000146014838F072BE00490120F3
:10AD600030B40023314D32494CF25034C5F8583ECE
:10AD7000304AD1F8780904E0D1F878391B1AA34297
:10AD80000FD8D368DB03F7D4D16811F4F9710BD174
:10AD9000D06810F0010002D001230846D36030BC17
:10ADA0007047032030BC7047D3689B0705D5D5F8A2
:10ADB000583E43F02003C5F8583E1E4BDB68DC06C6
:10ADC00005D5D5F8583E43F01003C5F8583E194B49
:10ADD000DB68980605D5D5F8583E43F00803C5F85A
:10ADE000583E144BDB68590605D5D5F8583E43F05C
:10ADF0000403C5F8583E0F4BDB681A0605D5D5F895
:10AE0000583E43F00203C5F8583E0A4BDB68DB05A9
:10AE100005D5D5F8583E43F04003C5F8583E054BDC
:10AE20004FF4F9720120DA6030BC7047583B0120C2
:10AE3000602A0120003C0240094B93F85E3E042B3F
:10AE400008D9053B032B08D801231A4600B103702B
:10AE50001046704700230122F8E700231A46F5E761
:10AE6000583B01202DE9F04FDFF8DC81DFF8DC9161
:10AE7000D8ED037A08F5B06399F8802EF8EE677A7A
:10AE80002DED028BC3ED007A83B0002A4ED1614EC6
:10AE9000C8F8882598F88C153278D9B1B9F8863E6B
:10AEA0000024DFED5D5A07EE103ADFED5C6A5C4B83
:10AEB000B8EE477A67EEA66A03EBC10085EE876AB3
:10AEC00036EE266A86EE867A1C60083303ED017A38
:10AED0009842F9D199F87E3E9FED525A06EE103A0B
:10AEE00096F8583B9FED507A1A44B8EEC66A27EEA2
:10AEF000877ADFED4E6A12FB01F14D4AC5EE065A24
:10AF0000C9B207EE901AF8EEE77AE7EE876AF7EE35
:10AF1000667AFCEEE77AC2ED005A17EE903A88F8AE
:10AF2000DC3603B0BDEC028BBDE8F08FFCEEE77AB7
:10AF30009FED404A99F8811EB9F8843EF8EE674AC1
:10AF400006EE101A002107EE103A324EB8EE466AAD
:10AF5000C4EE245A0191B9F8821E01239FED365A9E
:10AF600006EE901AC6ED057A98F88C15B8EEC77AF9
:10AF70009FED328AF8EE666AC8F88865327067EE2F
:10AF8000057A86ED016A88F88435C6ED036AC6ED58
:10AF9000047AC6ED025A89B3294B4FF0000B019990
:10AFA00003EB010A12B3AAF118045746002507EE75
:10AFB000905A01223846B0EE481AB8EEE70AD6EDAC
:10AFC000017AD6ED040A15447169283720EE270A64
:10AFD000283452F015F984ED028A84ED018A84ED5B
:10AFE000048A84ED038A32789542E0DB0BF1010B91
:10AFF00098F88C150AF1780A8B45D3DB019B03F591
:10B000007073B3F5346F0193C5D10E4BD3ED007A55
:10B0100043E700BFD034002083F9223EBD37863598
:10B02000E0490120555555406E12833A48E1FA3EF9
:10B03000BC0800200060EA480AD7233C000000005A
:10B04000E834002064070020E4010020583B012080
:10B0500007EE900ADFEDAF5AAF4B0022B8EE677AE9
:10B06000DFEDAE4AB3F8C81E85EE874A06EE101A29
:10B07000B3F8CC1EDFEDAA5A07EE901AB3F8CA1E39
:10B08000B8EE466A06EE901AF8EEE77AF8EEE66A4F
:10B0900036EE065A67EEA47A2DE9F04FC6FE856AB1
:10B0A000A04D2DED048BB4EEE54A05F5DC6993F86F
:10B0B000CE4E85B0C5F83007F1EE10FA89ED016A81
:10B0C000C5F8EC46C5F8F026C9ED026AC9ED007A6C
:10B0D00002D51446C5F8EC26F6EE004A9FED925ACA
:10B0E000F7EE003A914927EE055A9FED912A64EE5A
:10B0F000247A0B46F0EE002A9FED8E3A143381ED50
:10B10000045A87EEA67A01F5A677039301F12C067F
:10B1100091ED055A884A12F8542C87FE237ABDEE29
:10B12000C77AF8EEC77A17EE103A012BC5F88C39BA
:10B13000C4EE275AB8BF0123029383EEA74A65EEF7
:10B14000825A86EE257AA1EC014AC1ED005AC6EE7C
:10B15000A57A37EE247A87FE227ABDEEC77A77EE9B
:10B16000A47A17EE101AC7FEC37AFDEEE77A01F152
:10B17000FF38C5F8981917EE901AB8F1230F01F1AE
:10B180000100A8BF4FF02308C5F89C192328834667
:10B1900028EAE878A8BF4FF0230B5B468045C8BF7C
:10B1A00043460093A3EB0803019362BB624B9346B3
:10B1B000DFED629AA3F1500A9FED619A07EE90BA13
:10B1C0000BF1010B0AF1080AF8EEE78A68EEA98A8A
:10B1D000B0EE680A44F07CFEB0EE408AB0EE680A39
:10B1E00045F07AF8B0EE680A45F076F828EE098A5C
:10B1F00020EE090ABBF1240F0AED028A0AED010ACA
:10B20000DCD19FED505A019A00234F489446029A90
:10B210009FED4E7A9CFBF2FA0AF10101A246144618
:10B220008E460099324646F80C1C46E9053846E938
:10B2300002E4A2EC017A9742FBD13A4606F5107B74
:10B24000D0EDD67AD0F85CC3C2ED007A083242F86D
:10B2500004CC5A45F8D106F515763D4A07F5157721
:10B260009642DFD1039BB6EE008A5446012283ED5D
:10B27000005A4FF0000A374B4FF0000800932E4B56
:10B2800003F8542C002C35DD09EB0A06DDF800B07C
:10B29000002707EE907AD9ED016A99ED027A06EE61
:10B2A000104AF8EEE77A012237EE667AD5F83017C1
:10B2B000B8EEC66A06F1540077EE887A1744B7EE06
:10B2C000001A283667EE877A87EE860A30EE260A5D
:10B2D000ABEC010AD9ED000A51F092FFD5F8EC462B
:10B2E000C6F84480BC42C6F84080C6F84C80C6F818
:10B2F0004880CEDC009B0AF1C80A1433BAF5167FE9
:10B30000009302D0D5F8EC46BCE705B0BDEC048B49
:10B31000BDE8F08F00247449583B01200AD7233C34
:10B320000000FA44E40100209C534937740B0020CC
:10B33000398E633C00000C42DC120020C3B8B23DE1
:10B3400072F97F3FBC297E3F78D2050800000000DB
:10B350009C120020D80800200848002302461178DB
:10B360000632022904D00133062BF8D100207047A1
:10B3700003EB430300EB4300704700BFA01901201B
:10B380000021094B00B5084683B0C3F8D01E29F050
:10B39000B1FE0422054B06200DEB0201019329F0BA
:10B3A0009DFE03B05DF804FB583B01205475C52A8F
:10B3B00070B5461E00F13105344614F8011F601EB9
:10B3C000FF29A0EB060002D0C0B229F093FEAC42E8
:10B3D000F3D1A02040F2E93445F056FF01210220CC
:10B3E00029F088FE01E0013C04D04220FFF7B2FCC6
:10B3F0000028F8D16220FFF7ADFC1321242029F0AA
:10B4000079FE2520092129F075FEA020BDE87040B5
:10B4100045F03ABF30B54CF205028DB0002304462A
:10B420000321ADF8002001AD01228DF802300B930D
:10B430008DF814208DF82820CDF808D0CDE90633FA
:10B44000CDE90833CDE9035138F0E0FB204602A9ED
:10B4500038F09EF9204638F0D9FB9DF806000DB073
:10B4600030BD00BF2DE9F043734E83B0734C2422EE
:10B47000002106F1380051F087FD002394F8D55ED5
:10B48000F365002D37D16E4FD7F8903043B39B6AE8
:10B4900033B36C489847836813B3038800246A4F1A
:10B4A000013BBC4639469BB20878063103281BD0C5
:10B4B0000134062CF8D1002239780637022900F031
:10B4C0009D800132062AF7D1F16D052908D002FBD3
:10B4D00001C20131F165022000219380107051807A
:10B4E000284603B0BDE8F083062303FB0464638FA2
:10B4F000013B9BB2DFE704F6DC6794F8D40EC4F896
:10B50000D87E10B900254E4FBEE735F05BF8C4F881
:10B51000E40E35F023F90028F4D02946384638F0F7
:10B520003DFA05460028EDD0D4F8D83E454A986843
:10B53000C3F8942008B12023C3800D21404F35F07B
:10B54000CBF8D4F8D83E4FF00109986835F004FAEA
:10B550003E4838F061FAD4F8D83E024632209A804C
:10B56000C7F8B03087F8B49032F068FA04234FF08F
:10B57000000C9F21D4F8D80E0DEB0302CDF804C0C7
:10B5800038F0AAFA9DF805809DF8043007F1900084
:10B590004FEA08289DF8061048EA034848EA0108DF
:10B5A000414645F0C3FA00287FF46EAF4046FDF7F0
:10B5B00039FB034600287FF467AF9DF806009DF82D
:10B5C000052000029DF8071040EA0240204A084387
:10B5D000904217D0A7F89430A7F8A030C7E92633D7
:10B5E000FDF720FB034600287FF44EAF94F8D40EFD
:10B5F0001D4634F0E7FF38F0ABF845E7062101FBC4
:10B6000002C268E7134B4FF400314FF0006287F835
:10B61000A290C7F894304023C7E92612A7F8A030BB
:10B62000FCF7F8FD07F1900087F8A99045F0CAF9FA
:10B63000094BC7F8903027E768190120583B0120D3
:10B64000602A0120F02A0120A0190120404B4C0063
:10B6500021AAEF000004000878D205082DE9F04F78
:10B660000423BE4C402141F21C1504F6746704F11A
:10B6700060064FF0A042636661670023022194F8E0
:10B680001D048BB0C4F8607466512266C4F8903013
:10B690002367C4F88C30C4F88430A167E166C4E93C
:10B6A0001F33002800F0628103211F46164684F8EC
:10B6B0001D14936823F001039360F368304643F050
:10B6C0004003F36007F010FBB36B012F054643F412
:10B6D0008033B36317D005B3022384F81D34A04B25
:10B6E00093F8C450012D00F0FD80236E80210120CD
:10B6F00059625A6A42F480029A62FCF7B3FD002054
:10B700000BB0BDE8F08FB36843F00603B360B368D5
:10B7100043F02003B360002DDED1236E3220DA68BF
:10B7200022F0C042DA60DA6842F08042DA6009F062
:10B73000D7FB606E50B32A4601272946C2EBC203ED
:10B74000561C04EB830383F89C20A3F8A220F2B2DA
:10B7500083F89D70824283F89F10C3F8B010C3E94C
:10B760002911EBD300221146C2EBC203561C04EB95
:10B77000830383F85C22F2B283F85D12824283F87D
:10B780005F12C3F87012C3E99911EDD30022236E42
:10B79000D4F86CC01646D4F87080D4F88CE0D4E9A4
:10B7A0001E71019102F14001013203EB81010F2A68
:10B7B0004E60F7D19A6BBEF1000F40F0438122F446
:10B7C00000129A631A6842F040021A601A6842F046
:10B7D00080021A600022012F03F50066C3F8002ED4
:10B7E000D3F80028C3F80028D3F8002800F02181FE
:10B7F000032F00F01E8142F00302C3F800284FF42B
:10B800008461584A196102E0013A00F032811969F5
:10B810008F06F9D41021534A196102E0013A00F071
:10B8200026811969C906F9D4002131617161F1617C
:10B83000E0B103F510624FF0904A4FF0006B0F46F5
:10B840004FF67F399C4607E0176001311761C2F857
:10B8500008902032814261D01368002BF4DA11B1D4
:10B86000C2F800A0F1E7C2F800B0EEE73269B8F123
:10B87000010F22F48072326100F0ED8000216FF040
:10B88000804299615A61B8F1000F03D19A6942F080
:10B8900010029A619969344A0A439A61019A1AB16D
:10B8A0009A6942F008029A61BEF1010F00F0CE8061
:10B8B000002D7FF411AF0121D4F8842084F8985032
:10B8C0008A4284F81D1400F0D6807368032043F088
:10B8D0000203736009F004FB214B93F8C450012D5F
:10B8E0007FF403AF44F03EFD00287FF4FEAE236EEC
:10B8F0008022284640215A625A6A42F400129A6213
:10B90000FCF7B0FC20210220FCF7ACFC4021032016
:10B91000FCF7A8FC00200BB0BDE8F08F00216346C7
:10B920000CF530624FF0904A4FF0006B0F464FF627
:10B930007F39844607E0176001311761C2F808902B
:10B940002032614592D010680028F4DA11B1C2F8B3
:10B9500000A0F1E7C2F800B0EEE700BF68190120CF
:10B96000602A0120400D030000383C8000F0FF05F4
:10B970004C4B03204FF4C05684F81C541A6B42F011
:10B9800001021A630A221B6B069105A903F0010349
:10B99000089045480493049B07950596099206F084
:10B9A000C7FED4F88C30012B72D03E4B06214320C9
:10B9B0005A6B42F080025A635A6B02F08002029284
:10B9C000029A5A6C42F480425A645B6C03F48043DE
:10B9D0000393039BFDF77EFF266E0323334A082162
:10B9E000916084F81D34A26FB368012A276F23F099
:10B9F0000103B3607FF461AEB26B2D4B22F4803251
:10BA0000D4F89410B2630129F26803EA0203F360E8
:10BA1000F36823F44013F36003D1F36843F4801315
:10BA2000F360304607F060F9012F05467FF453AE0E
:10BA300069E6BCF1000F3FF4E0AE42F00102C3F84A
:10BA40000028DCE642F400129A63C3E69969194AB9
:10BA50000A439A612CE718490020184A31636FF0B5
:10BA60008041376B3A4332639861596112E701258F
:10BA7000DAE60125CEE684F854549969C4F85C24CA
:10BA800041F000610E4A9961596D0A435A651CE7FD
:10BA90004FF4007305A904480593CDE9065506F057
:10BAA00047FE82E7003802400000024000E100E06B
:10BAB000BFFFBDFF04000040000180000300010043
:10BAC0000300001010B51A4C94F8750FC0B9194B4B
:10BAD00083F8B505C3F8B80594F8783F012B05D075
:10BAE000022B21D0D4F87C3F1BB910BD124BC4F8F7
:10BAF0007C3F12495B68A1F10C00BDE8104018477B
:10BB000034F060FD94F8772F0A49003AC1F8B8057F
:10BB100018BF012281F8B5250028DDD01F22202181
:10BB2000C28034F0D9FDD7E7054BC4F87C3FE0E78D
:10BB3000583B01206819012084010120D84A0120C6
:10BB40006001012099B10A6B824216D9154BD3F8D6
:10BB5000C42F914221D34C3991421ED30B6B984292
:10BB6000F9D38B6B9842F6D80B46184670470D4BAD
:10BB7000D3F8C41F0A6B904212D30B680BB9F4E7D9
:10BB80000A6B90420B4602D38A6B9042EDD951F872
:10BB90004C3F002BF4D118467047002318467047DD
:10BBA0000A46D8E7583B01202DE9F047CC0143D1A4
:10BBB000034622494FF0FF32022443F8081B7E2639
:10BBC00042601846DFF878802644051D6FF0704704
:10BBD000D8F8C89F4FF0010A013E494608E0A34249
:10BBE0001CD0631C45F8043C321B1C460435CAB10A
:10BBF0000B6BA34202D88B6BA34204D22046FFF703
:10BC0000A1FF014690B10A794B6B002AE7D1A3420C
:10BC100004D0E6D2631C45F8042CE5E7631C45F824
:10BC2000047CE1E7C8F8C81FBDE8F087321B631C3D
:10BC3000494645F804ACD8E78026C3E7F8FFFF0F74
:10BC4000583B01200A44914219D0013910B4541EC6
:10BC500011F8012F0823504002E0013BD0B209D077
:10BC600010F0800F4FEA4002F7D082F0D500013B80
:10BC7000C0B2F5D1A142EBD15DF8044B70477047DB
:10BC8000194A00232DE9F04702F6DC7484B005461A
:10BC900092F9D58F1F46461804F5287A4FF0B60959
:10BCA000D4F800C0204600226946E034BCF1000F01
:10BCB00014D09CF838C0BCF1140F0FD018F1020F4B
:10BCC00001D0C4450AD1CDE90277CDE90056ADF8DF
:10BCD00008908DF80D702AF06FFA0346A245DFD167
:10BCE000184604B0BDE8F087583B01202DE9F04725
:10BCF0009AB004460D4617469846DDF89090DDE967
:10BD0000226A02E0206831F00BFF206831F010FF5A
:10BD10000028F7D10146642201A851F035F9264BDD
:10BD20008DF80450CDF85CA00293002D3FD0AB1EDF
:10BD3000012B3ED9042D14BF002303231F4A8DF885
:10BD400005300123926A039616448DF85B30CDE9E5
:10BD50000594049637B14246394607A851F0A2F837
:10BD60008DF85A80164E002396F8C6911893B9F1B3
:10BD7000000F19D196F8C501642201A902FB0060E9
:10BD800000F5E47051F08EF8012386F8C59186F82D
:10BD9000C631236843B143463A46294620461AB085
:10BDA000BDE8F04717F042B81AB0BDE8F0870523A8
:10BDB000C4E70223C2E700BFD44D0120602A01205E
:10BDC000504C01200C480D4BD0F8481210B48A1E7C
:10BDD0000B4C2231C0F83832B0F866321B01A4FB9C
:10BDE00003C3DB08A3F5B06322F8023F9142F3D10D
:10BDF0005DF8044B704700BF504C0120716F020882
:10BE0000CDCCCCCC70B5084C251D2E4614F8010BBA
:10BE10002AF0A6FB28B10378B44205F8013BF5D11E
:10BE200070BDFF23F8E700BFDC4E01202DE9F0478D
:10BE30001C4F01264FF03C094FF0000807F10805A0
:10BE4000B24617F8010B34F0BDFB044690B180F800
:10BE50000690C671FB7803F07F02012A17D013F019
:10BE6000800F20460CD185F8048034F06FFD85F8F2
:10BE700005802C6001360835052EE2D1BDE8F0873B
:10BE800085F804A034F068FD85F805A0F1E71B06ED
:10BE900005D40121204634F01FFCFB78DFE734F0A5
:10BEA0005BFDF6E7E44E01202DE9F047204E82B01D
:10BEB00000244FF00409DFF87C8006F10C05A6F59C
:10BEC000307716F801AB5046BAF1000F2CD034F0A1
:10BED00079FB0134034604215046E4B26B6113B18F
:10BEE00083F80690DC71224631F05AFB022182462B
:10BEF000D0B168699AF8082034F0B6FBB7F8BE32C2
:10BF0000B7F8BCC2002051460A4A01902846CDF835
:10BF100000C01835B8FBF3F39BB229F005F90123F3
:10BF2000082C05F8073CCCD102B0BDE8F08700BF73
:10BF3000104F012040420F002DE9F041204C00231A
:10BF40004FF0050894F8932304F5647704F56575BC
:10BF500084F88C2317F8010B5E1C20BB2860032E8D
:10BF600005F104053346F5D194F88C13D4F8940305
:10BF7000C94301F0010134F0A3FD94F88C13D4F807
:10BF8000980381F00201C1F3400134F099FD94F867
:10BF90008C13D4F89C0381F00401BDE8F041C1F397
:10BFA000800134F08DBD34F00DFB0121F3B2286027
:10BFB00010B180F80680C371286834F08DFBCEE79D
:10BFC000504C0120F0B5294C83B0B4F8A453A4F828
:10BFD000A653EDB994F8A00334F0F4FA94F8A12331
:10BFE000C4F8A803003A18BF012284F8AC2348B172
:10BFF00094F8A2132B220029C28014BF1121012121
:10C0000034F06AFB002003B0BDE8F04034F060BDBE
:10C0100094F8A07300222B21384631F0C1FA06466D
:10C02000384634F0CFFA00B10EB903B0F0BD2B2280
:10C03000C4F8C40302210027C280327A34F014FB12
:10C040000B4AA4F8C853314604F56C700197B2FB53
:10C05000F5F3C3F34F059BB2009529F065F8D4F8CA
:10C06000B0331F6084F8C173DFE700BF504C01207C
:10C0700040420F002DE9F84F264B002693F8D423B9
:10C0800003F2CB3703F57A7483F8CA235FFA86FB91
:10C090004FF0010917F8010F01360BEB090A494669
:10C0A0004FF000085FFA8AFA524631F079FA0546F5
:10C0B00048B3387804F80E8C04F80D8C04F80FBCE3
:10C0C00004F8109C44F8045C34F07CFA022118B1A6
:10C0D00080F8069080F807A02A7A34F0C5FA0E4A54
:10C0E000002128464CF036F90C4B221D21462360D6
:10C0F00028460B4BC4E901384BF0F8FF42466979FA
:10C10000286828F05FFF082E04F11C04BED1BDE8AA
:10C11000F88F00BF504C012040420F0079500308B7
:10C1200011FB020870B52C4C00222C4B022194F814
:10C130000005C4F8F834C4F8B824C4F8BC24C4F822
:10C14000C024C4F8F424A4F8FC2431F029FA00280F
:10C1500041D0234B0546026803F1C000597C11B160
:10C1600059688A422CD018338342F7D1002394F8BF
:10C170000005C4F8E45384F8D83334F023FA08B146
:10C180000223C38000262A7A022134F06DFA314658
:10C190002846144A4CF0DEF8134B144A2846C4F8DB
:10C1A000E833134B111FC4F8F063C4F8EC334BF0C1
:10C1B0009DFF324669792868BDE8704028F002BFCB
:10C1C000926A0C4801320C49D0F87431B3FBF2F397
:10C1D00081F8A831CAE770BD504C012000FFFF0074
:10C1E000AC13002040420F0039FB02083C500120F4
:10C1F000D5FC0208602A0120000001202DE9F04F43
:10C20000DFF878B180460B46DFF874A10BF1D0005F
:10C21000C02200212DED068B97B0CDE9023850F0F9
:10C22000B3FE9AF80185B8F1000F00F095829AF8F4
:10C2300002350893002B00F0CE82DFF8489199F880
:10C240006C3E012B00F0ED82022B00F0E5820BF535
:10C25000FC73444D99F8626E1C460F930FCD0FC4CA
:10C260000FCD0FC4311E404A99F85E3E18BF012120
:10C27000CBF81022072B8BF8301295E8070084E8E2
:10C28000070000F25D83042B0ED999F8613E374A0E
:10C29000012BCBF8382205D09A1E53425341002E71
:10C2A00018BF00238BF83C320023DFF8DCA0039397
:10C2B0002F4B04932F4B0593DDE90232934240F359
:10C2C000B081059B032113F8015B059309EB05037E
:10C2D000013593F8636EEDB230462A4631F060F9CD
:10C2E0000446002800F02283304634F06BF9049BAA
:10C2F000586110B10323C571837199F85E2E99F8C6
:10C300005F3EE77906920BB187F00107204637F0D0
:10C3100015F90346002800F006839BF83C2207929B
:10C32000002A40F01883D0F80480B8F1000F00F024
:10C33000FD829B6840460B9337F068F92A4603213B
:10C340000A9037F073F9002800F0F0829BF8406201
:10C3500025680948CAF89480002E00F0278300233E
:10C36000024617E028D70508558D0508194004082E
:10C37000AC130020C649012020150020DC1200204B
:10C38000504C0120583B0120A02600200133B3422D
:10C3900000F00C831168B8328D42F7D1DEB2B823B9
:10C3A0009BF84022039906FB0303013A8AF8111017
:10C3B000CAF898302079099234F004F907F00101A5
:10C3C0009BF8303201310BB187F001074901CAF8FF
:10C3D000084041F00E01CAF81410227A34F044F9F2
:10C3E000099B9E4200F01E84069B063B0C93002393
:10C3F00060220AF16401CAF8803008EE101ACAF807
:10C400006420CAE91A33CAE91C33CAE91E3317F09B
:10C4100002034FEA47070D9300F0E082012307F083
:10C420000207CAF86C30CAF87870002702234FF46C
:10C4300080310A22CAF87070CAF88420CAF8903095
:10C44000CAE9221763790C2B00F2BE82CB4A9BF813
:10C450003C1202EB8302D2F80874CAF85470002927
:10C4600000F0F982DAF89830C3F8A880CAF894800E
:10C47000079B002B00F073830AF118000E9006F062
:10C48000F1FA9BF83C320E98002B00F08E83BC49E9
:10C490004FF4907322684FF0030C03FB0613DAF895
:10C4A00098104C32C1F8B030CAF81C300B9BCAF857
:10C4B0001820CAF83C30CAF848C0069B40214FF407
:10C4C000806C082B4FF00403CAF820104FF4805101
:10C4D000CAF844304FF000030CBF06221222CAE90A
:10C4E0001333CAE909334FF40033CAF838204FF444
:10C4F0008042CAF84030079BCAF83420CAE90BC111
:10C50000002B00F040839DF83030CAF89480022B55
:10C5100000F25582994A9B4902EB8303069AD3F8AD
:10C52000FC33082AB1FBF3F308BF5F2203F12303B6
:10C5300018BF1322CAF85C30DAF8983050469A8057
:10C540004CF078FB9BF83C32002B00F02782079BD5
:10C55000002B00F0238218EE102A3946284605F0F9
:10C5600019FF012F00F0EC82042F00F05383102FED
:10C5700000F08682402F00F0AB83B7F5807F00F09B
:10C58000B583B7F5806F00F0B983B7F5805F00F031
:10C59000BD83B7F5803F00F0C1836A6D05F11800D7
:10C5A000082342F400626A6577490422DFF800C27A
:10C5B000C95C1CF803C00B5802FA0CF223EA020310
:10C5C0000B502B6843F001032B600D9B002B00F0F8
:10C5D000B3822B6A43EA87072F62099B9E420BD1E5
:10C5E0006B6C43F400436B642B6843F080032B6057
:10C5F0002B6843F001032B609BF83032002B40F096
:10C60000A782039A012304990AF1A00A01320AF8C9
:10C61000913C4B7401F11803082A039204937FF4B0
:10C620004BAE0F9B89E1DFED598A594AB0EE688A1B
:10C63000584BCBF8AC210022CBF8A831564BCDF8A3
:10C640001080039238EE887ADFED547AF5EE006AB6
:10C65000534C28EE278ADFF85CA1B0EE67AA0027CA
:10C66000C6EE879A9FED4F9ACBF8B431CDF814807F
:10C67000029BBB426DD01AF8015B032109EB050355
:10C68000013593F8638EEDB240462A4630F088FFBC
:10C690000646002800F0B782404633F093FF606101
:10C6A00010B10323C5718371327A022133F0DCFFAC
:10C6B000049B002B00F0EE81B9F85C3E4FF6FF7151
:10C6C00007EE903A384BF8EEE77AD3F87421FCEE97
:10C6D000E77A17EE903AB2FBF3F00144090CB2FB93
:10C6E000F1F2B2FBF3F399F85E1E042900F0E48145
:10C6F00007EE902AF8EE676A26EE887A69EE477AA6
:10C7000099F85F0E03999BB201902046E6EEA87A55
:10C710000091314684ED027AC4ED037A28F004FDDD
:10C72000002F40F3B58161681D4B02E09C4200F090
:10C73000AF815A6818338A42F8D1059B013783F0DC
:10C74000010301221834082F04F8083C04F8072CD0
:10C750008ED1164ECBF82C62DBF82C3263B300225C
:10C760000121029883F82D1083F82C001A6383F8B6
:10C770002E2017B0BDEC068BBDE8F08F78D20508EF
:10C78000E01A002000D0121370D705080000000046
:10C7900085010308B5C20308A9C203086F12833AD2
:10C7A000AC13002000007A44602A01206C140020A1
:10C7B00064D70508C6490120C54DC64C0FCD0FC42E
:10C7C0000FCD0FC495E80700A4F1200384E807000B
:10C7D000CBF82C32CDE7C04D0BF5C874DFF854937D
:10C7E0000FCD0FC40FCD0FC495E8070099F85E3E3A
:10C7F00099F8606E84E80700042B00F23C8101A2E6
:10C8000052F823F021CA000877CA000817CA0008A6
:10C81000F5C9000827C6000899F85E3E082B00F00D
:10C820000281029B0026AD4DCBF83432AC4C99F816
:10C830005E7E8AF804658AF83C750FCD0FC40FCD73
:10C840000FC499F8623EA4F58A729B1B049295E886
:10C85000070018BF0123354684E8070031464FF42E
:10C860004C72A0488BF8303250F08EFB9E4BDDF8B6
:10C8700010809E4E0393CDF810900AE034F066F8D5
:10C88000F368082D06F1200608F1180848F8043C62
:10C890005DD0DBF83432AB4259DD039A12F8013B2C
:10C8A0000392049A134493F8637E384630F000FFF5
:10C8B0000446384633F086FE049A8146E77992F8BA
:10C8C0005F2E0AB187F0010707F001049BF83022C0
:10C8D00001348AF803450AB187F00107484633F06E
:10C8E0003DFF002800F084814846013536F09AFD6E
:10C8F000C6F80C9061017060EAB2377441F0010132
:10C900007161B9F1000F05D04FF0030389F80720DA
:10C9100089F80630484633F0DFFEF9074846ADD4C3
:10C9200034F01AF8ACE79BF83C32A3B97049002305
:10C93000704ACBF81412CBF81C22CBF82C320BE740
:10C94000082B7FF4B1AC6C4BCBF83832ACE46448C4
:10C95000CBF82C0200E7D4F81480B8F1000FE5D032
:10C96000A36940460B9336F051FE644B2422451ECA
:10C970000A9002FB053595F8C831392B00F02C815F
:10C9800020684BF055FD024639210A98D2B236F0A4
:10C990004DFE0028CAD000230793D7E40A989022BE
:10C9A0009AF8113056494DF021F9D4E5B823721C9C
:10C9B00003FB06B38BF84022C3F84452EFE48D2307
:10C9C0001322CAF85C30B7E59BF83C32CAF85470C1
:10C9D000002B7FF447AD1F461A4641E001224FF479
:10C9E000807307F00207CAF86820CAF87C30CAF8DA
:10C9F00074701AE59FED438ADFED438A002E3D4AAD
:10CA0000424B16BF414600211346414A0491414919
:10CA1000CBE96A2116E69FED408AF0EE488AEDE701
:10CA2000DFED3E8A01E60BF5FC733D4D99F8626E31
:10CA30001C460F93003E0FCD0FC40FCD18BF01262B
:10CA40000FC4384B8BF83062CBF8103295E80700F2
:10CA500084E8070077E7344A02EB4303B3F83C2449
:10CA6000DAF89810AAF80C20B1F8B43023EA0203DF
:10CA7000A1F8B430FCE49FED2D8AF0EE488ABDE7C2
:10CA8000AA6905F11800022342F40062AA618BE54D
:10CA9000002353E6FAFE697AFCEEE77A244B17EEA0
:10CAA000901AD3F874214FF6FF73B2FBF1F11944D9
:10CAB000090CB2FBF1F216E607EE903AB8EE677A8F
:10CAC00007EE902AF8EE676A27EE0A7A16E600BFAC
:10CAD000D0D6050858510120D8D50508FCD6050840
:10CAE000A0140020A02B0020C6490120D02E002039
:10CAF000B1C20308A9C20308E53F040800000120F1
:10CB00009D370000ACC5A737ACC5A73641FD02086C
:10CB1000B5C2030885010308282930386F12833A0B
:10CB200028D70508558D050878D205086F120339F6
:10CB3000602A0120583B01202B6A1F432F624CE5DD
:10CB4000AA6905F11800002342F00802AA612BE54A
:10CB500023684FF6FF7162793433995051E5D8F864
:10CB600000205FFA88F3182128F0FF0022F001026C
:10CB7000103BC8F80020B3FBF1F105F0CBFF0A9899
:10CB80004DF05AF878E45FFA88F31821024628F04D
:10CB9000FF00103BB3FBF1F105F076FFD8F8003051
:10CBA00043F01003C8F80030ADE40B9A5821DFF8C9
:10CBB000A0C1CAF83C20039A01FB02C12268CAF84E
:10CBC0004830CAF89C1002F13403CAF81C1062798C
:10CBD0001344CAF8183070E420684BF029FC95F82B
:10CBE000C93183427FF4CCAE089B0793FFF7AEBBFD
:10CBF0004E4B01224E498AF80425CBE977314D4B43
:10CC0000CBF8E831A4E64C4A4A4BCBF8AC21CBF840
:10CC1000B4319FE5AA6905F11800012342F008022A
:10CC2000AA61C1E400224FF0FF311346ADF8442061
:10CC3000129214928DF854201391404A52F83320E6
:10CC400095424DD001330E2BF7D10020069B9A1F41
:10CC50000C92FCF7F7FE2B6839499DF8302023F041
:10CC60000103D1ED5D7A022A2B60F8EE677A22D8B3
:10CC70003449DFED356A01EB820292EDFF7AB8EEBE
:10CC8000477A87EE870A30EE260A4EF099FE069B19
:10CC90000138082BADF8440014BF13225F22002393
:10CCA00011A92846139214938DF85430129305F06D
:10CCB000C3FCFFF79CBB9FED257A9FED230AA7EEEF
:10CCC000870A4EF07DFE01381322ADF84400E6E7F6
:10CCD000AA6905F11800032342F00802AA6163E47F
:10CCE000184A02EBC30393F89003AFE7EA6905F132
:10CCF0001800042342F00802EA6155E4EA6905F1EC
:10CD00001800052342F00802EA614DE4EA6905F1E2
:10CD10001800062342F40062EA6145E46A6D05F1F9
:10CD20001800072342F008026A653DE4B5C2030813
:10CD3000B1C20308A9C203084DFE020804D60508C3
:10CD4000602A012078D205080AD7233CFCF4B234CB
:10CD5000E023002070B5524E96F8600233F032FCAA
:10CD600096F8615260B12D2304462021C38033F030
:10CD7000B3FC0A2030F056FE204636F049FB18B9C5
:10CD8000D6F84035DA0000D570BD013D092DFBD83D
:10CD900096F85F42CCB940202BF0F4F90028F3D08C
:10CDA00090F9043096F83112092BC8BF143B0A29B8
:10CDB000334493F8444566D093F8503596F85E2294
:10CDC000002A08BF1C46002CDED0204633F0FAFBB8
:10CDD000054608B12D23C3800121284633F07CFC91
:10CDE0000121084633F0B6FE0121284633F068FEE3
:10CDF0003C2030F023FE0021012033F0ABFE96F8FA
:10CE000061321BB3002400210134084633F0A2FE36
:10CE10000021022033F09EFE0021284633F050FE10
:10CE2000782030F0FFFD0121002033F093FE012136
:10CE3000022033F08FFE0121284633F041FE782096
:10CE400030F0F0FD96F861329C42DCDB96F85F3200
:10CE50008BB9D6F8603203F0FF13B3F5803F93D15E
:10CE6000D6F8403513F080538ED186F86132BDE894
:10CE7000704043F05BB9322030F0E0FD28460021DD
:10CE800033F02AFCE5E7D6F868355B057FF57CAF23
:10CE90000EF060FC00287FF477AF002C95D173E78B
:10CEA000504C012030B40438043A0C1F01F108053D
:10CEB00054F8043F52F8041FAC42A3EB010340F8BE
:10CEC000043FF5D130BC704738B5041E0D4611DB68
:10CED000092C1FDC0846134B0021134AA3FB04C393
:10CEE0004170DB0803EB8303A4EB4303D35C0370C3
:10CEF000284638BD64422D230846092C00F8013B22
:10CF0000E9D9084B01460A22A3FB0430C00842F0CD
:10CF100047F9E0E703480A22A0FB0430C00842F0CA
:10CF20003FF9D8E7CDCCCCCCE45B0608344870B4EC
:10CF300090F86C35A3F13001092958D800F26C54EF
:10CF400000F27B50224612F8015FA5F13001092959
:10CF500004D88242F7D1002070BC7047141B022C09
:10CF60004BDD2848002101E010F8013B01EB810175
:10CF7000161A044603EB4103022EA3F1300303F01B
:10CF8000FF01F1DC204B03FB01F1A2424FF0000353
:10CF90000ED903EB830314F8016B5B00A242A3F1EB
:10CFA0003003334403F0FF03F3D1184800FB03F3CD
:10CFB0002E2D06D01648A0FB032370BC01EB930076
:10CFC000704701320425002404EB84041078013DED
:10CFD000303864000928A4B2204401D8013284B258
:10CFE00015F0FF05F0D1642202FB0433E2E70021D3
:10CFF0001D4600F26C520B46DAE70021054CC4E7EF
:10D00000504C0120BD5101208096980040420F00F5
:10D01000ABAAAAAABC51012038B50D460446FF218F
:10D0200000682A464FF0B0FF22682A44226038BDCB
:10D030000C461646054683B529F01EFB204629F00E
:10D040001BFB0021204B0846002E08BF1E4633F074
:10D0500081FD0021012033F07DFD284630F068FD80
:10D06000B0B10121002033F075FD284630F058FDA5
:10D070000746204630F058FD0028FAD039462046B1
:10D0800030F07CFD3846B0470021084633F062FDA1
:10D09000204630F04DFD0028DFD00121002033F084
:10D0A00059FD204630F03CFD01462846019130F004
:10D0B0003BFD01990028F8D0284630F05FFD0021A3
:10D0C000084633F047FDC8E74D540308F0B5002289
:10D0D00089B0234E04AF13460A61BC46C1E9002261
:10D0E000C1E902220268C2F3855040FA03F46546A2
:10D0F000E40703D59C5D05F8014BAC460133062BD4
:10D10000F3D1184DC2F303240023C2F305302C5D84
:10D110000DF119068CF80030DFF850C08DF818407A
:10D1200040FA03F43546E40704D513F80C4005F83B
:10D13000014B2E460133062BF2D10023C2F3834567
:10D1400006AC0846337002F00F030749C2F303121E
:10D150000097CDE9014541F0A9FD09B0F0BD00BF40
:10D160002C5C0608245C06080C5C06081C5C06089F
:10D1700070B5094C0546D4F87C2562B1002601360D
:10D180002D21D4F87C0537F09DFFAE42F7DBBDE8DA
:10D19000704038F041BA70BD504C012038B505469A
:10D1A000084642F0A3FD041E0D4B0FDB93F88C25BF
:10D1B000944205DA21460B4839F05EFD204638BD21
:10D1C000FF2C03D1084839F057FDF7E793F88C2579
:10D1D000284606494FF0FF34013A38F0E3F9EDE70D
:10D1E000E40100203C5C06084D5C0608605C060813
:10D1F00030B583B04D1C0093002304688572C27261
:10D20000A469A04703B030BD03685B6C0BB1022179
:10D210001847704770B5104ED6F82C3293F82E2070
:10D22000CAB19B699847B0B1D6F82C3293F82C203C
:10D230006AB10A4D0024DB69E0B2B5EC010A0134A1
:10D240009847D6F82C3293F82C209442F3DB5B6A93
:10D25000BDE87040184770BDDC120020603000202F
:10D2600038B51E4C0968D4F884550068491B1C4D1C
:10D27000DFED1C6A00EE901AD4F88015D5EDFB7A2C
:10D280001C46F8EEE00A401A60EEA70A07EE900A84
:10D29000F8EEE77A20EEA07AB1EE670AA7EEA77A59
:10D2A000F1EEC77A67EEA67AFCEEE77AC2ED007A75
:10D2B00042F0B0FD9FED0C7ADFED0C7AE0EE077ADC
:10D2C000FDEEE77A17EE902A002A02DBC4ED007A21
:10D2D00038BD48F6A0431344236038BD504C0120AC
:10D2E000000001202C7D8E3FA00CB34500A00C4611
:10D2F00038B50F4C034694F89F1504F5B36084F8D5
:10D300009B3501F03F0101F10A058B1C083184F8BF
:10D310009A55254484F89D351FF07CFC85F89605C8
:10D3200094F89A35000A1C4484F8970538BD00BF6C
:10D33000504C012038B50A4C00250122802120469E
:10D340002AF00CFF30B194F904002AF03BFF08B139
:10D35000006838BD01350C34092DEED10020F8E706
:10D360001052012038B5041F00F1080554F8043F9D
:10D37000D81780EA430018F027FCA542F6D138BD43
:10D38000074B4FF6FF70002103F6AC4210B40024A7
:10D39000C3F8280D5167C3F8244D5DF8044B70475E
:10D3A000D4230020F8B5794CDFED797AD4F8302D0C
:10D3B00094F8103D07EE102AB4F8127D2DED028B83
:10D3C000B8EE478A28EE278A002B68D1D4F81C6D66
:10D3D00094F82D1D304626F007FB0F2894F8113DD8
:10D3E000B8BF0F2085B2A4F8125D002B00F0BB80FF
:10D3F000AF4258D094F8AC6CB4F8143D07EE905A94
:10D40000DFED645A002206EE103AF8EE677A6249C0
:10D410000020B8EE466AC5EEA76A0B4685EE867A0E
:10D4200076EE886AC8EE267A37EE087AC8EE076A82
:10D4300096BB58609860D860C3ED047A013210330F
:10D44000032AF5D1002E34D094F8163DB4F8185DB7
:10D45000C1ED106AC1ED147AC1ED187A002B7CD1B0
:10D4600094F82D1DD4F81C0D26F0BEFA0F28B8BF75
:10D470000F2080B28542A4F8180D6ED000286CD021
:10D4800007EE900ADFED436A444BF8EE677A86EECA
:10D49000A77AD3ED006A56E0C3ED047ACEE794F89C
:10D4A000113D002B5CD094F8AC6C002E66D13D464B
:10D4B000A2E7002394F8162DB4F8185DC1ED106AA8
:10D4C000C1ED147AC1ED187A4B638B63CB634B6467
:10D4D0008B64CB644B658B65CB6562B994F82D1D6D
:10D4E000D4F81C0D26F080FA0F28B8BF0F2080B2A8
:10D4F0000546A4F8180D41F26D0394F82C2DE25462
:10D500005DB307EE905A254BDFED226A0022F8EE5C
:10D51000677A41F26C010120C3F80823C3F80C2399
:10D5200086EEA77AD3ED006AC3F81023C3F8182358
:10D53000C3F81C23C3F82023C3F82823C3F82C23E3
:10D54000C3F83023605437EE267AC6EE877AC3EDEF
:10D55000C57AC3EDC97AC3EDCD7ABDEC028BF8BDB7
:10D56000D4F81C6D3D46304694F82E1D26F03CFA4A
:10D570000F28B8BF0F20A4F8140D39E794F8163D12
:10D58000B4F8185D002B3FF46BAFE6E7D42300201E
:10D59000BD3786354E2DA63D803000200831002055
:10D5A000012817D0304A41F29303D35C012B2DD0D0
:10D5B0002E4BF6EE006ABEEE007ADFED2D7A03EB1D
:10D5C000800090ED000A80FE660A80FE070A20EEC9
:10D5D000270A7047274A41F294032349F6EE006A6E
:10D5E00002F5C960BEEE007ADFED217A90ED010A06
:10D5F000CB5C80FE660A80FE070A20EE270A23B174
:10D60000B5EEC00AF1EE10FA03DC70479FED1A0A7E
:10D61000704707EE903AB2F93216B2F94636DFEDAE
:10D62000176AF8EEE77ACB1A07EE103AB8EEC77A27
:10D6300027EE267AB4EEE77AF1EE10FAE6DA77EE24
:10D64000C77AB2EE047AF4EEC77AF1EE10FADCD8BB
:10D65000B1EE047A67EEA67A30EE470AA7EE807A3A
:10D66000B0EE470A704700BFD42300209852012033
:10D6700000004843504C012000000000CDCCCC3DC0
:10D68000F8B5744B40F60301B3F854260A402DED6B
:10D69000048BB0EE408A04D0B0EE480ABDEC048B97
:10D6A000F8BD03EB4003B5EEC00ADFED6B7A00F185
:10D6B000D40EB3F93016B3F94436F1EE10FA674DD3
:10D6C000A1EB030305EB8E0CC8BF012600EE103A58
:10D6D000D8BF4FF0FF36DCF8344D05F63457B8EEBE
:10D6E000C00A20EE270AB5EEC00AF0EEC07AF1EECD
:10D6F00010FACCBF01214FF0FF31A31B18BF01234B
:10D70000002C08BF0023002B49D197EDCF7AF4EE0F
:10D71000C77AF1EE10FA07DD8E4208BF002C0CBF6D
:10D720000123002300F08180002C42D007EE901AE4
:10D73000B0EE408AD7EDD25AF8EEE77A9FED486A0C
:10D74000DFED486ADFED488A97EE878A28EE258A62
:10D7500088FE468A88FE268A002B58D141F278033B
:10D76000EB5C984298D1414D95F8983D262B93D18A
:10D77000B2EE049A20EE090A4EF022F9B0EE480A01
:10D78000A5F89E4DA5F89C0D4EF01AF928EE890AD1
:10D79000A5F8A00D4EF014F9A5F8A20D7CE797EDC1
:10D7A000CF7ACCF8342DF4EEC77AF1EE10FA3ADCE9
:10D7B00013462F4A9FED2F6A02EB8002D2ED097AC1
:10D7C000F0EEE76AF4EEC66AF1EE10FA28DC9FED9F
:10D7D0002A6A66EE866A97EDD06AF0EE408A67EEB6
:10D7E000867AE6EEA78AF5EEC08AF0EEE87AF1EEE8
:10D7F00010FAF4EE477ACCBF01224FF0FF32F1EE7F
:10D8000010FA01DD964217D00024002BA6D01B4A47
:10D8100000EB8003002102EB830343F8341C9DE7F7
:10D82000F7EE006AD7E78E42C2D105EB8E0E0C46AA
:10D830000123CEF8341D77E707EE902AB0EE688A10
:10D84000D7EDD26A0024F8EEE77A97EE878A28EEC1
:10D85000268ADCE7504C0120CDCCCC3DD4230020DF
:10D8600000007A4400007AC400000000583B012008
:10D87000E4010020FFFFF9436F12033BCC3400208A
:10D8800070B504466F4EC0B22DED048BF0EE408AA9
:10D890000D7820F037FB6C4A06EB8403694207EEF3
:10D8A000905AD3F8583607EE101AF8EEE76A82FB62
:10D8B0000312DB17B8EEC77AC3EB621307EE903A98
:10D8C000F8EEE77AE6EE807AF4EEC77AF1EE10FA37
:10D8D00005D407EE105AB8EE477A87FE677A06EB52
:10D8E0004404DFED5A9A40F60100B6F85426B4F924
:10D8F0003036B4F944161040A3EB010307EE903A1A
:10D90000F8EEE77AA7EEE97AB0EE478A07D0504BF7
:10D91000BDEC048B93ED7C0A27EE000A70BD20F06D
:10D92000F1FA0120B0EE409A20F0ECFAB6F9303668
:10D93000B0EEC00AB6F93216002B464AB0EEC99ACC
:10D94000B8BF5B42002992F8380FB8BF49429BB27A
:10D9500089FE009A89B28B42B8BF0B4607EE903A17
:10D9600002F63453F8EEE77A67EEA97A50BBF7EE89
:10D97000006A93ED807AB4EEE67AF1EE10FA50D4B4
:10D9800093ED7E7ADFED347AB4EEE77AF1EE10FAB9
:10D9900044D9DFED325AB7EE006AC5EE876AB0EEC1
:10D9A000467AA9EE667AC7FE466AC6FEA76AD3ED36
:10D9B0007D7AB0EE680A68EE277ABDEC048BA7EE9C
:10D9C000A60A70BD9FED246A93ED7E7AB4EEC67A06
:10D9D000F1EE10FA1FDDD3ED7F5AF4EEC65AF1EEE8
:10D9E00010FA18DDDFED1E6A75EEE77AB7EE005A21
:10D9F00029EE269AC7EEA56AC9EE077AC6FEC56A61
:10DA0000C6FE866A77EE857A66EEA76AC6FEC56AA6
:10DA1000C6FE866ACBE7F0EE466AC8E7F0EE676AB4
:10DA2000C5E776EEC76A9FED0F5A9FED0F6AD3EDFB
:10DA30007E5A66EE856A76EE677AA6EEA77A27EEBC
:10DA4000257A9FE7504C01201F85EB51CDCCCC3D72
:10DA500008310020D4230020000000000000C8424C
:10DA60000000C8C2610BB63B000034431C4991F86A
:10DA70006C259AB3F0B40026054633463046374647
:10DA80001BB991F86C452D2C22D02E2A18D0CA181B
:10DA900000EB800092F86C454000A4F13002092AA6
:10DAA00002D8A0F13002A0180E2B14D80133CA18E6
:10DAB00092F86C25002AE3D106B14042F0BC7047D1
:10DAC0000133002DF8D0CA182A4482F86C75DEE7BD
:10DAD00001231E46EBE70020F0BC70470020704792
:10DAE000504C01202DE9F041A02301240B4F1825B3
:10DAF000E6B2FF2B0BDCC5F11B0103F10108324636
:10DB0000DBB2C9B2D7F86006FFF772FB4346013DAE
:10DB1000EFD10134052CEAD1BDE8F081504C012051
:10DB20001FB503AC8DF80C30002300948DF80D3038
:10DB30000EF0CAFC04B010BDF8B50546262023F04F
:10DB40007BFF144C014608BBD4F8640690F83830CB
:10DB50001E3B012B02D894F871360BB130F00EF851
:10DB60000D4F0026AE4209DBB4F892360133A4F81B
:10DB700092360A4B9B6AC4F8A436F8BD17F8011B0D
:10DB80000136D4F864062FF0F9FFEBE7002384F8A0
:10DB9000A036EEE7504C0120C2520120602A01203D
:10DBA00010B51C2032F00EFD0446112132F094FD18
:10DBB000204632F0CBFEC8202FF040FF2046BDE8C3
:10DBC000104032F0C9BE00BF08B5002032F0FAFCA8
:10DBD000054BC3F8A80608B12A23C3804021BDE83D
:10DBE000084032F079BD00BF504C0120F8B56A4CB6
:10DBF000D4F834110B699E0702D5CB689D074BD42E
:10DC00000B69580702D5CB685A073DD40B691B072F
:10DC100002D5CB681F072FD40B69DE0602D5CB686F
:10DC2000DD0621D40B69D80702D5CB68DA073FD4CB
:10DC30000B691B0603D5CB681F0600F191800B69A9
:10DC4000DE0503D5CB681D0600F18E800B695C06EE
:10DC500003D5CB68580600F18B800B699A0602D574
:10DC6000CB689B0620D4F8BD6FF0100200230A6138
:10DC7000CA6984F85031D5E76FF0080200230A61C1
:10DC8000CA6984F85031C7E76FF0040200230A61C3
:10DC90008A6984F85031B9E76FF0020200230A6103
:10DCA0008A6984F85031ABE76FF020030B61F8BD4F
:10DCB0003A4B6FF0010299420A61B9D141F2041363
:10DCC0003748C558D5F81432002BB1D1354FD7F8A5
:10DCD000AC2692B1D0F858C602F03F066244C0F8B4
:10DCE0005826D0F85826B2F5006F01D1C0F8583642
:10DCF0000023C7F8AC36002E44D0D0F85826D0F810
:10DD00005C369A4294D0D0F85826D0F85C369A42C5
:10DD100032D9D0F85866C6F50066D0F858C6B6F5C0
:10DD2000007F214A28BF4FF40076D5F814326244B0
:10DD3000C5F81062C5F80822002B7FF479AF0123E3
:10DD400041F21C11C0F8A46EC5F814323346405895
:10DD5000812105F077FAD4F83411C7F8AC6667E78B
:10DD60006FF080030B616AE76FF480730B616DE7FE
:10DD70006FF040030B6170E7D0F85C66D0F858365E
:10DD8000F61ACAE7D0F85826074BC5F810621344B4
:10DD9000C5F808324CE700BF602A0120001400409B
:10DDA00068190120504C0120DC1F012070B5D0F80B
:10DDB000A852C1EBC1000C46002605EB80001C21D7
:10DDC000C0F80822C0F8103280F8FC41C0F8146294
:10DDD00080F8FD612B6901FB0451012B01F5FE71F7
:10DDE00008BFC0F80C22DAB228681CB904F0C2FFE0
:10DDF000002070BD05F04AF8002070BD0E4841F2C9
:10DE00000413C35810B5A3B190F8844E00F67460A3
:10DE1000D3F8042234B1002440230121FFF7C6FFC8
:10DE2000204610BD4FF400730121FFF7BFFF2046CD
:10DE300010BD0224204610BD6819012010B50C4CFD
:10DE4000D4F8603663B10B49013BD1F8B026C4F871
:10DE5000603612F8014BC1F8B026047013B10123EB
:10DE6000184610BDFFF7CAFF0123184610BD00BFBA
:10DE700068190120504C012013B5074CD4F8B03676
:10DE800003B9FEE701A8FFF7D9FF0028F6D09DF8F7
:10DE9000040002B010BD00BF504C012010B50B684B
:10DEA000064C074AC4F86036C2F8B0060BB1002031
:10DEB00010BDFFF7A3FF002010BD00BF68190120AF
:10DEC000504C012038B5D0F8A84201F00F03626829
:10DED00093422BD80A062BD41C25C1EBC10200208B
:10DEE00005FB014104EB820201F5FE7182F8FD01A0
:10DEF00001220B708A7094F8BC03904216D084F80B
:10DF0000BC234A782068012A09781DD000F53062C8
:10DF100002EB41121568002D00DBF1B9116841F4E4
:10DF2000001111601BB3002384F8BC33002038BDFE
:10DF30001C21C3EBC302012001FB034104EB82025D
:10DF40003C3182F83D00D3E700F5106202EB41124C
:10DF500015680029E2D0002DE0DB116821F0804136
:10DF60001160116841F400111160002BDBD104F540
:10DF70007172217C04F0D2FED5E700BF10B50446D3
:10DF80008021FFF79FFF00212046BDE8104099E760
:10DF900011F0800F01F00F01F0B4D0F8A8424FF05B
:10DFA0001C0042D1C1EBC10500FB0140002604EB7F
:10DFB000850500F5FE7085F8FD6145780170836088
:10DFC000C27005B1C180022A01D10023037194F807
:10DFD000BC33012B1AD00122236884F8BC2341787A
:10DFE000057891422CD003F5006605F00F0103F58A
:10DFF00030638A40F16903EB451341EA0242F26162
:10E000001A68120405D5002384F8BC330020F0BC44
:10E01000704782681D68C2F30A02C07818492A4313
:10E0200042EA804211431960EDE7C1EBC1050126C8
:10E0300000FB014004EB85053C3085F83D60BCE702
:10E0400005F00F06D3F81CC803F5106203F500674E
:10E05000B14002EB451241EA0C01F9611368190461
:10E06000D1D483681668C3F30A03C07804493343E4
:10E0700043EA804343EA855319431160C3E700BF75
:10E08000008000102DE9F04F854D83B02C6E636940
:10E0900013F0010B02D003B0BDE8F08F6269A369F1
:10E0A0001A42F8D06369A26913409E0703D56369D9
:10E0B00003F0020363616369A2691340180379D412
:10E0C0002046436982691340590300F1D4804269B4
:10E0D00083691A4200F1B9804369826913401A05C5
:10E0E00008D5D4F80838DB0700F15383436903F4FB
:10E0F000006343614369826913401F0110D543697E
:10E1000003F00063436195F85434002B40F04A82D9
:10E11000012385F85434436DC3F38303C5F85834A1
:10E12000436982691340DE0400F1D3814369826947
:10E1300013409A0400F17681436982691340DB063B
:10E1400012D5836923F010038361236AC3F343422A
:10E1500003F00F01022A00F0E582062A00F05E8239
:10E16000836943F0100383614369826913401F0789
:10E1700000F10D82436982691340DE0200F10282E0
:10E180004369826913409C0200F1F7814369826907
:10E190001340590000F1EC814369826913405A072A
:10E1A0007FF579AF4468630700F1E78243681C4359
:10E1B000446070E7D4F81868D4F81C381E40360C58
:10E1C0003FF47EAF374B20460027CDF800B099468C
:10E1D00006E0760807F1010709F11C0900F0328218
:10E1E000F107F6D5F9B200F5306A0AEB41129268F0
:10E1F000D0F8143802EA030818F0010F40F0288222
:10E2000018F0080F40F05C8218F0100F05D004F5EC
:10E210003063102203EB47139A6018F0200F09D0E7
:10E22000296F012900F0568304F53063202203EBA7
:10E2300047139A6018F4005FCBD004F530634FF4B5
:10E24000005203EB47139A60C3E7D4F8043823F075
:10E250000103C4F8043895F85434012B00F0B78159
:10E26000D5F8603493F8752283F87422436903F07B
:10E270000043436130E7D0F81838D0F81C2803EA8F
:10E2800002081FFA88F8B8F1000F3FF420AF054EDE
:10E290004FF0000A04F51067CDE9004B0CE000BF19
:10E2A00068190120C81901205FEA58080AF1010A1B
:10E2B00006F11C0600F0C98118F0010FF4D05FFAD6
:10E2C0008AF9D0F81028D0F8344800F5106309F026
:10E2D0000F0103EB4913CC409B68E401E4B2144303
:10E2E0001C40E20732D54FF0010E009B0AF00F0CE4
:10E2F00007EB4A12D3F834180EFA0CFC21EA0C0191
:10E30000D5F870C0F445C3F83418C2F808E003D15A
:10E31000D6E911231344B364D5F860B4B9F1000F02
:10E3200040F0E681DBF86C32022B00F0D88233F04B
:10E33000040300F01A839BF87832012B02D10023EA
:10E340008BF87832BCF1010F00F0F182230703D57E
:10E3500007EB4A1308229A60E10603D507EB4A133C
:10E3600010229A60620603D507EB4A1340229A6096
:10E37000A30703D507EB4A1302229A60210693D51F
:10E38000D6E91441A1428FD8621A736C00EB4A1C83
:10E3900093420CF5106C28BF1346DCF818200333A9
:10E3A00092B2B2EB930F2ED309F10109864600EB2E
:10E3B00009393CB3A14280F0C682621A736C95F8A9
:10E3C00070009A4228BF1A46B36C02F1030B4FEA61
:10E3D0009B0B70B990B2033080080AD003EB800128
:10E3E00053F8040B8B42C9F80000F9D1B36CD6E99D
:10E3F0001441DCF818001344114480B2B364716511
:10E400008345D6D97046A142FFF44EAF0AF00F0102
:10E410000124D0F8342804FA01F122EA0102C0F8FC
:10E42000342841E7D0F8001900F50063B84A0A40E3
:10E43000C0F800299A6802F00602042A00F0CB8096
:10E440005A6842F480725A609B6813F0060340F0E9
:10E45000AA81C268EB6622F47052C260C36843F4BA
:10E460001053C3604FF00009D5F860644FF04008C6
:10E4700000220127434630461146FFF789FD4346F7
:10E48000002230468021C6F84471C6F85081FFF75B
:10E490007FFD0023D6F8A022B761C6F8248086F855
:10E4A0007472C6F86C327360C6F87C32002A00F0D1
:10E4B000EC81D6F88C32304600215B689847D5F85D
:10E4C0006034286E83F81090436903F4005343616D
:10E4D00032E6D4F804284FF4846104F500678D4BCC
:10E4E00022F001027A60016101E0013B02D0026981
:10E4F0009106FAD4D5F864C0BCF1000F16D004F52B
:10E5000010634FF67F3199600BF1010B1A682033CD
:10E51000E34522F4001243F8202CC3F8E811D3F8A5
:10E52000E02122F40012C3F8E021ECD1FB69D5F818
:10E53000902043F00113FB61002A3DD17A6942F239
:10E540002B0313437B613B6943F00B033B61D4F81E
:10E55000003895F8701023F4FE636F4AC4F8003851
:10E5600004F0DCFB286E436903F480534361DDE56E
:10E57000436903F0804343610EE6436903F40013EB
:10E58000436103E6436903F480134361F8E5D5F87A
:10E59000603493F87422032A37D0436903F00803E8
:10E5A0004361E7E5D5F86034042193F8742283F8D9
:10E5B000741283F87522B3E5D7F8843043F00B0367
:10E5C000C7F884307B6C43F00B037B64BFE7002308
:10E5D00085F854344AE6D0F8002942F00302C0F826
:10E5E00000295A6842F480725A609B6813F006034F
:10E5F00040F0D980C368002223F47053EA66C360F8
:10E60000C36843F41053C3602CE7D3F88C22D2695B
:10E61000002AC2D018469047286EBEE7C1EBC10160
:10E6200004F58054C3F30A1305EB81022668D2F87F
:10E630007412C5F824640B442168C2F87432C5F81A
:10E6400028148DE5DDF800B03BE5DDE9004B3EE543
:10E6500004F530634FF0010C2A6F0AEB471A03EB05
:10E66000471B6245CBF808C0D0F840E0DAF8083024
:10E6700000F01681294A964540F0FB801A0440F1CB
:10E68000F3804FF4004218F0080FCAF808203FF456
:10E69000BBAD026CDAF80800204B9A4200F0D08043
:10E6A0001D49D5F86004019205F0C2FC1C4B019A8B
:10E6B0009A4200F2D0800822286ECBF80820A3E509
:10E6C0007B01296F026C03F5306A012904F5306182
:10E6D000824401EB030BDAF80800DDD1104B9A42BB
:10E6E00000F2AE800C49D5F8600405F0A1FCE2E729
:10E6F000DBF88C325B69002B3FF428AE9BF8742268
:10E70000032A7FF423AE584649469847286E1DE6F3
:10E7100000F8FFFF400D03008C1D01200A31544F0B
:10E720000A30544F47F6F07213423FF419ADC3F369
:10E730000A16C1EBC1024FEAC10C3346033605EBA2
:10E740008202B608D2F8682208D004F5805402EBA1
:10E750008607266842F8046BBA42FAD1ACEB010294
:10E7600005EB8202D2F86842D2F874121C440B44C2
:10E77000C2F86842C2F87432F2E4D5F860040122AB
:10E78000D0F88C3280F8742201795B689847286E43
:10E790000CE5D5F86034042193F8742283F87412E0
:10E7A00083F87522A2E423F00403002B3FF422AF88
:10E7B000A74A0326A74BD2F87421A7491344EE6653
:10E7C0008B4240F2C280A54BA54913448B4240F2D4
:10E7D000D480A44BA44913448B4240F2F380A34B52
:10E7E000A34913448B42C0F02481A24BA249134495
:10E7F0008B4240F22181A14BA14913448B42C0F0CE
:10E800001E81A04BA04913448B42C0F01E819F4B38
:10E810009F4913448B42C0F015819E4B9E4913447F
:10E820008B4234BF4FF4E0534FF4C053C2684FF0F3
:10E83000010922F47052C260C2681343C36013E638
:10E84000000403D54FF40042CAF808209349D5F8D4
:10E85000600405F0EDFB296F01297FF42CAF8F4A8E
:10E86000286E04F05BFA26E79B0602D52023CAF83F
:10E870000830C1EBC103D5F8600405EB8303D3F87E
:10E88000682205F0C1F9286EBAE4D6F89032002B60
:10E890007FF40FAED6F89832002B7FF40AAE0EE666
:10E8A0001A0755D57E4A964505D9190403D54FF464
:10E8B0000043CAF808307949D5F8600405F0B8FB80
:10E8C000764A0121286E04F029FA0823286ECAF836
:10E8D000083095E4714A04F021FA286EA4E4DBE9DB
:10E8E00008239A4259D8DBF81C10B1FBF3F203FB62
:10E8F00012120AB98B4268D9DBF88C32DB682BB173
:10E900009BF87422032A01D1584698478021584623
:10E91000FFF7D8FA0023052258461946CBF86C2297
:10E920001A46FFF743FAD5F870C0286E03E5D5F80C
:10E93000B0305AEA03037FF409AD6146574A04F048
:10E94000EDF9286E02E5704660E54FF470536DE70F
:10E950009A0615D52022CAF8082018F0080F3FF4AF
:10E9600053AC026CDAF80800B8E680215846FFF78D
:10E97000A9FAD5F870C0286EDDE44FF4605355E76E
:10E9800013F0280FE9D1464A96452CD91B042AD505
:10E990004FF40042CAF80820DFE7D31A4946D5F8F9
:10E9A000A820DBF8A802CBF820309BB204F04AFC88
:10E9B0004B464A4649465846FFF7F8F9D5F870C025
:10E9C000286EB8E44FF4505330E7DBF870329942C8
:10E9D00092D24B464A464946DBF8A80204F032FC84
:10E9E000CBF87092E4E7DAF81020C1EBC100D9F857
:10E9F0000432C2F3120CD9F8082205EB80001A4445
:10EA0000A3EB0C03C9F80822D0F86822D5F86004FB
:10EA1000C9F8143205F0F8F8D5F870323B437FF4AA
:10EA200032AF1E4A0121286E04F078F9286EFFF7F4
:10EA3000E7BB4FF44053F9E64FF43053F6E64FF49A
:10EA40002053F3E64FF40053F0E64FF41053EDE695
:10EA5000602A0120405327FFFF340C00401E1BFF9B
:10EA60003F420F0000DC0BFF7F4F1200808CF9FE4D
:10EA700020D6130060B6E5FE5FE3160000D3CEFE9D
:10EA800040771B00C05BB3FEC091210000CA91FE1D
:10EA900020753800E05459FEE09C41008C1D012097
:10EAA0000A30544F2DE9F0414FF0FF35324A002330
:10EAB00032482C4603E0013310320B2B14D0917AEC
:10EAC0000429F8D103F5B17100EB0111C979CF0721
:10EAD000F1D4661C116801D0A942ECD21C46013366
:10EAE0000D4610320B2BEAD1631C02D10120BDE888
:10EAF000F081224D04F5B17705EB07139988E9B948
:10EB00002601DFF88480AA19D8F87C3F41F218600A
:10EB10001B491E690023105801EB4421194AB047D4
:10EB2000E0B1022817D141F2CC6205EB07170121B1
:10EB30000020AB58B971013BAB50D8E7DFF84880F3
:10EB400005EB041241F218602601D8F87C3F1058FA
:10EB5000DB689847D7E70020BDE8F08141F2CC623E
:10EB6000032405EB071741F2D061AB58BC710124B7
:10EB7000013B6C54AB50BAE7288B01200C75012087
:10EB800024750120A5EB0008583B0120044B41F2FD
:10EB9000E472995C09B90121995401225A707047B5
:10EBA0000C75012070B50024164D41F2D066164B4D
:10EBB0002046AC5503E0013010330B2814D053F835
:10EBC0000E4C8C42F7D11C78032CF4D16AB10F4B58
:10EBD00003EB40239A4201D0FFF7D8FF00F5B17054
:10EBE000012305EB0010837170BD41F2CC6100F58B
:10EBF000B17304206A5805EB0313013298716A500F
:10EC000070BD00BF0C750120328B012024750120DE
:10EC100038B50020114B9C7B14B11D688D4204D087
:10EC2000013010330B28F6D138BD82B10C4B03EB09
:10EC300040239A4201D1022C01D0FFF7A7FF00F533
:10EC4000B170084B012203EB0010827138BD00F552
:10EC5000B170044B03EB0010827138BD248B01208E
:10EC6000247501200C7501202DE9F04F83B002F0CE
:10EC7000020C019310B9BCF1000F60D1844C41F635
:10EC800038056559002D61D14FF0FF36814F0025C1
:10EC9000B146B046B2463B68984200F0BE8097F855
:10ECA0000EE0BEF1000F62D0BEF1010F15D105F5E7
:10ECB000B17E04EB0E1E9EF807E01EF0010F0CD192
:10ECC0001EF07E0F09D15FEADE1340F0B080D7F866
:10ECD00008E0F24501D9F246A946013510370B2D5F
:10ECE000D9D1751C04D1B8F1FF3F00F0A78046468A
:10ECF00041F2C86806F5B17704EB061E41F21C6AC2
:10ED000054F808504FEA071941F2186B01354EF8D4
:10ED10000B0044F8085004EB07184EF80A5044F86A
:10ED200009500025C8F8045004EB0715AD79042DEF
:10ED300000F2A980DFE805F02139163955000225D7
:10ED4000FFF724FF284603B0BDE8F08F04F5C25753
:10ED500041F63C063F68A65907FB0565A84293D3D8
:10ED6000FFF714FF0025284603B0BDE8F08F2E46BC
:10ED7000013510370B2D8ED1B3E712F0010E6FD194
:10ED800004EB0710019BD51090F80780032B65F367
:10ED9000C71880F8078061D94FF6FF70834228BFFB
:10EDA00003469BB204EB07108380BCF1000F18D020
:10EDB00004EB061041F218630344987B042810D03A
:10EDC00041F2C86C41F2CC654FF0040E54F80C00CF
:10EDD000013044F80C00586083F80EE063590133A9
:10EDE0006351500705D504EB0710C37943F00103C5
:10EDF000C371D30608D504EB0714E379C3F34502C6
:10EE0000013262F34603E371234B012503EB4626EF
:10EE100028460E6003B0BDE8F08F05F5B17704EB2E
:10EE200007164FEA071EB6796EB92E4660E7A84668
:10EE3000013510370B2D7FF42EAF52E7B9F1FF3FAC
:10EE400090D04E4654E741F2C8682E4654F8085018
:10EE5000013544F8085044F80E5065E77346A1E7C1
:10EE60000E4A00230C49D2F87CCF01EB46210C4A14
:10EE7000DCF80860B04700283FF474AF04EB0714D7
:10EE80000223A3715EE70225FFF780FE5AE700BF69
:10EE90000C750120248B012024750120583B012092
:10EEA00011EC0008F0B5154D83B00E462B78022BFF
:10EEB0000FD14FEA102CC4B241F6300700230122D3
:10EEC00001A9E8596044FFF7CFFE012806D003B03E
:10EED000F0BDC0F3D41C00F07F04EDE72B78022BCB
:10EEE000019B04D133F81430336003B0F0BD53F804
:10EEF000243023F07043336003B0F0BD0C75012063
:10EF000010B5144602070B4610D50B4941F2C472E6
:10EF1000581C8B58834204D305D100230120236061
:10EF200010BDFFF733FE2060012010BD21461846BA
:10EF3000BDE81040B6E700BF0C7501202DE9F04197
:10EF40000D46416882B00446C1F308032B44B3F573
:10EF5000007F58D390F91A30591C0AD0304A03F573
:10EF6000B173FF2102EB0313DA796FF30002DA7158
:10EF7000817694F91B305A1C0FD0294A03F5B173DE
:10EF8000FF2002EB0313DA79C2F34501013921EACC
:10EF9000E17161F34602DA71E0762378022B38D012
:10EFA0001F4A02F5C2531B68B5EB432F4FEA4328B3
:10EFB00025DC41F648036768D6583E407242AA42B3
:10EFC0001DDCAB19434512D301AA2169207EFFF74E
:10EFD00097FF012813D16768A5EB0805206908EBA6
:10EFE0000703019A354460619F1B226167602046D8
:10EFF000F9F766FB20B93D440120656000E0002080
:10F0000002B0BDE8F08129440120616002B0BDE892
:10F01000F081616801202944616002B0BDE8F0819F
:10F020000C75012070B5154604460E46FFF786FFA5
:10F0300050B994F8280028B90223C4E90B5684F883
:10F04000283070BD022070BD1DB12046A8470120A8
:10F0500070BD012070BD00BFD0E9011310B48B4218
:10F0600090F91A2038BF0B46511C83600AD0144B0C
:10F0700002F5B172FF2103EB0212D3796FF30003A3
:10F08000D371817690F91B305A1C0FD00C4A03F5CE
:10F09000B173FF2402EB0313DA79C2F3450101399E
:10F0A00021EAE17161F34602DA71C4760022436A13
:10F0B0005DF8044B1146426142600361B2E700BF54
:10F0C0000C75012070B544220021114841F602045C
:10F0D0004DF05AFF0F4B032141F64C001A784FF6C2
:10F0E000FF761D5803F5C050022A1E5341F2E87600
:10F0F00041F60C0418BF0A4600F8181941F6010140
:10F100001D519A5510225A54FFF7A6FF012070BDD9
:10F11000F48C01200C750120B1F904300F2B2DE97E
:10F12000F0410C4682B01646054633D02846F9F722
:10F13000EFFA95F91B800746B8F1FF3F34D02D4B0D
:10F1400041F2186203EB08118A58904212D1183329
:10F1500003EB4823A1882846013109B203EB411390
:10F16000A1803360F9F7D4FA03460120236002B08E
:10F17000BDE8F081FFF70AFD2846F9F7A1FA28B1AA
:10F1800000230120336002B0BDE8F081002002B00E
:10F19000BDE8F0814FF40071FFF7D0FE0028F5D0F4
:10F1A0004FF6FF73A380C1E72846F9F789FA0028D4
:10F1B000E2D10FB9FFF7EAFC38460023112201A97A
:10F1C000FFF752FD0128D7D1019B0B4A9A1A48BF7D
:10F1D00002F2FF12B2F5B05F4FEA622106D24FFA97
:10F1E00081F885F81B80002BB4D1C5E7FFF7CEFC72
:10F1F000019BF6E70C7501202475012030B504460B
:10F20000C06983B010B9012003B030BD0D460023A2
:10F21000032201A9FFF728FD0128F5D1B4F9203018
:10F22000002B03DAFFF7B2FC0220EDE7019A012D73
:10F230004FEA431102EB431303D0022D12D1E5250F
:10F240005554A268DA612278032A04D100221A7781
:10F250005A779A77DA77626AC2F30F415A839982B2
:10F2600003B030BDE268DA61EDE700BF10B50378A6
:10F270000446023B012B037E02D913F0060F5AD13C
:10F2800098063AD494F91A30591C0AD02D4A03F53D
:10F29000B173FF2102EB0313DA796FF30002DA7125
:10F2A000A17694F91B305A1C0FD0264A03F5B1738E
:10F2B000FF2002EB0313DA79C2F34501013921EA99
:10F2C000E17161F34602DA71E076237E1B070BD50C
:10F2D0001C4841F2C873C35C072B01D0FFF756FCF2
:10F2E00041F2C8730022C2540023E26A237084F8FA
:10F2F0002830FAB1BDE81040104700231249E069F8
:10F300001A018A58904206D001330B2BBAD01A0149
:10F310008A589042F8D10B4A03F5B17302EB0313FC
:10F32000DA79C2F34501013921EAE17161F346025C
:10F33000DA71A7E710BD0121FFF760FF0128F9D1BD
:10F34000237E9DE70C750120248B0120B8B138B5D0
:10F35000027822B190F828201AB1002038BD01208F
:10F3600038BD826803244568C162AA4280F82840FB
:10F3700038BF2A468260FFF779FF012038BD01209F
:10F38000704700BF2DE9F04FDFF84C91174683B06E
:10F390008A4699F800300A68022B7BD1D6B241F632
:10F3A00030044FF48071A6EB020859F80450B844B9
:10F3B00005EB12258844BA4208F1FF38B8FBF1F892
:10F3C00064D200F0010BA844032B06EB0704A8EB62
:10F3D00005030CBF80214FF48071A41A8C4228BF12
:10F3E0000C460EB98C4235D20B2201A92846FFF7F4
:10F3F0003BFC012802D003B0BDE8F08F99F8001063
:10F40000DAF80020022902F1010325D0A64210D229
:10F41000019A6FF04040111F304401EB840102EB70
:10F42000800242F8043F914203F10103F9D1DAF876
:10F430000020A61B3244BA42CAF8002002D1BBF118
:10F44000000F39D1BA4205F101051FD299F80030F9
:10F450000026B9E70A22C8E7A642EAD201996FF06E
:10F46000004C881EB44400EB440001EB4C0121F831
:10F47000023F884203F10103F9D1DAE76FF000435C
:10F48000019A4FF6FF71234422F81310012003B0B4
:10F49000BDE8F08F41F6300102F07F06032BC2F386
:10F4A000D41559F80140A6EB020814BF4FF480713F
:10F4B0008021B84425447DE799F80030022BDDD047
:10F4C0006FF04043019A4FF0FF31234442F823107C
:10F4D000DAF80020B6E700BF0C750120F8B590F807
:10F4E00038300446032B4ED8DFE803F002303944AD
:10F4F0002B4B41F2A87EC56841F2C47C187803F515
:10F50000C25153F80C2041F2AC770328096853F834
:10F510000E000CBF80264FF48076226101FB06F1BD
:10F5200005EB4125A0EB4120E560951943F80E005D
:10F53000D85943F80C50A0EB4121E06AD951C4E9F5
:10F540000C2548BB6262012384F83830002115483D
:10F55000FFF754FE012811D1022384F83830626B82
:10F5600004F130010120FFF70DFF012806D103232C
:10F5700084F8383000212046FFF740FE431EDBB2FE
:10F58000012B01D9F8BD022094F82830062BF9D1BF
:10F59000002384F82830F8BD921B2263D3E700BF14
:10F5A0000C750120AC8C01202DE9F04FDFF824818F
:10F5B000012887B00C4698F800608CBF0023012317
:10F5C0001546032E02930B6839D0022E62D14FF4F8
:10F5D00080724FEA1329DFB201920138012823D843
:10F5E000012203929D421AD9384E06F1880A06F18B
:10F5F0001C0B32681AB1DBF8001099424ED0DAF8D1
:10F6000000000023092205A94844FFF72DFB01282B
:10F610001FD002280FD020B123689D42E9D80320D3
:10F62000256007B0BDE8F08F87B1FFF7AFFA022081
:10F6300007B0BDE8F08F022007B0BDE8F08F802250
:10F640000192C3F3D41903F07F07C6E7019A03922E
:10F65000C8E7059ADDF804E0DDE902C198F800305A
:10F66000022B14D0032BE6D152F8273023F070433D
:10F67000B3FA83F30F445B096345236823D00B443B
:10F6800077452360EAD309F101090027C5E732F87D
:10F690001730EDE74FF480720192D2E70C49013A3E
:10F6A000096802EB41224902B2FBF1F203991344CB
:10F6B000B3FBF1F201FB12320AB10B449B1A9D42DB
:10F6C000236096D8ABE7AB42ABD3A8E7B48C01205C
:10F6D0004C8D01200C750120F0B5114D83B00E4604
:10F6E0002B78022B17D14FEA102CC4B241F6300709
:10F6F0000023032201A9E8596044FFF7B5FA012865
:10F7000007D12B78022B019B0CBF23F8146043F820
:10F71000246003B0F0BDC0F3D41C00F07F04E5E723
:10F720000C7501202DE9F043002990F83C3083B09E
:10F73000044614BF02210021042B7BD8DFE803F02C
:10F74000030C3C476900FFF759FD012870D1626B3B
:10F75000002A75D184F83C00404E4FF6F777DFF869
:10F7600004813F4D1BE0B94594BF4FF000094FF0B5
:10F77000010901A9B9F1000F48D1FFF793FB012856
:10F78000494652D1206BFFF7A7FF01284DD1019ABE
:10F790002B68511E22638B4228BF0B462B603378A7
:10F7A000206B032B1FFA80F9DDD1404594BF4FF049
:10F7B00000094FF00109DCE7426B04F13001002041
:10F7C000FFF7E0FD012833D1032384F83C30234BBD
:10F7D00041F2C470E16A41F2A8771A5803F5C255A4
:10F7E000195041F2AC76511A2A68D85902FB01F23D
:10F7F000995900EB422503F5BD5001EB422200214F
:10F80000DD519A51FFF7FAFC012811D1042384F845
:10F810003C3094F82830042B02D1002384F828309F
:10F82000A36B8BB120469847012003B0BDE8F0835D
:10F830000228FAD194F82830042B09D00220F4E7EA
:10F84000022384F83C30B8E7012003B0BDE8F08320
:10F850000023022084F82830E7E700BF0C75012060
:10F86000508D0120F7FFFF0F38B590F83430044673
:10F87000052B42D8DFE803F01E033B0F1868006B2E
:10F880004FF0FF31FFF728FF012836D1E06AB0BB07
:10F89000032384F8343000212046FFF7AFFC012811
:10F8A0002BD1042384F8343094F82830082B2AD044
:10F8B000012038BD41F63803244D00F1300101200C
:10F8C000EA580232FFF770FE01282AD00238C0B28F
:10F8D000012812D8052384F8343094F82830082BF6
:10F8E00016D041F2E57301220220EA5438BDC06A05
:10F8F000216BFFF7F1FE0128CAD0002038BD02239A
:10F9000084F83430F4E70023012084F8283038BD2F
:10F9100000230122022084F8283041F2E573EA54E2
:10F92000E4E705F5C252E368206B41F64401126832
:10F93000685003EB4223E26AC4E9033002B9606213
:10F94000012384F834309BE7004DC6E70C75012095
:10F9500043682DE9F04F164683B0C3F30808002A28
:10F9600000F0DF80704B054689464FF0000AA3F196
:10F97000180BC8F5007495F91A702846B44228BFD0
:10F980003446791C2ED0F8F7C3FE41F218620BEB17
:10F9900007139B58984205D0FFF7F8F8504603B07C
:10F9A000BDE8F08F604B03EB4720224649464044B8
:10F9B000A2444DF077FA002221462846FFF732FB99
:10F9C0000028EBD02B7E1B0706D5584B2A691B68F5
:10F9D0009A4201D3FFF7DAF8361BA1444FF0000832
:10F9E000C7D1DBE7F8F76CFE002846D12846F8F7C8
:10F9F0008FFE6968C1F308031BBB4D4AAB680A4020
:10FA000002F500729A422CBF062207222B7E03F0D9
:10FA10000C030C2B1BD0002301A9FFF725F90128AB
:10FA2000BCD10198404BC31A48BF03F2FF13B3F592
:10FA3000B05F4FEA63224CD257B2AF760028B4D100
:10FA4000ACE72B7E072203F00C030C2BE3D19BF8D1
:10FA500000C0384BBCF1030F1B680CBF4FF0800C8B
:10FA60004FF4807C03FB0CF34FEA432C0CF1FF3C7A
:10FA70000CEA0101A3EB5123CEE72B7E1A072CD50C
:10FA80009BF800202B4B032A95F828201B680CBFFD
:10FA900080214FF48071062A03FB01F34FEA4323D0
:10FAA0003FF47CAF24490868834231D891F83D3057
:10FAB000002B7FF473AF002A7FF470AF06216B69CF
:10FAC000284685F8382085F82810EB62FFF706FDF8
:10FAD0001AE0FFF75BF80198AFE795F82830002BA4
:10FAE0007FF45CAF154B1A78002A7FF457AF0821DA
:10FAF00085F834206A69284685F82810D3F85F30E5
:10FB0000C5E90B23FFF7B0FE01283FF46FAF45E7CF
:10FB100041F2E573012250460BF8032003B0BDE823
:10FB2000F08F92463AE700BF24750120D08C012067
:10FB300000FEFFFF4C8D0120B48C0120F18C0120D0
:10FB40002DE9F04790F8384082B00546032C00F2CA
:10FB50009980DFE804F00218600BFFF785FE0128AA
:10FB60000FD0022809D1032385F8383000202B6CF0
:10FB7000022485F8280003B19847204602B0BDE86A
:10FB8000F08785F838002B78022B50D03E4941F69B
:10FB900048026B688A5803EA0208C8F34F282846CF
:10FBA000DFF8E890F8F7B4FD0646A8EB000802225B
:10FBB00001A930460023FFF757F808EB0607012894
:10FBC0004FF40072BFB24FF00001044606F1010687
:10FBD000D3D101984DF0D8F9EB694FF40071284664
:10FBE0000BB16B684BB3D9F80030013B9F4206D292
:10FBF000FFF7A4F90028DAD1FEF7C8FFD7E7C3EB77
:10FC0000C35328465902FFF799F908B9FEF7BEFF1A
:10FC1000022385F8383000222B6C85F8282053B158
:10FC2000012428469847204602B0BDE8F0876B685B
:10FC3000C3F34F28B3E701249FE7019B4FF0203225
:10FC40002E244FF0100C1A605A601C70C3F8072065
:10FC5000D5F824E01A625A62CEF30F4A83F82040A6
:10FC600083F82140C3F8272083F80BC0EA6BA3F880
:10FC70001AE0C2F30F44A3F814A05A879C8683F8B5
:10FC80002BC0B0E7002478E70C7501204C8D0120D3
:10FC90002DE9F04F90F8303089B00446042B00F283
:10FCA000A780DFE813F0A800B10005008900E70095
:10FCB000B54D41F61003EB5C002B40F09980B34F3B
:10FCC00004F11C0901AEB84607F1380BBA463246BA
:10FCD00049464046FFF720FA012840F01681019876
:10FCE000002800F0F98003780BB1E52BEFD1A84A8A
:10FCF000821A48BF02F2FF12B2F5B05F4FEA6223E8
:10FD000080F03B811B01A34A13449A7B042A0CD048
:10FD100041F2C86641F2CC610427AA590132AA51C6
:10FD20005A609F736B5801336B5041F60202AB5619
:10FD30005E1C09D003F5B173FF2105EB0313A95431
:10FD4000DA796FF30002DA7141F603016B565A1C3F
:10FD50000ED003F5B173FF2605EB0313DA796E5469
:10FD6000C2F34501013921EAE17161F34602DA711A
:10FD7000202200214DF008F92346019A05A853F8E6
:10FD8000315F59681560516019899B7A11819372AE
:10FD9000019B627EDA723FF02FFABDF81430002B1F
:10FDA00040F02E8144F28172019903200A82CB81B6
:10FDB0000A83CB8284F83000237E980600F1A88065
:10FDC0002046FFF749F92369002B00F0AD80237E20
:10FDD00003F0F70213F00403227640F0B380122AF6
:10FDE00000F0B9800022E36A204684F82820984772
:10FDF00009B0BDE8F08F6548FFF72EF94FF6FF72A6
:10FE00000123228484F8303004F11C0801AE5F4FD6
:10FE100004F13109324641463846FFF77DF90128A1
:10FE20002FD00228E4D1584D41F60202AB56591C9E
:10FE300009D003F5B173FF2105EB0313A954DA7957
:10FE40006FF30002DA7141F603016B565F1C0ED0AE
:10FE500003F5B173FF2005EB0313DA796854C2F39D
:10FE60004501013921EAE17161F34602DA710423A7
:10FE700084F830300020E36A2070984709B0BDE86C
:10FE8000F08F019D0B2249462846002D00F0868008
:10FE90002B78002B00F0828095F80BA01AF0080F49
:10FEA000B8D14DF057F90028B4D1637E8AEA030334
:10FEB000DB0640F1C680344D41F60202AB565F1CB2
:10FEC000C1D003F5B173FF2105EB0313A954DA790F
:10FED00060F30002DA71B6E73B78092250462E49FA
:10FEE000022BC4D00B78002BC1D10A708BF80030E4
:10FEF0004A6B0B73C1E9053351F8143CC1E9013277
:10FF0000FFF71EFE01283FF4E2AE0228AFD06FE7F4
:10FF10000023112205A9E069FEF7A6FE01283FF49F
:10FF20004FAF09B0BDE8F08F237E19077FF55AAFB8
:10FF3000154A41F2C873D15C00297FF459AF0721FB
:10FF4000D1544FE70023E26AA168204684F82830A4
:10FF5000FFF768F84CE7E56A0421626A204684F8F6
:10FF60003C306363A56384F828106362C4E90233FC
:10FF7000C4E90B22FFF770F83AE7FEF707FE019895
:10FF80006FF00F03BFE600BF0C750120F48C012059
:10FF900024750120248B01201C8D0120474D41F642
:10FFA0000202AB565E1C09D003F5B173FF2105EBCD
:10FFB0000313A954DA796FF30002DA7141F60301F1
:10FFC0006B56581C0ED003F5B173FF2005EB0313DD
:10FFD000DA796854C2F34501013921EAE17161F32C
:10FFE0004602DA71237EDA067FF541AF3448FFF727
:10FFF00033F84FF6FF720223228484F8303058E63B
:020000040801F1
:10000000304B05A902A8B3F9B4263FF015F99DF8C5
:100010000C309DF80D00DB029DF80A509DF80B2076
:10002000BDF8081043EA401342EA45129DF80E005D
:10003000A1F2BC7143EA500342EA41229BB292B260
:10004000B2E6A98A6A8B204B42EA01421B686262CF
:100050005A02EB69B3FBF2F102FB1131A36009B163
:1000600013445B1A154D41F60202E36084F819A0AF
:10007000AB565E1C09D003F5B173FF2105EB0313EA
:10008000A954DA796FF30002DA7141F603016B5675
:10009000581C0ED003F5B173FF2005EB0313DA797A
:1000A0006854C2F34501013921EAE17161F3460266
:1000B000DA71032384F830307EE600BF0C7501202E
:1000C000F48C0120504C01204C8D01202DE9F04191
:1000D00090F8283084B00446013B082B41D8DFE873
:1000E00003F048054D525865406A4300394B41F6CC
:1000F000480241689F5803F5C253056B0F401B68C7
:10010000EA194FEA4328B2EB432F16D258E021698F
:10011000207EFEF7F5FE012823D1256B6168A5EB53
:10012000080522694144039B3D446261C91B236168
:10013000A84537466160256342D82046F8F7C0FAE3
:1001400003AA06460028E2D06168A3680020E26A9C
:10015000994284F8280038BF1946A1600AB12046A8
:10016000904704B0BDE8F081FFF7EAFC04B0BDE8B9
:10017000F081FFF78DFD04B0BDE8F081FFF776F860
:1001800004B0BDE8F0810021FFF7CCFA04B0BDE86F
:10019000F0810121FFF7C6FA0128E2D10023216C8A
:1001A000204684F82830FFF7D1F8DAE7FFF796F910
:1001B00004B0BDE8F081FFF757FB04B0BDE8F08163
:1001C00020460191F8F77CFA01990028BDD1294415
:1001D0006160BAE70C7501202DE9F04782B0054651
:1001E00018461C4602AF0E4690464AF0D7FB083030
:1001F000013C20F00700ADEB000D0DF1080AD146DF
:1002000014F8013F5BB94246314689F80030284670
:10021000CDF800A033F050FABD46BDE8F08718468F
:100220003EF056FEC3B2A3F120023F2A88BF20232E
:1002300009F8013BE4E700BF2DE9F0470D46904681
:100240000021442204461E46089F4CF09DFE0123D7
:100250004FF6FF722676628384F828302B782E2B97
:1002600042D004F1310A04F139092E4632782023B4
:1002700010462AB12E2A03D03EF02AFE0136C3B220
:100280000AF8013BCA45F1D130782E2801D17078A7
:10029000013604F1380904F13B0A202318B13EF07D
:1002A00017FE0136C3B209F8013FD14507D03078B7
:1002B00020230028F3D109F8013FD145F7D118F0E8
:1002C000100F84F81980E76214BF03230123237001
:1002D0002B782E2B24D00023204684F83030FFF7D3
:1002E000D7FC2046BDE8F0876B78002BB9D1124BC4
:1002F00041F60C0041F2F47141F2F0721E589A5826
:10030000585841F601016662C4E9022041F2E872E0
:10031000595C61769B5CE76223702B782E2BDAD1D7
:100320006B78002BD7D10323204684F83030FFF7B9
:10033000AFFC2046BDE8F0870C75012001210320A9
:1003400008B549F01FF872B640F02AF82DE9F04FD1
:10035000CF4C8DB04FF00008DFF84893CD4D0090A2
:1003600054F80B0C002800F0FE802DF0E1FB06464F
:10037000002800F0DC81D9F82830E026A4F10B0B2E
:10038000C54F44F8073C002306FB08F604F8033C7D
:1003900054F80B0C2DF0CCFB002800F0E48054F84E
:1003A0000B0C2DF0BDFB14F8023C82465A1E0B2AA2
:1003B0000DD8DFE812F01F003A004600530083001A
:1003C0009B00E200160136014101790191012428C8
:1003D0000CD0009A3AB995F82E26824240F08281DC
:1003E000012204F8032C0D2BD2D186E0012304F85E
:1003F000023CCDE700234D28C4F8C53084F8CD3049
:1004000084F8CE3004D0582808D004F8023CBFE766
:10041000022284F8C43004F8022CB9E7032304F85C
:10042000023C022384F8C430B2E704233C2804F8D9
:10043000023C0BD0BAF13E0F0CD0002304F8023C72
:10044000A6E70A233C2804F8023CF3D1002304F871
:10045000013C9DE7012304F8013C99E7D4F8C5006D
:10046000BB19421C0344C4F8C520022A83F8E7AF35
:1004700094F8CD008AEA000184F8CD1088D1237861
:10048000C02BDAD86278FF2A08D1052BD5D90123F1
:1004900084F8C430072304F8023C79E7A4F8C120AB
:1004A0000022C4F8C930934284F8C320C4F8C520A0
:1004B00014BF0523062304F8023C69E7D4F8C500FD
:1004C000BB19421C0344C4F8C52083F8E7AF94F875
:1004D000CD00D4F8C9308AEA00019A4284F8CD10E0
:1004E0007FF456AF062304F8023C51E794F8CD3070
:1004F0008342A2D10D2304F8023C14F8017C002FA2
:1005000040F0F780654B04AE0894ADF82A7003976D
:100510000FCB86E80F00D4F8C930324608A9D4F8CA
:10052000D10023440993B4F8C130ADF8283094F8D1
:10053000C3308DF82C3001238DF82D3003AB28F01B
:1005400057FB48B1049B314694F8C42058460593A4
:10055000534B049325F030FE0023039E04F8023C25
:10056000002E40F0DC8008F10108E034B8F1030F00
:100570007FF4F6AE0DB0BDE8F08FD4F8C500BA191F
:100580005146431C0244C4F8C53082F8E7AF94F8E2
:10059000CD2094F8CE008AEA0202019384F8CD209F
:1005A000D5223EF03FFF019B84F8CE00072B7FF45D
:1005B000EFAEB4F80530C02B3FF63FAFB4F80320E0
:1005C000C4F8C930A4F8C120A27884F8C32000225E
:1005D0009342C4F8C52014BF0823092304F8023C41
:1005E000D6E6D522014694F8CE003EF01BFF94F8E3
:1005F000CD3084F8CE008AEA0303D4F8C50084F82D
:10060000CD30BB19421C0344C4F8C52083F8E7AFC2
:10061000D4F8C9309A427FF4BBAE092304F8023CF7
:10062000B6E694F8CD30434084F8CD3094F8CE301F
:1006300083427FF402AF55E7D4F8C500BA1951469A
:10064000431C0244C4F8C53082F8E7AFD52294F8C1
:10065000CE0001933EF0E6FE019B84F8CE00052B10
:100660007FF496AEB4F80120B4F80330A4F8C120AA
:100670002278C4F8C93084F8C32000229342C4F819
:10068000C52014BF0B230C2304F8023C80E600BFF6
:100690003F4B0120504C0120583B012054D7050806
:1006A000D4170220602A0120D522014694F8CE00FA
:1006B0003EF0B8FEBB1984F8CE00D4F8C500421C49
:1006C0000344C4F8C52083F8E7AFD4F8C9309A4290
:1006D0007FF45EAE0C2398E694F8CE3083427FF42C
:1006E000ACAE07E723287FF47EAE022204F8032C89
:1006F00079E6012F4FF0000602D004F8026C32E7D1
:10070000D4F8C93008A8089423440993B4F8C13038
:10071000CDE90A66ADF8283025F0C4F9EDE754F8C4
:100720000B0C25F0A9FF54F80B0CB0471BE714F88D
:10073000033C002B3FF417AFD9F8282054F8071CCE
:10074000521A632A7FF60FAF012B29D0022B7FF4B8
:100750000AAF54F80B3C012285F8C906C5F8B83633
:10076000C5F8BC36C5F8C436402385F8B62685F8EA
:10077000C8360C4A0C4B0D48C5F8C026C5F87C3568
:10078000C5F80C3734F04CFF4FF4005028F090F8C7
:10079000074834F03BFF85F8106785F81167E2E6FB
:1007A000FFF7CCFD79DB030810530120865C0608B7
:1007B000BC5C060803460A2201481A80704700BF45
:1007C000F00301200346202201481A80704700BF31
:1007D000FC0301200346202201481A80704700BF15
:1007E0001C0401200346202201481A80704700BFE4
:1007F0003C04012003460A2201481A80704700BFCA
:100800005C0401200023D0F8982218461373704727
:100810000346222201481A80704700BF6804012065
:100820000346222201481A80704700BF8C04012031
:100830000346222201481A80704700BFB0040120FD
:1008400003460A2201481A80704700BFD4040120E1
:100850000346432201481A80704700BFE00401208C
:100860000346432201481A80704700BF2405012037
:100870000346432201481A80704700BF68050120E3
:10088000D0F8943283B110B5D0F8904294F80002B9
:10089000FF2807D09B68214694F801229847FF2340
:1008A00084F80032002010BD0020704701F00F01D5
:1008B000D0F8A822C1EBC10102EB810238B5D0F813
:1008C0009032D0F89452D2F8144203F50371EA68DA
:1008D000D3F80402C3F80C429047002038BD00BF93
:1008E00008B5D0F88C325B689847002008BD00BF7F
:1008F00008B5D0F88C321BB11B68984700B908BD09
:10090000022008BD0022836BA3F85A20A3F85220CE
:10091000704700BF836B1A6810B45C6F986F916862
:10092000090601D5212C1AD09168490601D5222843
:1009300006D0DA6F5DF8044B42F01002DA677047B8
:1009400000202024A3F85A00116821F4907111604E
:10095000916821F00101916018669C67E9E7002128
:100960002024A3F85210116821F0C00111605C67C7
:10097000DAE700BF704700BF704700BFC369B3F537
:10098000807F12D0826B002120201368A2F85A10B9
:10099000196821F480711960996821F0010199604A
:1009A000996821F04001996090677047C369B3F579
:1009B000807F0CD0826B00211368A2F852109A68D5
:1009C00022F080029A601A6842F040021A60704772
:1009D00011F0010307D090F8413003F02803282BD1
:1009E0000CBF4223F2238A0709D590F8412002F078
:1009F0002802282A0CBF43F0440343F0F4034A07BB
:100A0000016848BF43F0B8030A6822EA03030B6099
:100A1000704700BFC16838B5022903689A699C69AC
:100A20009A68DD680DD1C2F3C21282EA144212F054
:100A3000060206D1816C01318164816C022907D0E4
:100A400038BD0421FFF7C4FF002380F8403038BDD3
:100A500008218264D96180F8402038BD836B002270
:100A6000D3E90E0102650A6593F84120602A02D19C
:100A7000202283F8412070470023202210B5134C18
:100A80004363C462036380F8412080F842304B071F
:100A900012D50268436A526A1A70436A028D0133A2
:100AA00043624AB1438D013A013B02859BB24385C3
:100AB000436C43F0040343640721FFF789FF1021CF
:100AC00002680023D16180F8403010BD0000FFFFB4
:100AD00038B5002580F8425090F84130292B04D0D9
:100AE00090F841302A2B0BD038BD28222123012138
:100AF00080F841200363FFF76BFF80F8405038BD5A
:100B000028222223022180F841200363FFF760FF9F
:100B100080F8405038BD00BF38B50025202280F84D
:100B2000425090F8413080F84120212B0BBF112317
:100B30001223012102210CBF456345630363FFF7C4
:100B400047FF80F8405038BD90F8BC33012B29D0C6
:100B5000012380F8BC330B060ED402681021124B1F
:100B6000116101E0013B02D01169C906FAD40023EA
:100B700080F8BC331846704701F00F010A4B890119
:100B800010B441F020010468216101E0013B02D072
:100B900022699206FAD4002380F8BC3318465DF827
:100BA000044B704702207047400D030011F0800F86
:100BB0004FF01C0301F00F0170B432D103FB0103AD
:100BC000C1EBC102002400EB820203F5FE7382F840
:100BD000FD41197090F8BC23012A31D0012102682F
:100BE00080F8BC135C781D7802F500638C422AD033
:100BF00005F00F04DE6B02F53062A1401C4C02EBE5
:100C0000451226EA0146DE63DD6925EA0141D96124
:100C100013681C401460002380F8BC33184670BC75
:100C2000704703FB0103C1EBC102012400EB820208
:100C30003C3382F83D40197090F8BC23012ACDD195
:100C4000022070BC704705F00F01DE6B02F51062E8
:100C50008C40084902EB451226EA0406DE63DD6992
:100C600025EA0404DC61136819401160D3E700BF72
:100C70000078F3EF007833EC836B40221A645A6CEF
:100C800042F004025A647047704700BF836B1A6CCD
:100C900012F0500F1A6C20D142F4007219681A64D5
:100CA0008A6812F0405F1AD19A69C2B9CA6A12F40E
:100CB000700F02D08A68500511D44A6822F02002D1
:100CC0004A601A6C22F480721A641A6CD10406D439
:100CD0001A6C42F001021A647047D20600D57047C0
:100CE0009B6BDB6C184700BF836B0121002283F8EC
:100CF0003D101A77704700BF0122836B83F83D20B7
:100D0000704700207047114A1068A8B153689BB122
:100D100088420FD88B4234BF00230123DBB243B19A
:100D2000D368916099421FBF094B1420D16083F8AA
:100D3000BB0170470023F1E7A1F59C53083BB3F5D5
:100D40007A7F2CBF00230123E9E700BF608D0120DB
:100D5000F0030120054B5A7C19748A421FBF044AD4
:100D60001420597482F8BB01704700BF608D0120C8
:100D7000F0030120704728B1034B987C012894BFF1
:100D800000200120704700BF608D012008B5FFF7EB
:100D9000F2FF50B1054AD37C127C5B0003F00203E2
:100DA000002A18BF43F001030B6008BD608D0120CD
:100DB00008B5FFF7E0FF10B1014B5B690B8008BD80
:100DC000608D012070B5FFF7D6FF50B10A4A158B30
:100DD00035B1D6690023B3421C4603DB002000E096
:100DE0000D7070BD02EB44040133248CDBB2AC42C5
:100DF000F1D10B70F5E700BF608D012008B5FFF75A
:100E0000BAFF10B100230B70137008BD04207047A7
:100E100028B1034B93F9BC01003818BF012070477B
:100E2000F003012008B5FFF7F3FF50B1054B93F92C
:100E3000BC21012AC9BF93F8BF310020C3F340038E
:100E40000B6008BDF003012008B5FFF7E1FF18B102
:100E5000024B93F8BE310B7008BD00BFF0030120B8
:100E600070B5FFF7D5FF38B10E4C94F8BF31DB07F2
:100E700003D500230B70137070BD0B4D94F9BD3179
:100E800095F8306093FBF6F301330B7094F9BD4194
:100E900095F8301094FBF1F301FB13430133137009
:100EA000EAE700BFF0030120608D012003207047B6
:100EB0000A4A70B592F8343006255E1CB6FBF5F48C
:100EC00005FB146492F83550AC421EBF02EBC3031D
:100ED00082F83440C3E90E0170BD00BF608D01206F
:100EE000002230B504461046914200DC30BDA35CC0
:100EF0000825584010F0800F4FEA400318BF83F0D8
:100F0000D503013DD8B2F5D10132EDE710B5D9B125
:100F10000E4B986E814217DCB2B11B6B9A4213DC08
:100F2000013A01390A4C03FB012104F5E37084F80E
:100F3000CA110521FFF7D4FF062184F8CB0104F57F
:100F4000E370BDE81040B3E710BD00BF608D012025
:100F5000F00301200023038083708380C38003811A
:100F6000704700BF074A084992F86C30097801338E
:100F7000DBB2994282F86C3004BF002382F86C30F7
:100F8000704700BF608D012070070020F8B5774CD6
:100F9000236F83B1764B1B6893F82E305BB1754B92
:100FA00094F87420A3FB0013012A4FEA93132FD067
:100FB000022A08D002B1F8BD6F4B9842FBD9012339
:100FC00084F87430F8BDA26F64329A423DD894F828
:100FD0006C3004EB031393F88C20FF2A06D0013207
:100FE0006649012083F88C2081F8CC01FFF7BAFF15
:100FF000634B01221B7884F87420092BDBD1B4F8F1
:101000000E31604A01339BB2A4F80E315380F8BD13
:1010100094F86C1004F180055B48002701EB810611
:10102000A367E567022500EB461355480A2684F8B6
:101030008A7000789A70092884F88B6084F874505C
:10104000B9D101314F4B1980F8BD94F88A2094F83A
:101050008B309A42AFD104F17F0004F18805002360
:1010600010F8011F08224B4013F0800F4FEA430194
:101070000B4616BF81F00703CBB2DBB2013AF3D1C6
:101080008542EDD194F88910994238D1B4F8836043
:10109000012794F86C5076BA94F887C004EB0511D8
:1010A000B4F88500B6B294F8883040BA81F88C2044
:1010B00043EA0C23C1F8906094F881C080B294F8A0
:1010C00082601BB2C1F89400032D46EA0C2294F909
:1010D0008000A1F89830A1F88E20284A81F88D0070
:1010E00082F8CC7108D8264A12780C2A29D00D2A09
:1010F00002D1244B23F81500FFF734FF5FE794F883
:101100006C3004EB031393F88C20FF2A06D00132D5
:101110001A49012083F88C2081F8CC01FFF722FFC7
:10112000174B01221B7884F87420092B7FF443AFFE
:10113000B4F80C31134A01339BB2A4F80C319380FC
:10114000F8BD03EB83031149114A03EB830391F8C4
:1011500022100C48F9409B0093FBF1F382FB031231
:10116000DB17C3EBA20320F81530C5E7608D012023
:1011700008150020D34D62103F4B4C00F0030120B6
:10118000F0480120F4480120A0260020B4490120A5
:10119000676666660A4B93F88A1093F88B20914233
:1011A0000DD0C0B210B493F88A20DC6F511CD2B2BB
:1011B000C9B283F88A10A0545DF8044B7047704799
:1011C000608D01200F4B104AD3F81031B2F90000A6
:1011D0005B0707D400EB8000400080B200F5C870C8
:1011E00080B27047094B0A4AD3F8C430323382FBCD
:1011F0000312D817C0EBA20080B200F5C87080B20D
:10120000704700BF608D0120844B0020043A01200C
:101210006766666680F08003042B70B520D941288C
:101220001ED0FD2806D0F0281DD0EF281FD00224A4
:10123000204670BD0B2004260F4D2E44002401359E
:10124000FFF7E8FF2044AE42C4B2F1D015F8010B1D
:10125000FFF7E0FF2044AE42C4B2F7D1204670BD94
:101260000424204670BD03200526044DE5E70C202C
:101270000626034DE1E700BF105D0608085D06087D
:10128000005D060870B5D0F8A052044695F81832F3
:1012900013B9D5F814323BB981212046FCF712FE70
:1012A0006B7A022B07D070BD6B7A002BF4D1012131
:1012B000FCF708FEF0E705F5037220461F23012125
:1012C000BDE87040FCF772BD70B5037C0446012593
:1012D0007BBB4FF4007302222946FCF759FE4FF402
:1012E0000073C4F85851174E812102222046FCF7A2
:1012F0004FFE321DE5620025D4F8A432C4F8A022C6
:101300002846B581A6F860521B6898470121D4F899
:10131000A802FFF719FC8121D4F8A802FFF714FCFA
:1013200006F5047220461F230121FCF73FFD2846E5
:1013300070BD402302222946FCF72AFE4023C4F850
:101340005851D0E7844B002038B5044600250121D0
:10135000D0F8A802FFF72AFC8121D4F8A802C4F82B
:101360005851FFF723FCD4F8A002E5624BF0DCFDF6
:101370002846C4F8A05238BD38B504468321D0F8B9
:10138000A8020025FFF712FCD4F89802656518B191
:101390004BF0CAFDC4F89852002038BD38B5044659
:1013A00000258121D0F8A802FFF700FC0121D4F824
:1013B000A802E562FFF7FAFBD4F8A8028221C4F87C
:1013C0005851FFF7F3FBD4F8903225644BB1D4F8B1
:1013D00094325B689847D4F890024BF0A5FDC4F8AE
:1013E0009052002038BD00BF10B50823032283218E
:1013F0000446FCF7CDFD0123102063654BF08CFD06
:10140000C4F8980218B103460020187310BD0220DA
:1014100010BD00BF2DE9F041037C04460125BBBB94
:101420004FF4007302228121FCF7B2FD29464FF4EC
:10143000007302222046E562FCF7AAFDC4F8585169
:101440004FF001080823032282212046FCF7A0FD6B
:101450004FF40770C4F840804BF05EFD0546C4F8B9
:10146000900258B3D4F8943200271B689847267C22
:10147000C5F814724146D5F804222046C5F8187202
:10148000AEB140233E46FCF791FC3046BDE8F0810A
:10149000402302228121FCF77BFD294640230222C2
:1014A0002046E562FCF774FDC4F85851C8E74FF4D4
:1014B0000073FCF77BFC3046BDE8F0814646E4E76C
:1014C00007B50DF1060212F02DFA68B1084BBDF810
:1014D0000620B3F814111A8391421FBF0549142046
:1014E000A3F8142181F8BB0103B05DF804FB00BF31
:1014F000608D0120F003012013B50446FFF788FC3E
:1015000000B300230DF106022046ADF8063012F0BC
:1015100009FAB8B10C4C9DF8062094F9BC1184F876
:10152000D121032909484FF0050104BF62F07F0271
:1015300084F8D121FFF7D4FC062184F8D2010348B6
:10154000FFF7B6FC02B010BDF0030120BD0501207D
:101550002DE9FF47002304461E200193ADF80C300F
:101560001D4B93F8009093F801A09D78B3F8048088
:10157000DF881E7A20F060FA28B1002F1EBFB8461F
:1015800001254FF00009154A92F81631D9070AD4FF
:1015900092F81B213AB9012E1BD0022E03D113F071
:1015A000020F08BF012501AB8DF80C608DF8049087
:1015B0008DF805A08DF80650ADF80880ADF80A70DA
:1015C00003CB1B88206020466160238104B0BDE806
:1015D000F0873546E7E700BFB8520120608D012053
:1015E000144B30B4D3F8404114B383F84611090AC0
:1015F00000220F2583F8450103F5A27083F84711F7
:101600000121C3F84821C3F84C21C3F8502183F8C5
:10161000445110F8015F01312A440E29D2B2F8D1A9
:1016200083F8522120461022034930BC2CF084BAA2
:1016300030BC7047608D0120A48E0120034B002137
:1016400083F85411C3F85811CAE700BF608D012018
:1016500013B504462620019120F0EEF9019920B936
:10166000204602B0BDE81040BAE702B010BD2DE937
:10167000F743B74C0D46D4F840314BB14FF0020858
:1016800000264FF00109D4F840012CF051FA58B966
:101690000027A37C042B00F25781DFE813F08F00B2
:1016A000E400F7003D014601D4F840012CF038FA7F
:1016B000D4F858315A1C234483F85C0194F854310F
:1016C000C4F85821012B0AD0022B11D0002B70D165
:1016D0000F280CBF84F85491C4F85831D3E7A0F117
:1016E0007203012B01D9762863D184F85481CAE7AB
:1016F000102AC8D197490023012211F8010F0132A5
:1017000003440E2ADBB2F8D194F86A2184F85461BC
:101710009A42C4F85861B6D194F86B31002BB2D11B
:1017200094F85D71732F37D0762F0DD0722FAAD118
:1017300094F85F2194F85E3153EA0223A3D023602A
:10174000B4F860316360A4E794F85F2194F85E31E7
:1017500053EA022397D094F8611194F8602194F829
:10176000650142EA012294F862116361E17494F820
:101770006311A4F86C2184F86E1194F8641141EAA5
:101780000021A4F87011A16801B9A360238B002B7C
:101790007FF47FAF22837CE794F8632194F8623171
:1017A00043EA02231AB2002B3FF46DAFA4F8722172
:1017B0006FE784F85461C4F8586164E7722F44D12C
:1017C00001230022A374644B1B78402B2FD1634E5E
:1017D000A37C94F86EC1208B33804FEA0C33050252
:1017E000B4F86CE103F44053217C05F47065778014
:1017F0006769704514BF042000202B434FEA0E1583
:1018000043EA8133614514BF02210021EDB22B432D
:10181000A5681BB2BD4214BF0825002513432B4306
:1018200018434F4B014393F8BB31B180F380A36E53
:101830001BB1E369002B40F09D801F2249494A48B3
:1018400003B0BDE8F0434BF097BCD4F87431474A7D
:10185000EB1A934201DC0022B5E77220FFF7EEFE9F
:10186000C4F87451F7E7762F03D102230022A37442
:10187000A9E7D4F874313D4AEB1A9342EBDD7620A8
:10188000FFF7DCFE0022C4F874519CE7344ED4F814
:10189000743196F8BB21EB1A82B3344A934230DD9F
:1018A000E27CD2071BD4A168626991420ED089B252
:1018B0004620FFF7CDFE96F8BB310122C4F87451E3
:1018C000013B86F8BB310423A3747CE7218BB4F879
:1018D0006C218A4203D05020FFF7BAFEEBE7217C4F
:1018E00094F86E218A4206D0B1FA81F14920490963
:1018F000FFF7AEFEDFE7142286F8BB211C4A9342B5
:10190000BDDC762FA7D17320FFF798FE03230022BA
:10191000C4F87451A37456E7732F9CD0D4F8741193
:10192000124B691A9942A0DC95E7D4F874310F4A3A
:10193000EB1A93428FDD7620FFF780FE0223002210
:10194000C4F87451A3743EE700231A46A3743AE71F
:10195000608D0120BC8E0120F0480120F448012058
:10196000F0030120C15C0608C30501203F0D030000
:101970003F420F00334D2A23D4F878610DF1020263
:1019800085F8D33120230DF10101304685F8D4319B
:1019900012F05FF830B19DF801109DF8027051EA25
:1019A000070339D1552385F8D531462385F8D6313B
:1019B000202301A9304685F8D73112F044F80346B8
:1019C000214813B1BDF804209ABB20493DF06EF9BF
:1019D000B4F870711E4D87B30DF10301304612F05B
:1019E00035F850B30DF106029DF80310304611F0A2
:1019F00099FF10B3BDF806203B4616492846BA4267
:101A00000CBF20222A223DF051F9B4F87231A4F81B
:101A10007C3103B0BDE8F083304611F0FFFF39465A
:101A200085F8D501304611F0E5FF037885F8D63109
:101A3000BEE709493DF03AF9CAE7084928463DF0B2
:101A400035F9E2E7F0030120C8050120E35C060850
:101A5000CC050120DB5C06082A9C0608E25C06082F
:101A600038B50B680C460E4D5A1C20460A600522FC
:101A70001A700B6895F8BC21591C21601A702368F4
:101A800095F8BF21591C21601A70B5F8C2113DF0BC
:101A9000A3F9236895F8C421591C21601A7038BD38
:101AA000F00301202DE9F0472DED028BFFF7B0F98F
:101AB000C8B31E4B93F9BC01012834DD93F8F24101
:101AC00015461B4F8E1E02EB44089FED1A8A4FF0FD
:101AD0003209454504D12046BDEC028BBDE8F087B4
:101AE00037F802ABB2EE040A07EE90AA26F802AF6E
:101AF000F8EEE70A60EE880A4AF00CF8BCEEC00A7D
:101B0000BAF10E0F10EE103A9BB209D91933B3FB9C
:101B1000F9F39BB203EB830303EB83035B009BB2FC
:101B200025F8023BD5E70024D5E700BFF0030120EC
:101B3000DE8E0120CDCCCC3D38B50D46FFF768F9DF
:101B4000044638B10C4890F8BF31DB0704D5B0F833
:101B5000C0012880204638BD084A00F5FA7010F907
:101B6000373C92F8302093FBF2F102FB1132013145
:101B7000013211F0EBFEECE7F0030120608D012053
:101B800038B5134C94F8353094F834209A4219D073
:101B900004EBC3030F49D3E90E200023984212DC63
:101BA00093780D4A5B08C4F890011370FBF7C4FFEB
:101BB00094F8353006210133B3FBF1F201FB123307
:101BC00084F8353038BDD55C013301F8015BE5E7B9
:101BD000608D0120C2520120F0520120AA4B1B78D7
:101BE0002DE9F04F81468BB0002B40F0B680A74E18
:101BF000D6F87851002D00F0B080A54AD2F8F8410F
:101C000004F0F021B1F1E02F6CD1C2F8F831D6F830
:101C10009421944266D004930DF11008C8F8043062
:101C20000DF11C0EA8F808309A4BC6F894419A881A
:101C30001F78ADF8142093F801C01A7A93F802A027
:101C40008DF810708DF811C08DF812A08DF8182045
:101C500098E80700AEE803008F49AEF80020C4F30F
:101C60004252895CC4F303428F4202F101021F46D3
:101C700001D1944508D028468DF81C108DF81D2000
:101C800011F064FEADF82000284604F0070B12F0B6
:101C9000B0F8032833D0042835D000239A4501A991
:101CA000284618BF8DF81E3011F0CAFE48B1019BBE
:101CB000C4F3001103F001038B4202D0284611F057
:101CC0006FFF0A2207A940464BF036F950B19DF844
:101CD0001E30BDF81C20BB70BDF820303A80BB80A0
:101CE0003EF024FA96F898A104AFDFF8A8B196F870
:101CF0009831032B7BD8DFE803F00A3376A3674BD8
:101D000013F80B30CAE7664B13F80B30C6E73946B9
:101D1000284611F09BFE044658B107A8FFF718FCAF
:101D20009DF81E109DF810308B4260D0284611F0AF
:101D3000C3FF96F89831013303F0030386F8983116
:101D40000CB99A45D3D196F81631DB0700D524B1EA
:101D50002B68494628461B6898470BB0BDE8F08FB2
:101D600001A8FFF7F5FB96F816819DF8044008F0EE
:101D70000108ECB1B8F1000F39D13A460DF1030179
:101D8000284611F066FE044688B307A8FFF7E0FB7B
:101D90009DF81C109DF803309DF81D208B4203D147
:101DA0009DF81030934222D0284611F08FFFC0E7F3
:101DB000B8F1000FBDD13946284611F044FE044663
:101DC000A8B107A8FFF7C4FBBDF82010BDF810307C
:101DD0008B420CD086F89981284686F89A812B6828
:101DE0009B699847A5E796F81631D80701D50024D6
:101DF0009FE707A9284611F023FE04460028F6D0E5
:101E00001E201FF019FE96F89B3180468342EED0CB
:101E100086F89B0160B1BBF80630002BE7D1079B29
:101E2000D907E4D401212846444611F0B9FE80E7E1
:101E3000079BDA07DBD50146284611F0B1FE78E7AB
:101E40003846FFF785FB07AB97E8070003C31A8006
:101E50009DF810309BB10DF11D0207A9284611F025
:101E6000F8FD0DF11E01284611F0F0FD0A2207A928
:101E700038464BF061F8041E18BF012459E708A941
:101E8000284611F0E0FDECE706530120608D0120AB
:101E9000F0030120B8520120305D0608245D0608D9
:101EA000185D0608FD292DE9F041044684B000F0D4
:101EB000D880F02900F0BC80EF2900F02B814AB1D6
:101EC0000346861803AD002003F8010B9E4205F877
:101ED000010BF9D19B4B0B2003F1090501E013F82D
:101EE000010F814200F0C280AB42F8D14B1E832B20
:101EF00000F29280DFE813F01E01340184003E01FD
:101F0000AA01B001450150015C01900090006201FE
:101F1000620162017801780178015C019000900013
:101F200082018A0190009000900090009000900043
:101F30009000900090009000900090009000900021
:101F40009000900090009000900090009000900011
:101F50009000900090009000900090009000900001
:101F600090009000900090009000900090009000F1
:101F700090009000900090009F01900090009000D1
:101F800090009000900090009000900090009000D1
:101F900090009000900090009000900090009000C1
:101FA00090009000900090009000900090009000B1
:101FB00090009000900090009000900090009000A1
:101FC0009000900090009000900090009000900091
:101FD0009000900090009000900090009000900081
:101FE0009000900090009000900090009000900071
:101FF000900090009000900090009000190119014D
:10200000514B93F8AB11002900F05D81019223F050
:10201000EFF9019AADF80C003AB103AB224413F882
:10202000011B04F8011BA242F9D104B0BDE8F08104
:1020300003214FF00508454FB8440025013701E062
:1020400017F8011B0846FFF7E5F806466019324607
:10205000FFF728FF7019B845C5B2F1D104B0BDE84B
:10206000F0810B214FF00408394FE5E7364BD3F8E8
:10207000100180060CD4002AD7D003AB224413F8F9
:10208000011B04F8011B9442F9D104B0BDE8F081B2
:1020900093F89C01870742D52E4D287D052834BF33
:1020A00002260326142917D97C39C8B20628E2D89B
:1020B0000629E0D801A050F821F000BF9F220108B6
:1020C0009F2201088922010877200108AF22010818
:1020D000A9220108B52201080929CCD90A390A29FF
:1020E000C9D801A757F821F06F220108BB220108C7
:1020F0007720010877200108772001087720010860
:102100007720010877200108772001088122010843
:102110009F2201080C214FF006080F4F8CE70D4B52
:102120000B29187DA7D10126C8E00C4BD3F8C0308D
:10213000039371E70192FFF745F8019AADF80C009F
:102140006AE700BFF45C0608608D0120085D0608A0
:10215000105D0608D0510120005D0608043A0120F8
:10216000684BD3ED767AFDEEE77A17EE903AADF84C
:102170000C3051E7019223F03BF9019AADF80C00C5
:102180004AE7604D95F81631DE0700F1A580B5F8F5
:10219000E831ADF80C303FE75B4B5C49B3F90430F4
:1021A00081FB0301DB17C3EBA103ADF80C3033E770
:1021B000544BB3F80432ADF80C302DE70C39544BC6
:1021C0009FED547AC9B2D3ED9C7A03EB810367EE9D
:1021D000877A93EDAE7A67EE877AFDEEE77A17EEAF
:1021E000903AADF80C3017E70F39474B33F8113000
:1021F00003EB83035B00ADF80C300DE7414B93F824
:10220000163103F00103ADF80C3005E7424B198895
:10221000CD0556BFCB43032303F0010311F0440F58
:1022200018BF042311F0020F18BF072311F4806FA9
:1022300018BF0923ADE70192FEF7C4FF374B019A9F
:10224000D3F8C83043EAC0400390E5E62D4BD3F8FD
:10225000F831ADF80C30DFE62A4BB3F8E81100296D
:1022600034D0019223F03EFD019A80B2D2E62B8A4F
:1022700003EB830303EB83039B00ADF80C30FAE61A
:10228000EB89ADF80C30F6E6EB89254903EBC30387
:102290009B00A1FB03135B09ADF80C30EBE6B3F830
:1022A0009E31ADF80C30E6E66B680393E3E62B68ED
:1022B0000393E0E6AB680393DDE6F6B28DF80C60BD
:1022C0008DF80D00D7E6B3F8C401A3E6D3F80002F9
:1022D00080F3100080B29DE6019220F0E3FFD5ED7F
:1022E000767A019AFCEEE77A17EE903A9BB20028D4
:1022F0007FF44FAF0B49096811F0100F18BF00238E
:1023000047E700BF608D0120805201206766666646
:10231000844B002000007A44A4520120043A01209A
:102320001F85EB51B8510120014B1B681B6A1847F0
:10233000D44A0120024B186808B1836918477047D6
:10234000D44A0120024B186808B143691847704706
:10235000D44A012010B5074C606D40B131F058F8F7
:1023600094F8513013B180F00100C0B210BD0120CB
:1023700010BD00BFCC1E0120002807DB00F01F01AC
:1023800001234009024A8B4042F82030704700BFC9
:1023900000E100E0B1F5805FF0B400F0D4802AD80D
:1023A000102900F0F580B1F5807F4ED1046A1669DE
:1023B00024F4807457689A4B0462016A446821F4DB
:1023C0000071C56941EA0621964E2B40156821F43B
:1023D0008071B04245EA030541EA072173D0924B70
:1023E000984270D0D26800234460C561C263016224
:1023F0001846F0BC7047B1F5803F00F08180B1F520
:10240000801F48D1046A156924F480145668874BEC
:102410000462016A446D21F400112340146841EA0A
:102420000551804D43EA042421F48011A84241EA79
:1024300006515DD07C4B98425AD0D2680023446547
:10244000C26501621846F0BC7047012923D1046AB5
:10245000166924F001045768714B0462016A4468EC
:1024600021F00201856931436E4E2B40156821F041
:102470000101B04245EA030541EA07010FD06A4B6A
:1024800098420CD0D26800234460856142630162A7
:102490001846F0BC70470123F0BC18467047D2E9DB
:1024A000056321F0080124F4807441EA86011C438D
:1024B0009668D36921F0040124F4007441EA86018E
:1024C00044EA4304DEE7D2E9056321F4006124F421
:1024D000805441EA8621966844EA0314D36921F4C2
:1024E000806124F4005441EA862144EA431479E7E8
:1024F0004368956923F4802343EA852343609CE77E
:10250000046A156924F480345668494B0462016AF0
:10251000446D21F400312340146841EA0541414DE6
:102520001C4321F48031A84241EA064155D03E4B7C
:10253000984252D0D26800234465846D826501625E
:102540001846F0BC7047046A166924F48054576832
:10255000384B0462016A456821F40051C46941EABC
:102560000631304E2340146821F48051B04243EAD2
:10257000042441EA073138D02B4B984235D0D26839
:1025800000234560C461026401621846F0BC7047D4
:10259000046A166924F010045768264B0462016A25
:1025A000446821F02001856941EA06111D4E2B4047
:1025B000156821F01001B04243EA052541EA0711F0
:1025C00019D0194B984216D0D26800234460856117
:1025D000826301621846F0BC70474368956923F432
:1025E000803343EA05234360A4E725F480459369DB
:1025F00045EA8315C3E7D2E9056321F0800124F49D
:10260000806441EA8611966844EA8304D36921F024
:10261000400124F4006441EA861144EAC304D3E78C
:102620008CFFFEFF0000014000040140FF8FFFFE11
:102630008FFFFEFFFF8CFFFE70B4344CB0F1804F73
:102640000368A0EB0404B4FA84F44FEA541406D0EF
:102650002CB92F4D2F4A904218BFA8421DD12E4AA7
:1026600023F070034D68821A2B43B2FA82F25209AA
:1026700023F44073D1E902652B430D880360C662E1
:1026800085623CB932B9436943F0010370BC4361D0
:10269000002070470B7C0363F5E702F580629042EF
:1026A00020D002F5784290421CD01C4A1C4DA84212
:1026B00018BF90420CBF0122002224D0194EA5F56C
:1026C0009635A84218BFB042D2D0174A90421AD0CD
:1026D00002F58062904216D08C680A880360C4625A
:1026E0008262D0E70C4A23F07003104D821A4E68C4
:1026F000A842B2FA82F243EA06034FEA5212B7D076
:10270000002AB5D1D1E70022B2E700BF00000140A6
:102710000004004000080040000401400040014067
:102720000044014000480140001C0040000C0040F3
:102730002DE9F04F002383B0DFF810820D68DFF839
:1027400010E203E00133102B00F0B88001229A4020
:1027500032EA050405EA020CF4D14C6824F01007B3
:10276000022F40F0AE80DF0803F0070A4FF00F0B96
:102770000E6900EB87074FEA8A0AD7F820900BFA18
:102780000AFB06FA0AF64FEA430A29EA0B094FF058
:10279000030B46EA09090BFA0AF604EA0B0BC7F821
:1027A00020906FEA060907680BFA0AFB27EA06067B
:1027B0004BEA060606608768C4F3001607EA090BB1
:1027C000CF689E4007FA0AF747EA0B078760476819
:1027D00027EA020216434660C668E7008A6806EAEE
:1027E000090902FA0AF242EA0902C260AAD5D8F837
:1027F000447023F0030903F003020F2647F48047D7
:1028000009F180499200C8F8447009F59C39D8F85C
:10281000447006FA02FA07F480470197444F019E7C
:10282000B842D9F8086026EA0A061AD007F5806788
:10283000B8425ED03F4FB84260D03F4FB84262D0FE
:102840003E4FB84264D03E4FB84266D03D4FB8428A
:1028500068D03D4FB8420CBF0727082707FA02F29D
:102860001643C9F808606FEA0C07DEF80020E6039B
:1028700003F1010354BF3A404CEA0202CEF80020B3
:10288000A203DEF8046054BF3E404CEA0606E202B2
:10289000CEF80460DEF8086054BF3E404CEA0606FD
:1028A000A402CEF80860DEF80C2054BF3A404CEA8F
:1028B0000202102BCEF80C207FF448AF03B0BDE825
:1028C000F08F4FEA430A4FF00309D0F800B0013F00
:1028D00004EA090609FA0AF9012F2BEA090B06FA9C
:1028E0000AF66FEA090946EA0B0606603FF674AF7E
:1028F00061E7012707FA02F21643B2E7022707FA57
:1029000002F21643ADE7032707FA02F21643A8E7DF
:10291000042707FA02F21643A3E7052707FA02F293
:1029200016439EE7062707FA02F2164399E700BF0F
:102930000000024000080240000C0240001002406B
:102940000014024000180240001C024000380240FF
:10295000003C014030B40023154C0168C367256872
:102960000B681B0709D4002220231446436780F814
:1029700070208367204630BC7047CB6913F4001386
:10298000F1D12268521BB2F1007FF6D30A682025EC
:10299000032422F4D0720A608A6822F001028A605D
:1029A000456780F870308567204630BC704700BFAF
:1029B000D8330120436ADA0710B406D50168846A67
:1029C0004A6822F4003222434A609C0706D5016817
:1029D000C46A4A6822F4803222434A60590706D505
:1029E0000168046B4A6822F4802222434A601A0775
:1029F00006D50168446B4A6822F4004222434A60CB
:102A0000DC0606D50168846B8A6822F48052224372
:102A10008A60990606D50168C46B8A6822F4005260
:102A200022438A605A060AD50168046C4A68B4F5E4
:102A3000801F22F4801242EA04024A600BD01B0677
:102A400006D50268816C536823F400230B4353605E
:102A50005DF8044B70474A68446C22F4C00222437C
:102A60004A60ECE70023C0E90033C0E90233C0E963
:102A70000433C0E90633C0E90833C0E90A33C0E9CA
:102A80000C338363704700BF1F4BF0B4595C04469E
:102A9000D2E9023645181069334356696758034333
:102AA00090693343D6690343906A3343174E034317
:102AB0003E40D06A3343635090B16E69176B26F085
:102AC0000706536B3843976B30436861605820F0BA
:102AD000C07018436050635823F4C0033B436350F5
:102AE000566800201368EE60AB60094E6B681E40AC
:102AF000D2E908321E436E60635823F0F05313434B
:102B00006350F0BC704700BFE85C06081F80FCFF04
:102B10000000FFFF30B4614C0346614A655C0C1E47
:102B200018BF0124821A405918BF012220F0010069
:102B3000585192B98CB95B4A002121201160516033
:102B40009160D160116150615A5922F0F0525A518E
:102B50003F2200209A6030BC70475348181A18BFB3
:102B6000012014B908B9514AE6E74C1E18BF0124E8
:102B70001ABB14BB4E4A00202124106050609060A4
:102B8000D060106154615A5922F0F0525A51012913
:102B90000DD0022915D0032924D0042927D00529D6
:102BA00014D006292BD0072935D00120D3E74FF4C4
:102BB0007462002030BC9A60704760B95CB93D4ACD
:102BC000D9E74FF47C1200209A60C4E74FF4746296
:102BD0000020DA60BFE78C1E18BF01245AB954B92F
:102BE000354AC8E74FF0746200209A60B3E73F228D
:102BF0000020DA60AFE738B934B9304ABBE74FF4A8
:102C00007C120020DA60A6E7CC1E18BF01243AB976
:102C100034B92B4AAFE74FF074620020DA609AE7CC
:102C200010B90CB9274AA6E70C1F18BF012412B926
:102C30000CB9254A9FE710B90CB9244A9BE74C1FF1
:102C400018BF012412B90CB9214A94E710B90CB984
:102C5000204A90E78C1F18BF012412B90CB91E4AF4
:102C600089E710B90CB91D4A85E70D4A934203D193
:102C7000072901D11A4A7EE71A4A00202124106050
:102C800050609060D060106154615A5922F0F05247
:102C90005A5100297FF47BAF5AE700BFE85C060871
:102CA0000060024010600240006402401064024074
:102CB00028600240286402404060024040640240B4
:102CC00058600240586402407060024070640240E4
:102CD0008860024088640240A0600240A064024014
:102CE000B8600240B86402400B4B01E0013B10D0D9
:102CF0000269002AFADA0369074A43F00103036113
:102D000001E0013A05D0036913F00103F9D1184637
:102D100070470320704700BF400D0300144B10B4F0
:102D2000046C9C421AD800F530600023012903612D
:102D3000036943F400230361036943F0180303614B
:102D4000036943F0C043036104D14261036843F067
:102D50008023036000205DF8044B7047D0F8003BEF
:102D600000F53060002BE0DA00205DF8044B70477E
:102D70000A30544F4B78012BF0B50D7826D000F572
:102D80003060404C404B00EB45104D6906693440C3
:102D900004610469234003618B6805B14B610469D8
:102DA000C3F31203012A44F400240461046943EAD2
:102DB0000403036105D0036843F00443036000206B
:102DC000F0BDCB68002BF6D04361F4E74B6993B3B9
:102DD00000F510642B4FD1F808C004EB45142A4EBF
:102DE0006345D4F810E00EEA07072761276906EA71
:102DF00007062661266938D946F40026C1F814C0B2
:102E0000CCF31203012A2661266943EA06032361F3
:102E100026D0BCF1000F08D005F00F020125D0F834
:102E2000343895401D43C0F834582368002043F0DF
:102E300004432360F0BD00F51060134EA3F500239A
:102E4000012A00EB4514206906EA00062661206984
:102E500040F400202061206903EA00032361E4D1EB
:102E60000B69002BE1D06361DFE746F40026C3F372
:102E70001203012A2661266943EA06032361CBD1A6
:102E8000EEE700BF0000F8FFFFFF07E02DE9F04389
:102E90004D780F78012D4DD000F530636F4E4C69A1
:102EA00003EB47136E4D1F693E401E611E6935409E
:102EB0001D616CB38D68012A6A4E2C441F6904F1B0
:102EC000FF34B4FBF5F41FFA84FC06EAC44405FBA6
:102ED0000CF544EA0704C5F312051C611C6945EAB8
:102EE00004051D6121D0CA78012A0AD1D0F808282A
:102EF00012F4807F1A680CBF42F0005242F08052F8
:102F00001A601A6842F004421A600020BDE8F0839B
:102F10008C68012A1D69C4F3120444EA05041C618B
:102F20001C6944F400241C61DDD1CA68002ADAD08F
:102F30005A61D8E74B6900F51064002B37D104EBD8
:102F40004714474E454D012AD4F810C00CEA060636
:102F50002661266946F400262661266905EA0605EB
:102F60002561CE7872D0012E59D1D0F8085815F4C9
:102F7000807F25680CBF45F0005545F080552560E1
:102F8000256845F004452560002ABED19BB2033375
:102F90009C08BAD0CA6800F5805302EB840403EBA6
:102FA000073352F8041BA2421960FAD1ADE704EBD3
:102FB0004714D1F808E0DFF8A490C3F31206D4F860
:102FC000108003EB0E0C08EA09090CF1FF3CDFF856
:102FD0009080C4F81090D4F81090BCFBFEFE09EA73
:102FE0000808DFF880C0C4F810800CEACE4CD4F892
:102FF00010E04CEA0E0CC4F810C0D4F810C046EA39
:103000000C062661CE78012E10D0012A22D007F0BE
:103010000F03D0F834789D403D43C0F834582368FE
:10302000002043F004432360BDE8F0832569012AB2
:1030300025F0C0452561256945F00055256194D1ED
:103040000D69002D91D0164665618CE70D69002D44
:1030500089D0F9E70D69002DF6D1E0E70000F8FF0F
:10306000FFFF07E00000F81F70B41D4E056803E085
:103070003468A41AA14226D3AB6913F02003F7D019
:1030800010222023EA61EB61AB699A0701D5002386
:10309000AB62AB69DB0703D4AB6943F00103AB61FF
:1030A0006B6800220F4C202123406B60436C80F83A
:1030B000402043F00403436480F8411080F842202C
:1030C000012070BC7047426C202180F840300A43D8
:1030D000426480F8411080F84230012070BC704793
:1030E000D833012000E800FE2DE9F041DFF85480DC
:1030F00004460E4615460AE09B69DB0602D5FFF73B
:10310000B3FFE0B9D8F800305B1BB34209D823689D
:103110002A46314620469F69BF07EDD50020BDE80D
:10312000F081636C2021002201200B4384F84020B1
:10313000636484F8411084F84220BDE8F0810120E6
:10314000BDE8F081D8330120F0B484460568049FBF
:10315000104E03E03468E41B9C420AD8AC6931EAA3
:1031600004000CBF012400249442F3D00020F0BCE2
:103170007047DCF844302021002201200B438CF8FA
:103180004020CCF844308CF841108CF84220F0BC40
:10319000704700BFD83301200268436B9169126801
:1031A00003B11847704700BFF0B490F841200346C0
:1031B000002A40D02420DC68D3E9002183F84100B4
:1031C000012C106821F0706120F001001060116185
:1031D000916821F400419160996828D041F404413C
:1031E000022C916002D14FF40061516051680020BF
:1031F000134C20269F690C43D3E9041554602943DE
:10320000DC69D56841EA07211F6A25F400453C4383
:10321000D560D1601460116841F0010111605864FB
:1032200083F84160186383F84200F0BC704741F4B2
:1032300000419160DAE702F0FF0180F84010B9E741
:1032400000800002F8B501F00F05012600271C21BF
:10325000C5EBC50401FB050100EB84043C31A2640D
:10326000236584F83C50676584F83D600369B34288
:1032700008BFE264DAB200681DB9FFF77BFD0020E9
:10328000F8BDFFF703FE0020F8BD00BF2DE9F041B7
:103290000A46D0F8A05200270B4E044685F8382283
:1032A0002F7205F50B720D238121C5F82C62D0F821
:1032B000A802FFF7C7FF05F5037220461F2301216F
:1032C000BDE8F041FAF772BD555342532DE9F0477E
:1032D000137882B0914604468A465A2B5CD8DFE8C0
:1032E00013F0CF005B005B0080005B005B005B00C5
:1032F0005B005B005B005B005B005B005B005B00F6
:103300005B005B005B00B5005B005B005B005B008B
:103310005B005B005B00AA0177005B005B0077004D
:103320005B005B005B005B00CD015B00F7015B00B5
:103330005B003C015B00E1005B005B005B005B004D
:1033400029015B005B005B005B005B005B005B00D6
:103350005B005B005B005B005B005B005B005B0095
:103360005B005B005B005B005B005B005B005B0085
:103370005B005B005B005B005B005B005B005B0075
:103380005B005B005B005B005B005B005B005B0065
:103390005B005B005B001802D0F8A012052400203F
:1033A00091F85D325A1C01EBC303D2B283F83C4260
:1033B00083F84002042A15BF4FF0FF354FF0FF3568
:1033C00081F85D2281F85D02284602B0BDE8F087F1
:1033D000D0F8A032002005465881284602B0BDE84A
:1033E000F087D0F8A042002104F10B0304F11D0086
:1033F00003F8011F8342FBD1702094F85C320C2546
:10340000207394F85D02E574984213D004EBC30076
:10341000013390F83C52DBB2A573042B90F8415273
:10342000257690F8400218BF84F85C32607608BFB9
:1034300084F85C121223638199F80430122B98BF30
:1034400063810025284602B0BDE8F08799F8013075
:10345000D0F8A002DB0740F17F8100F112030725BD
:1034600000F10B0483224581C3F10601D44800E03A
:10347000825C03F80129CA18A34292B2F8D1E0E7AE
:10348000D0F8A062D6F81472002F40F02682D0F84F
:10349000A43208469B6898470546002840F05382AE
:1034A000708191E7D0F8A062357A002D40F08A81D2
:1034B00096F91832002BC0F26E81D0F8A43208467B
:1034C0009B6898470746002840F07C82D4F8A432D5
:1034D0005046DB6898470546002840F06082D9F8DE
:1034E0000210D4F8A00209BAD0F86072C6F86412CB
:1034F000B9F807305BBA9BB21944C6F86832B942D2
:1035000000F27182B6F85E12D6F8142203FB01F3C2
:10351000934240F09881B3F5007F4FF001012046BF
:1035200006F10C0228BF4FF4007331729BB2FAF718
:103530003DFC49E799F80150D0F8A03215F002009F
:1035400040F01B82D3F86012D3E9992422448A42C6
:1035500000F2E8810546588136E7D0F8A08298F855
:103560000860002E40F0298198F91832002B80F273
:10357000C781D0F8A43208469B68984705460028C2
:1035800040F04382D9F80200D4F8A06200BAD6F81D
:103590006072C8F86402B9F807305BBA9BB218448D
:1035A000C8F86832B84200F2F680B8F85E2202200D
:1035B00003FB02F3D8F8142288F808009A4240F07E
:1035C000EA80B6F85E324FF4007CD6F8687206F1F5
:1035D0000C05D4F8A422504607FB03F72946A8F8A7
:1035E0000AC06745D2F81080D6F8642228BF674623
:1035F000B7FBF3F39BB2C0470028C0F25A812A46BA
:103600003B46D4F8A8028121FFF71CFEB6F85E52B3
:10361000D6F83432B7FBF5F5D6E99920DF1B2A44FA
:10362000451BC6F83472C6E99925002D7FF409AF11
:1036300003233372C8E6D0F8A07208200022604E3F
:1036400007F11303788107F10B05C3F1070000E0D0
:10365000127A03F80129C2189D4216FA82F2F7D1B4
:10366000D4F8A4325046DB68984700283FF4E9AE0E
:10367000BB7B002563F07F03BB73A5E6D0F8A06297
:10368000002506F10B0306F1170203F8015F9342D0
:10369000FBD1D4F8A43250460DF1020201A95B68B7
:1036A0009847002840F0DF80019B0821BDF80220E8
:1036B0000220013BF17352BA0C211C0EF374F2820A
:1036C0001A0C1B0A34747274B374B0827181B8E638
:1036D000D0F8A0620846D4F8A43206F25E2206F5BD
:1036E00018715B6898470546002840F0CF80D6F8EF
:1036F00060320821B6F85E22013B308252BA7181F5
:10370000180EF373190C72821B0A30737173B37342
:103710005AE6D0F8A07208200022294E07F11303C0
:10372000788107F10B05C3F1070000E0127C03F874
:103730000129C218AB4216FA82F2F7D1D4F8A432AA
:103740005046DB68984700283FF47BAEFB7B0025A2
:1037500063F07F03FB7337E6D4F8A44201EBC101A9
:1037600099F80430E46904EB81042279053293422C
:1037700028BF13464381002B3FF463AE013B9AB24E
:10378000531C0C322344024413F8011D9C4202F8DE
:103790000119F9D155E696F85D3205211A46013333
:1037A000DBB206EBC202042B82F8405282F83C12D4
:1037B00000F0A38086F85D3243E6464601E700BF8D
:1037C00094D70508B6F85E5206F10C08D6F8687270
:1037D0000846D4F8A432414607FB05F7D6F8642220
:1037E000D3F81490B7F5007F28BF4FF40077B7FBEC
:1037F000F5F39BB2C8470028C0F22A81B6F85E02F2
:10380000D6F83432B7FBF0F1D6E99925DB1B0A4430
:103810006D1AC6F83432C6E9992525B920462946DD
:10382000FFF734FDD0E505FB00F3424620460121B9
:10383000B3F5007F4FF0000528BF4FF400739BB233
:10384000FAF7B4FAC0E590F85D3205215A1C00EB96
:10385000C303D2B283F8405283F83C12042A39D011
:1038600080F85D22EDE5D4F8A022022092F85D32C6
:10387000591C02EBC303C9B283F8405283F83C02DF
:10388000042900F0D68082F85D12DAE5D4F8A0228F
:103890000220002592F85D32591C02EBC303C9B225
:1038A00083F83C0283F840520429ECD182F85D523F
:1038B0008AE5D4F8A0220420002592F85D32591C34
:1038C00002EBC303C9B283F83C0283F84052814241
:1038D000D9D1EBE780F85D5276E596F85D320521A7
:1038E00000251A460133DBB206EBC202042B82F834
:1038F0003C1282F840527FF45DAF86F85D5263E57A
:1039000098F85D3205211A460133DBB208EBC2029A
:10391000042B82F8406282F83C1200F08D8088F817
:103920005D328EE593F85D22052411460132D2B254
:1039300003EBC101042A81F8400281F83C427FD0A8
:1039400083F85D227DE5D4F8A0220220002592F8BC
:103950005D3219460133DBB202EBC101042B81F861
:10396000407281F83C0218BF82F85D324FF00503C7
:1039700008BF82F85D72337226E593F85D22052058
:10398000002511460132D2B203EBC101042A81F8AD
:103990003C0281F84052D3D183F85D5214E5D4F84B
:1039A000A022022092F85D3219460133DBB202EB0D
:1039B000C101042B81F8407281F83C0244D082F8A6
:1039C0005D323EE5D4F8A022022092F85D3219461D
:1039D0000133DBB202EBC101042B81F8405281F8C4
:1039E0003C02ECD162E790F85D3205211A460133C2
:1039F000DBB200EBC202042B82F8405282F83C1288
:103A00003FF468AF80F85D321BE5D4F8A0220220B5
:103A100092F85D3219460133DBB202EBC101042B8F
:103A200081F8406281F83C02C9D1354682F85D6276
:103A3000CAE482F85D5204E5354688F85D62C3E465
:103A4000054683F85D02BFE43D4682F85D72BBE443
:103A5000D4F8A0220420002592F85D3219460133E3
:103A6000DBB202EBC101834281F83C0281F8405293
:103A7000A5D11BE7D0F8A01210B50B7A022B07D006
:103A8000033B012B02D80021FFF700FC002010BDF2
:103A900001F21B2291F819120446FFF717FC0028C7
:103AA000F4DA20460121FFF7F1FBEFE7F8B5D0F893
:103AB000A0420546267A5EB1012E07D104F21B22F0
:103AC00094F81912FFF702FC00282FDB0020F8BD44
:103AD000D0F8A832D4F81012D3F83032D4F8142227
:103AE0001F2BC4E98C1208D12D4BD4F80C229A421A
:103AF00003D194F8191201291DD994F85D320021DF
:103B000005205A1C04EBC303D2B283F83C0283F8AD
:103B100040120223042A2846637214BF84F85D22EF
:103B200084F85D12FDF7AEFB0020F8BD28460121A8
:103B3000FFF7ACFBCAE794F81A32013B0F2BDCD835
:103B400004F21B22FFF7C2FB0028237A1DDB013B96
:103B5000022BBBD96189F1B1D5F8A07204F10C0236
:103B60000420D7F83432D7F814425B1A87F8386249
:103B7000A1423872D5F8A802C7F834320B4628BFE4
:103B800023468121FFF75EFBA0E7052BCED0284618
:103B9000FDF778FB9AE72846FFF778FB96E700BF2A
:103BA0005553424370B5D0F89062E6B101EB810500
:103BB00000EB8505EB695BB1D0F8A802C1EBC1044D
:103BC00000EB8404626CB3FBF2F402FB14341CB10E
:103BD0000020C6F8140270BD23462246EC61FFF7B0
:103BE00031FB204670BD022070BD00BF002310B520
:103BF00004241A461946C0F86C42D0F8A802FFF710
:103C000021FB002010BD00BF70B5054641B9D0F8BA
:103C10006C320C46032B10D0052B1FD0002070BD3A
:103C2000D0F88C329B6933B190F87422032A02D108
:103C30009847002070BD022070BDD0E953639E42BA
:103C400012D8D0F88C321B6923B190F87422032A61
:103C500000D198472846FFF7C9FFDFE7C5F86C1287
:103C6000FAF730F9204670BDF61AB342C0F84C613D
:103C700028BF33469BB2FAF799F8204670BD00BFC3
:103C800010B5134602240A460021C0F86C42C0E970
:103C90000733D0F8A802FFF7D5FA002010BD00BF07
:103CA000F0B5002383B00E460446ADF806300B781D
:103CB000D0F8A07213F0600522D0202D19D14A78D7
:103CC000FE2A11D0FF2A14D14A8892B9CD8885B92D
:103CD0001B060ED44FF4807107F503721F23398140
:103CE0000121FAF763F808E04D8815B9CE88012E56
:103CF00073D020460225FAF741F9284603B0F0BDFB
:103D00004B780B2BF5D801A252F823F04B3D01085C
:103D1000733D0108F33C0108F33C0108F33C010842
:103D2000F33C0108F33C0108F33C0108F33C0108B3
:103D3000F33C0108613D01083D3D010890F87432F3
:103D4000032BD6D18B787B60D7E790F87422032AB7
:103D5000CFD102220DF106011D46FFF791FFCCE7FE
:103D600090F87432032BC4D1391D0122FFF788FF6C
:103D7000C3E70979D0F8A802FCF7E6FE3179D4F858
:103D8000A802FCF713FFB38896F9042003F00F0391
:103D9000002A4FF0000203EB830304EB83032ADBCA
:103DA000C3F84421237C9BBB4FF400730222012102
:103DB0002046FAF7EDF80123C4F85831D4F8A07280
:103DC0007B7A022B32D03279D20996D0012B94D053
:103DD00020460121FFF75AFA8FE71A0689D5D0F855
:103DE000A4329B69984703463246204639463B60D9
:103DF000FFF746FF81E79A61237C83B94FF4007394
:103E0000022281212046FAF7C3F80123E362D5E7B5
:103E10004023022201212046FAF7BAF8CBE74023DB
:103E2000022281212046FAF7B3F8EEE720468121ED
:103E3000FAF748F800237B725FE700BF10B50C78F3
:103E400082B00023D0F8982214F06004ADF8063058
:103E500016D0202C0ED14B78023B092B0AD8DFE874
:103E600003F033390909090909093F2F90F8743221
:103E7000032B5AD00224FAF781F8204602B010BD75
:103E80004B780B2BF6D80FF2080C5CF823F000BF30
:103E9000153F0108753E0108753E0108753E010891
:103EA000753E0108753E0108EB3E0108753E0108AC
:103EB000753E0108753E01086D3E0108073F010887
:103EC0008B7800241360D8E7111D01220024FFF72E
:103ED000D7FED2E7114601220024FFF7D1FECCE73E
:103EE0004B8800241B0A5360C7E74B881B0A222B10
:103EF0001FD0212BBED1CA881149092A28BF092207
:103F0000FFF7BEFEB9E790F87432032BB2D18B787D
:103F10009360B2E790F87422032AABD102220DF12C
:103F200006011C46FFF7ACFEA7E702F108010122DB
:103F3000E6E7CA880349362A28BF3622E0E700BFF1
:103F400024060120EC0501202DE9F0410A7884B017
:103F500000270D4612F060060446D0F890328DF826
:103F60000D70ADF80E7016D0202E1AD1CE8806B383
:103F7000120643D519460193D4F894323246687834
:103F80003E46D3F80880C047019BEA882046194680
:103F9000FFF776FE09E04B780A2B20D00B2B28D0B8
:103FA0008BB120460226F9F7E9FF304604B0BDE8A0
:103FB000F081D0F89432324648789B689847304672
:103FC00004B0BDE8F08190F87432032B29D00226AA
:103FD0002046F9F7D3FF304604B0BDE8F08190F8F1
:103FE0007432032BF3D101220DF10D01FFF748FECE
:103FF000DBE790F87432032BD7D0E8E74A78032543
:1040000083F80162394683F800221A46C0F84861F5
:104010003346C0F84C613E46C0F86C52F9F7C6FE14
:10402000C3E702220DF10E01FFF72AFEBDE700BF34
:104030002DE9F0430D784FF0010883B0044680F875
:10404000805205F01F0C4F7800F5207EC44580F8A3
:104050008172CB788E7806EB0326B6B2A0F8826226
:104060004A790B7903EB02239BB2A0F8843291F8D2
:1040700007908A79C0F86C8202EB092292B2A0F80C
:104080008622C0F870220DD0BCF1020F3ED0BCF1E8
:10409000000F19D005F08001F9F714FF002003B0DC
:1040A000BDE8F08305F06002402A67D06A0665D556
:1040B00080212046F9F706FF20460021F9F702FF8C
:1040C000002003B0BDE8F08305F06005202D6FD01F
:1040D000402D6DD0002DEBD1092FE9D801A151F869
:1040E00027F000BFFD4101082B420108B140010843
:1040F00049420108B140010859420108B94201088A
:10410000B1400108E5420108C541010805F060051C
:10411000202D4DD0402D4BD0002DC9D1012FD9B22B
:1041200000F00481032F00F0EF80002FC0D190F841
:104130007422022A00F0CC81032AB9D113F0800F37
:1041400001F00F0303EB830300EB830340F0D881FE
:10415000D3F84431002BABD001F07F03142202FBD3
:10416000030202F5A072002B40F00D8200231360C1
:10417000114620460222FFF783FD8FE794F8742250
:10418000013A022A94D8DBB2032B91D8D4F88C32AE
:10419000714620469B689847B4F88632002B7FF41E
:1041A0007DAF00287FF47AAF2046FFF71FFD75E74B
:1041B000D4F88C32714620469B689847002003B0A3
:1041C000BDE8F083F1B2C14D012985F806123FF632
:1041D0006FAF90F87432022B00F0BE81032B00F019
:1041E000A9818021F9F76EFE00212046F9F76AFEC9
:1041F00095F806122046FCF773FB4FE790F87432EF
:10420000013B022B3FF654AF022A7FF451AF01224B
:10421000D0F87C32C2600BB10323C360022204F1E8
:104220000C012046FFF72CFD38E790F87432013B73
:10423000022B3FF63DAF012E7FF430AF0023C0F8D4
:104240007C32FFF7D3FC29E7012E7FF427AFC0F8BB
:104250007C62FFF7CBFC21E713437FF429AF7F2E6D
:104260003FF626AF90F87432032B3FF421AFF1B242
:10427000D0F8A83280F8761293F8BC23012A11D026
:104280001A68002083F83810D2F8001821F4FE6173
:10429000C2F80018D2F8001841EA0611C2F8001856
:1042A00083F8BC032046FFF7A1FC002E00F07C81C0
:1042B000022384F87432F1E6330A013B062B3FF601
:1042C000F7AE01A252F823F0494401082F44010837
:1042D0001D440108B1400108B1400108074401082C
:1042E000C1430108012A7FF4E3AE90F87432022B37
:1042F00000F2FF80002B3FF4DBAE0023014641F8C3
:10430000083FFFF7BDFCC9E690F87432022B00F0BD
:10431000D380032B7FF4CCAE4F063FF445AF56EA73
:1043200002037FF441AFF9F7CDFD3DE790F8742229
:10433000022A00F0C180032A7FF4BAAE002E7FF477
:10434000ADAE48063FF430AFD4F8A80201F00F013B
:10435000426891423FF628AF13F0800F4FF01C03E4
:1043600040F0268103FB01020025134602F5FE7290
:1043700083F8FD5100231170937090F8BC33012B2A
:104380003FF412AF0121036880F8BC13557811780F
:10439000012D0CBF03F5106303F5306303EB4113EC
:1043A000196821F400111960D278023A012A03D861
:1043B0001A6842F080521A60002380F8BC33F3E69A
:1043C000037C002B7FF474AED0F88C320DF1060024
:1043D0001B6B984707234370BDF806306BB1B4F8E8
:1043E0008622002A3FF4E0AE9A420146204628BFCA
:1043F0001A46ADF80620FFF743FCB4F88632002BCE
:104400007FF44CAED0E6037C002B7FF451AED0F8A5
:104410008C320DF106005B6B9847DDE7F6B2052E96
:104420003FF646AEDFE806F0302820184038037C1F
:10443000002B40F09F80D0F88C320DF106009B6A73
:10444000984702234370C7E7D0F888320DF1060180
:10445000007C1B689847BFE7D0F888320DF1060151
:10446000007C1B699847B7E7D0F888320DF1060148
:10447000007CDB689847AFE7D0F888320DF1060181
:10448000007C9B689847A7E7D0F888320DF10601B9
:10449000007C5B6898479FE7D0F888320DF10601F1
:1044A000007C9B69984797E7D0F888320DF10601A8
:1044B000007C5B6998478FE74D063FF4F9ADF9F74B
:1044C00001FD20468021F9F7FDFCE7E5608D012024
:1044D0004A067FF4EDAD1B064FF000034FF00202D9
:1044E0004CBF00F1140100F5A0710B60FFF7C8FB91
:1044F000D4E5032B7FF4DCAD011DFFF7C1FBCDE557
:104500009B69002B3FF4D4AD01F07F035A1C02EBF2
:10451000820200EB8202002B3FF428AED0F8A812F2
:104520001C2000FB031393F83E30002B3AD00123EC
:1045300013601DE679B3416801293FF435AEC9B275
:10454000FCF7CEF995F8061220466160FCF7D0F929
:1045500002287FF429AEABE500293FF425AE012106
:104560000323416080F87432FCF7C2F902287FF41B
:104570001BAE9DE5D0F88C320DF10600DB6A984742
:104580000223437028E7D0F8A8321C2000FB013337
:1045900093F8FE31C9E70223416080F87432FCF7DA
:1045A0009FF901E61360E3E5012384F8743275E5B1
:1045B00003FB0102012513463C3283F83D50D9E646
:1045C00003682DE9F04F13F0010785B000F0F0808B
:1045D000C44A13F40025916821F400019160C46A73
:1045E0009168B4FA84FE41EA04014FEA5E1E9160CC
:1045F00000F0E380BB49446BD1F88C20B4F5801FF8
:1046000022F4401242EA0402C1F88C2000F0B68184
:10461000B4FA84F413F480124FEA5414019240F077
:10462000D280990600F1E480DE060CD5AD49D1F8C0
:104630008C2022F08072C1F88C20D1F88C20066B7F
:104640003243C1F88C20590408D5A649C66DD1F86B
:10465000902022F440323243C1F890201A0408D549
:10466000A049066ED1F8902022F440223243C1F8CE
:104670009020DE0308D59B49466ED1F8902022F4A5
:1046800040123243C1F89020590608D59549C66BAF
:10469000D1F8902022F003023243C1F890201A068C
:1046A00008D59049066CD1F8902022F00C023243D4
:1046B000C1F89020DE0508D58A49466CD1F89020D3
:1046C00022F030023243C1F89020990508D585497F
:1046D000866CD1F8902022F0C0023243C1F89020BD
:1046E0005A0508D57F49C66CD1F8902022F4407253
:1046F0003243C1F890201E0508D57A49066DD1F8DD
:10470000902022F440623243C1F89020D90408D5A9
:104710007449466DD1F8902022F440523243C1F8DA
:1047200090209A0408D56F49866DD1F8902022F424
:1047300040423243C1F8902013F4001C0ED0694966
:10474000D0F87480D1F89020B8F1006F22F00062A8
:1047500008BF012442EA0802C1F890205E0309D58F
:10476000DFF88081C26ED8F8901021F040710A43C2
:10477000C8F89020190209D5DFF86881826FD8F84F
:10478000901021F080510A43C8F890205A0100F19E
:104790008E80B3F1007F00F09980BEF1000F40F0F1
:1047A0009580012C00F0F180002005B0BDE8F08F6D
:1047B00013F40025BE467FF41DAF2C4613F480127F
:1047C00001923FF42EAFDFF81CC1816BDCF88C2026
:1047D000B1F5800F22F4400242EA0102CCF88C20AD
:1047E00000F0D080002908BF012499067FF51CAF96
:1047F000DFF8F0803C4AD8F840903C49944649F0B4
:104800008059C8F84090D8F8408008F08058CDF81A
:104810000C80DDF80C80D2F8008048F48078C2F873
:104820000080D1F8008005E00A68A2EB0802642A43
:1048300000F2A080DCF80020D205F5D5DFF8A480D6
:10484000D8F8702012F4407C826A02F4407919D0C2
:10485000E14517D0D8F870C0D8F870A02CF4407C8F
:104860004AF4803AC8F870A0D8F870A02AF4803AC8
:10487000C8F870A0C8F870C0D8F870C01CF0010F5C
:1048800040F00581B9F5407F00F0EE80DFF854C0BC
:10489000DCF8081021F4F811CCF808101149C2F323
:1048A0000B02D1F870C042EA0C020A67BCE6DFF8DE
:1048B0003480B3F1007FC26FD8F8901021F000511E
:1048C00042EA0102C8F890207FF467AF054A074921
:1048D000D2F80080964628F08068C2F80080D1F8AF
:1048E00000800AE00038024000700040D833012008
:1048F0000A68A2EB0802642A3CD8DEF80020160100
:10490000F6D46FB1C26A5AB98268DEF8847046681C
:10491000120707F0706742EA86123A43CEF8842005
:10492000002D40F08380019A22B1826BB2F5800F96
:1049300000F081809A010AD5C36842681B06876827
:1049400043EA82135B4A43EA0773C2F88430594B47
:104950001F681A4647F080671F600F6803E00B6806
:10496000DB1B642B06D813681B01F8D5012C7FF4E0
:104970001BAF0AE0032005B0BDE8F08F00244FF024
:10498000010E1BE74FF0010E4BE64A4B4A491C68EB
:104990001A4624F080541C600C6803E00B681B1B53
:1049A000642BE7D813689E00F8D4002D6BD1019BCF
:1049B000C3B1836BB3B93F4A4369D2F888400569F4
:1049C0001B0604F4403443EA85132343C2F88830BD
:1049D000D2F88C30046A23F4F853013C43EA0423F0
:1049E000C2F88C30BCF1000F10D0436FB3F1006FF0
:1049F0000CD183692F4C00691B04D4F8882043EA4A
:104A0000801302F070621343C4F88830294B186891
:104A10001A4640F080501860086803E00B681B1AC3
:104A2000642BA7D813689B00F8D5BDE6426BB2F59E
:104A3000801F7FF478AFDFF87CE0C268DEF8847016
:104A40004668120607F0E04842EA861242EA080287
:104A5000CEF88420DEF88C70C26927F01F07013A77
:104A60003A43CEF88C2065E7DFF84880DFF84CC089
:104A7000D8F8081002EA0C0C21F4F81141EA0C01F4
:104A8000C8F808100AE7436B002B94D08FE7D1F8E1
:104A900000B041F2883A06E0D1F800C0ACEB0B0C54
:104AA000D4453FF667AFD8F870C01CF0020FF3D0C2
:104AB000E8E600BF00380240D8330120FFFCFF0FBA
:104AC000054A064B92680649C2F3822208681344DD
:104AD0001B7ED840704700BF0038024094D70508BD
:104AE000D42B0120134908B58B6803F00C03042B69
:104AF0001DD0082B19D14A684B68496802F03F0263
:104B000013F48003C1F388111ABF0B4800230B482C
:104B1000A1FB000145F09AFF064B5B68C3F301431C
:104B200001335B00B0FBF3F008BD044808BD024848
:104B300008BD00BF0038024000127A000024F400D3
:104B4000F8B504468368B749E669E768B64DD0E929
:104B500004201A43236802431868AB4201EA0001AB
:104B600042EA060242EA0102A1691A605868226A12
:104B700020F4405042EA010240EA07005860996878
:104B800021F4306142EA01029A605FD0A74A934261
:104B90001CD0A74A934200F00581A64A934200F038
:104BA0000F81A54A934200F08980A44A934200F005
:104BB000A180A34A934200F05181A24A934200F09F
:104BC0001D8100230120C4E91833F8BD9E4B9F4A84
:104BD000D3F8903003F00C03134493F82430B6F567
:104BE000004F17D0082BECD801A151F823F000BFDB
:104BF000254D0108674C01080B4D0108C34B010806
:104C0000DF4C0108C34B0108C34B0108C34B01082B
:104C1000954C0108082B06D8DFE803F0B8A59C05E1
:104C200090050505870001200023A3F110014FF630
:104C3000EF729142C5D823F00F02C3F342032168FB
:104C40001343CB600023C4E91833F8BD7E4B7F4A81
:104C5000D3F8903003F00303013B022B40F299801C
:104C6000B6F5004F7FD07849794B89681B68C1F34E
:104C7000423160680A44127ED34003EB5003B3FB19
:104C8000F0F39BB2A3F110020DE0302B99D1B6F5F1
:104C9000004F4AD06268530803F50043B3FBF2F3B8
:104CA0009BB2A3F110024FF6EF718A4289D82268B5
:104CB0000020D3600023C4E91833F8BD624BD3F859
:104CC000903003F44073B3F5007F1BD065D833B345
:104CD000B3F5807F7FF475AFB6F5004F2ED0FFF7A8
:104CE00001FF636800EB5300B0FBF3F39BB2A3F149
:104CF0001002D8E7544BD3F8903003F44063B3F577
:104D0000006F6FD1B6F5004F24D06268514B03EBB2
:104D10005203B3FBF2F39BB2A3F11002C3E7B6F563
:104D2000004F33D0FFF7CCFEDBE76268002053086A
:104D300003F58033B3FBF2F39BB276E7FFF7D2FEC5
:104D40006168034600204A0802EB4303B3FBF1F31A
:104D50009BB26AE7626800203F4B03EB5203B3FB50
:104D6000F2F39BB261E738490020394B89681D682E
:104D7000C1F3423166680A447308127E25FA02F2D2
:104D800003EB4203B3FBF6F39BB24EE7FFF798FE4B
:104D9000D6E7134493F8203021E7B3F5407F3FF482
:104DA00076AF0EE7284BD3F8903003F03003202B7A
:104DB000A8D03FF66AAF002BB1D0102B8CD000E703
:104DC000214BD3F8903003F0C003802B9AD005D844
:104DD000002BA4D0402B3FF47FAFF2E6C02B3FF472
:104DE00056AFEEE605D8D3B1B3F5806F3FF474AF9C
:104DF000E7E6B3F5406F3FF44AAFE2E6124BD3F873
:104E0000903003F44043B3F5004F3FF47BAF3CD800
:104E1000002B84D0B3F5804F3FF45EAFD1E60B4A50
:104E20001EE700BFF369FFEF00100140004400409F
:104E300000480040004C0040005000400014014079
:104E400000780040007C00400038024094D70508FC
:104E5000D42B01200024F4000048E8010D4BD3F8C6
:104E6000903003F44053B3F5005F3FF44BAF07D8E5
:104E7000002B3FF454AFB3F5805F3FF42DAFA0E6B5
:104E8000B3F5405F3FF403AF9BE6B3F5404F3FF40B
:104E9000FEAE96E6003802400368042201F01F01CE
:104EA000186A02FA01F120EA010010B418621A6AC5
:104EB0000A4C114319625A6C42F400425A649A68CF
:104EC0001440062C06D0B4F5803F03D01A6842F097
:104ED00001021A6000205DF8044B704707000100D2
:104EE000034A0130116813685B1A8342FBD3704791
:104EF000D83301202DE9F8433C4E337D012B6DD092
:104F0000012380460F463375F5F72AFF0546002832
:104F10005FD14FF0FF333B60D8F80030012B3DD01C
:104F2000D8E901934B444B4553D9314C2DE0022B2A
:104F30000CBF4FF400734FF44073226922F44072A7
:104F40002261226913432361236923F0F80323615B
:104F5000236943EAC90343F002032361236943F44D
:104F600080332361BFF34F8FF5F7FAFE236923F0F7
:104F70007A032361002835D1D8F8083009F10109F6
:104F8000D8F8042013444B4523D998F80C30002B53
:104F9000D3D0012BCBD14FF48073CEE7144CD8F88B
:104FA0000C3022691B0222F440729BB222612269FA
:104FB00042F0040222612269134343F480332361E7
:104FC000BFF34F8FF5F7CCFE2369054623F00403AA
:104FD0002361002328463375BDE8F883022528465F
:104FE000BDE8F8830546C7F80090F2E7984901202C
:104FF000003C0240754B002108222DE9F0411D685C
:1050000082B080460191D0E9166334689A4022420A
:1050100004D001680F68780700F18A8001229A4065
:10502000224204D0D8F800104969090678D4042235
:105030009A40224204D0D8F8001009688F0767D43C
:1050400010229A40224204D0D8F800100F68380786
:1050500049D420229A40224217D0D8F800100C6878
:10506000E00612D5B26098F83520052A73D00B6897
:1050700013F4802F0B6800F09080190340F19B809F
:10508000D8F83C300BB140469847D8F854303BB381
:10509000D8F85430DA071BD5D8F8002005214C4B3E
:1050A00088F83510A3FB0535136823F00103AD0A1A
:1050B000136002E01368DB0704D5019B0133AB42A8
:1050C0000193F7D90022012388F8342088F835307D
:1050D000D8F84C3023B1404602B0BDE8F041184743
:1050E00002B0BDE8F081B2600A6812F4802F0A684D
:1050F0002AD1D70503D40A6822F008020A60D8F83A
:105100004020002AA5D040469047D8F85C30A0E760
:10511000B260D8F8542042F00402C8F854208FE757
:10512000B260D8F8542042F00202C8F854207EE75A
:105130000F6827F004070F60B260D8F8542042F0DF
:105140000102C8F8542069E71203D8D5D8F84820DE
:10515000002AD8D17DE70A68D8F8404022F016022C
:105160000A604A6922F080024A6154B30A6822F058
:1051700008020A603F220024012102FA03F3D8F852
:105180005020B36088F8344088F83510002AA7D042
:10519000404602B0BDE8F041104713F480737FF43D
:1051A0006FAF0A68012422F010020A6088F83430D8
:1051B00088F8354064E7D8F84430002B7FF463AFBB
:1051C00063E7D8F84820002AD0D1D3E7D42B0120B8
:1051D000B5814E1B90F835200346022A03D0802269
:1051E00001205A65704702680521002083F83510B8
:1051F000136823F001031360704700BF70B5324A93
:10520000002590F84130044680F84250283BC262A5
:105210004585426C022B41EA020141642BD80321EF
:10522000FBF7D6FB2822294B80F841204363056316
:105230002268136813F4804312D01368A06B23F420
:1052400080431360B0B1224A0023026584F84030E5
:10525000FFF7C0FF70B1A06BBDE87040036D184749
:10526000116811F4004114D194F84130602B24D01E
:1052700084F8401070BD0721FBF7AAFB90F841307D
:10528000602B02D0202380F8413000232363636326
:10529000CEE71168E06B21F4004111600028E9D0ED
:1052A0000B4A026584F84030FFF794FF0028E1D0F4
:1052B000E06BBDE87040036D1847202384F8401070
:1052C00084F8413070BD00BF0000FFFFC1530108EA
:1052D0005D0A01080368202270B51E680D46DA6178
:1052E00007210446FBF774FB03683348596841F40F
:1052F000004159605A6802405A609A69910701D585
:1053000000229A629A69D20703D49A6942F0010294
:105310009A6170042BD5A26B1AB11268526892B2CE
:1053200062856A0709D55A6A25F00405636A1A700E
:10533000636A228D013363624ABB638D9BB21BB1EA
:10534000636C43F0040363640023236384F84230F6
:10535000666C636316BBE36A184DAB420DD194F8DB
:105360004130202384F8406084F8413070BD31041E
:10537000D7D5E26B002AD0D1D3E72046FBF7A8FBB4
:105380002023E56284F8406084F8413070BD638D6D
:10539000013A013B22859BB26385CEE7616C2046D2
:1053A000FFF72CFF94F84130282BDFD12946204607
:1053B000BDE87040FBF760BB00E800FE0000FFFFA7
:1053C000F8B590F84030C66A012B00F0848017468B
:1053D0000123CA0604460D4680F8403020D5FB065E
:1053E0001ED5438D9BB2002B62D190F84130B6F1AF
:1053F000007FDBB202D1282B00F0848094F841308A
:105400001021292B2368D96102D116F5803F68D17C
:10541000AA0601D5BB0659D4002084F84000F8BD87
:10542000680710D42A072ED53B072CD594F84130B5
:1054300003F02803282B61D0216808200023C861CD
:1054400084F84030E4E77907ECD5638D9BB27BB1FB
:10545000216825F00405636A496A1970638D606AE2
:10546000218D013B01309BB201396062638521854A
:10547000638D9BB2002BCBD116F5803FC8D0204660
:10548000FBF726FBC4E7A807C2D5B907C0D5638DD3
:105490009BB213B3606A236810F8016B218D9E6282
:1054A000638D01396062013B21859BB26385AFE763
:1054B00003681021D961436C43F00403436436F060
:1054C0008073A5D1416CFFF799FEA1E729462046DC
:1054D000FFF700FFA0E70220F8BD36F0807397D1F8
:1054E000CDE799698A0701D5002199629969CE07AC
:1054F000C5D4996941F001019961C0E72046FBF7E5
:1055000089FA85E7FBF7B8FA82E700BF38B52022B1
:105510000368204D0024DA615A682A401E4D5A6003
:1055200004634463CC06C56205D51022DA61426C7F
:1055300042F0040242649A69910701D500229A62FE
:105540009A69D20703D49A6942F001029A61032151
:10555000FBF73EFA436C90F84120602A0CD01A1EEB
:1055600018BF012243B990F84130212B08D090F8A0
:105570004130222B04D038BD416CBDE838403DE6B7
:10558000202380F8402080F8413090F8423080F8A5
:10559000422038BD00E800FE0000FFFF38B590F85B
:1055A00040300446C06A012B71D0012384F840309A
:1055B000CB0615D5D50613D5D30BC2F3803543EAF8
:1055C0009232D20729D5E26B5AB3DB0729D513688B
:1055D0005B6833BBA36B53B34DB31B685B6826E0BA
:1055E0000B0707D4880601D5930612D4002084F84F
:1055F000400038BD1507F5D594F8413003F0280375
:10560000282B46D0236808220020DA6184F8400065
:10561000EFE72046FFF75EFEE8E723681022DA6135
:10562000E4E7A36B23B31DB31B685B6803BB94F86B
:105630004130282B02D1B0F1007F2ED094F84130B8
:105640001022292B2368DA61D0D110F5803FCDD00C
:105650009A69910701D500229A629A69D20703D408
:105660009A6942F001029A612046FBF731FABDE7E0
:1056700023681022DA61636C43F00403636430F042
:105680008073B3D1616C2046FFF7B8FDAEE702200E
:1056900038BD2046FBF7BEF9A8E72046FBF7ECF93A
:1056A000A4E700BFF8B590F84030012B7BD0012370
:1056B000CD06044680F8403023D5D00621D51022EF
:1056C0002368616B4548DA61626C814242F00402F2
:1056D000626466D0424A914263D0F4211A680A4358
:1056E0001A609A69910701D500229A629A69D207D5
:1056F00003D49A6942F001029A61002084F84000C4
:10570000F8BD0B0631D5570643D523681A6822F039
:1057100040021A60628D92B2002A46D05868618DAC
:10572000C0F309008AB2FF2A4BD8628DE56A91B2B4
:1057300015F5803F2185CDB24BD0E76A2D045A681C
:10574000284E324002433A432A435A60628D521A2D
:1057500092B2628594F84120222A1A680CBF42F462
:10576000004242F480421A60C7E74D0611D5500648
:105770000FD5638D9BB2FBB923685A689101BCD4E5
:10578000E26A12F5803F13D15A6842F480425A60AF
:10579000B3E78B06B1D59206AFD52046FFF7B6FE2C
:1057A000ABE760219AE70220F8BD5B689E0103D455
:1057B0002046FBF7B1F9A0E740212046FFF71EFD88
:1057C0009BE7FF224FF47F054FF08077114622853B
:1057D000B5E74FF000772D04B1E700BF9D550108F4
:1057E000A5560108009C00FC90F84030012B00F009
:1057F0009C8001232DE9F041044680F84030C80622
:105800000D4690461BD512F0100F18D023681021BA
:10581000D961616C41F0040161649969890701D51E
:10582000002199629969CA0764D5AB0602D518F0C0
:10583000200F71D1002084F84000BDE8F0816B0793
:1058400012D4AF0724D518F0020F21D0606A236864
:1058500010F8016B218D9E62638D01396062013BFE
:1058600021859BB26385E0E718F0040FE9D0216839
:1058700025F00405636A496A1970638D606A218D99
:10588000013B01309BB20139606263852185CCE721
:105890002E0615D46906C8D518F0400FC5D0638D03
:1058A0009BB2002B33D1236859688A01BDD4E16AC9
:1058B00011F5803F27D1596841F480415960B4E720
:1058C00018F0400FB1D0638D9BB2C3B1238DB3B933
:1058D00020684168638DC1F309019BB2FF2B26D973
:1058E0004368FF27204E27853340204E19430E433F
:1058F00046609AE7996941F00101996195E723684B
:105900005B68980103D42046FBF706F98DE7402138
:105910002046FFF773FC88E720462946FFF7F6FD8F
:10592000002084F84000BDE8F08102207047638DBC
:10593000E66A9BB216F5803F23850AD0E76ADBB2A0
:105940004668094A16403E4346EA0343194341600C
:105950006BE74668DBB2044F3E40314341EA034304
:1059600043F00073436060E7009C00FC0000FF010F
:1059700003689A69196810B4D4052ED50C061FD592
:10598000416C4FF4807441F0010141645105DC61C8
:1059900028D5416C4FF48064920541F008014164C0
:1059A000DC6106D5426C4FF4007142F002024264A1
:1059B000D961416C11F00B0F0CD15DF8044B7047AD
:1059C0005405F6D49405F4D50906EBD4416C11F0D6
:1059D0000B0FF2D05DF8044B10E45405F2D5090624
:1059E000D7D4E6E79205DDD4E3E700BFF0B4044680
:1059F00090F834000128A66D38D0012594F83500C0
:105A0000A84284F8345005D00023022084F83430B2
:105A1000F0BC704725680227002084F83570A7681D
:105A200060652868402F20F4802028606B601AD0C1
:105A3000A960EA60E16D3F23226C8B40B3602B6864
:105A400043F016032B606B6943F080036B611AB15E
:105A50002B6843F008032B602B68002043F0010300
:105A60002B60F0BC7047AA60E960E3E70220F0BC5D
:105A7000704700BFF0B490F83530022B38D003687F
:105A800000221D4D2127D9B21E68103926F00106CB
:105A90005F29A5FB0145194C4FF03F011E6004EB47
:105AA00015141A605A609A60DA601A618CBFA2F508
:105AB0008062134A5F6188BF1A4094F8344098BFEF
:105AC0001A404FF0000388BF0432C465A1401C4651
:105AD00082659160436580F8343080F83530C0E9E4
:105AE0000F33C0E91133C0E913332046F0BC7047CF
:105AF000DCB22046F0BC7047ABAAAAAA94D705082E
:105B000000FCFFFF0246F0B44A4C2068002A57D040
:105B100002231168002582F8353082F834500B6872
:105B200023F001030B6003E023681B1A052B3FD809
:105B30000B68DD07F8D4D2E90130D56803430F685C
:105B4000D2E904402B432343146AD2E90665034398
:105B50003948334338402B43556A2343042D40EAE8
:105B6000030030D008604B6923F007031D43CBB21C
:105B7000324C4D61103B3248A4FB03545F2B314B38
:105B80004FF0010500EB14104FF0000403EA01038D
:105B90004FF03F0190F8340088BF04338140D06556
:105BA000204693659960546582F83550F0BC704783
:105BB000032320211846516582F83530F0BC704728
:105BC0000120F0BC7047D2E90B74936A3C43204338
:105BD00008604D6925F007051D4345F00405002FB9
:105BE000C5D07EB1B6F5005F12D0022B03D9032BCE
:105BF000BDD1FB01BBD5012340211846516582F878
:105C00003530D3E7012B11D033F00203AFD1F0E7E9
:105C1000032BACD801A050F823F000BFF75B0108BC
:105C2000F35B0108F75B01082D5C0108B7F1C07F49
:105C30009DD1E0E7D83301203F8010E0ABAAAAAAAB
:105C400094D7050800FCFFFF01F01F01036A10B4A0
:105C500001248A408C4023EA04035DF8044B03626C
:105C6000016A0A4302627047034690F83C0001282B
:105C700000F0C6800220F0B4012483F83D0083F8D0
:105C80003C40002A31D0042A73D0082A1A6800F058
:105C90009580166AC86826F480560D684F688C682F
:105CA000010316622D03D06989B2166A05F42045F6
:105CB00020F4407026F4204640EA0720354320F4C3
:105CC00070400143D1611562D06920F44060D06119
:105CD000D16941EA0421D16100220121104683F8F3
:105CE0003D1083F83C20F0BC70471A68DFF814C1FF
:105CF000166A62450C6826F001064D68C86816628F
:105D00009769166A1DD0B2F1804F1AD0ACF57C4C61
:105D1000624516D00CF5806C624512D00CF5806C93
:105D200062450ED00CF5784C62450AD00CF5705CDB
:105D3000624506D0ACF5943C624502D047F00105BF
:105D400002E027F003073D43000125F0F00526F0AF
:105D50000A0604F00A04C0B28F68344328439061F5
:105D60001462906920F00C0090619169394391614F
:105D7000B2E71A68C868166A0D6826F010064F6800
:105D80008C68010316622D01906989B2166A05F0CC
:105D9000A00520F4407026F0A00640EA0720354315
:105DA00020F47040014391611562906920F44060D5
:105DB0009061916941EA042191618DE7176AC86891
:105DC00027F480770E684C688D68010117623602EF
:105DD000D069C9B2176A06F4206620F0030027F4E0
:105DE000206720433E4320F0F0000143D16116625A
:105DF000D06920F00C00D061D1692943D1616BE7F3
:105E000002207047000001400368012201F01F01D9
:105E1000186A02FA01F120EA010010B418620F4C6E
:105E20001A6AA34241EA0201196212D00C4A934253
:105E30000FD099680B4A0A40062A06D0B2F5803F77
:105E400003D01A6842F001021A6000205DF8044B8A
:105E500070475A6C42F400425A64EAE7000001407D
:105E60000004014007000100F0B490F83D30002B21
:105E700066D0026802233B49B2F1804F80F83D3082
:105E8000A2EB01011368B1FA81F14FEA51113BD045
:105E9000002939D1344D354CA24218BFAA4233D023
:105EA000334F05F50065D71BAA42B7FA87F74FEACB
:105EB00057174AD0002F48D12E4F2F4CA24218BF5F
:105EC000BA420CBF012700274AD02C4DA4F59634C6
:105ED000A24218BFAA4220D004F58064A2423FD05B
:105EE00004F58064A2423BD0816923F08003C4683A
:105EF0000B4341681360D46291620123536180F8BF
:105F00003D300020F0BC7047194F23F070038568C6
:105F1000D71B2B43B7FA87F77F09046923F4407333
:105F200085692343C668446823F080032B431360CC
:105F3000D662946209B9002FDFD043691363DCE7AE
:105F400003F0FF0280F83C2093E70D4C23F0700330
:105F50008568A24243EA0503DFD0002FDDD1ABE71D
:105F60000027DAE70000014000040040000800407C
:105F7000000401400040014000440140004801404D
:105F8000000C004010B4016802240B4A034680F85C
:105F90003D4088680240062A06D0B2F5803F03D013
:105FA0000A6842F001020A600122002083F83D20C5
:105FB0005DF8044B704700BF070001000B4B93F8DE
:105FC0001621D20703D5012283F80722704793F8E0
:105FD00007224AB9D3F8783133B1054B1A78104407
:105FE0005A78114418705970704700BF608D0120B5
:105FF000B852012040F0080210B50D4C84F841223F
:1060000094F9BC21022A06DD420704D583071CBF90
:10601000012384F8C43105210648FAF761FF0621FF
:1060200084F842020348BDE81040FAF741BF00BFC0
:10603000F00301202D06012010B5FAF7E9FEA8B300
:106040001B4C94F9BC31012B30DD59B3022B2DD000
:1060500094F8C4319BB971B180230521154884F8A7
:106060004732FAF73DFF062184F848021148BDE89F
:106070001040FAF71DBF0420BDE81040BAE7002920
:1060800014BF0020042094F8BF311A0748BF40F025
:1060900002005B0701D411B108B940F00100BDE86E
:1060A0001040A7E7022BD3D10420ECE710BD00BFBE
:1060B000F003012033060120F8B5224C030A0546FF
:1060C000062104F2492784F84E0284F84D323846FE
:1060D000FAF706FF94F8BF3184F84F02DB072AD4A1
:1060E000B4F8C021AA4226D1174D41F26F71D4F8FD
:1060F000493205F50276C5F80832C3B2304685F854
:106100000E324FF6FF738A4218BF01230621134453
:10611000C3F3072285F80D3285F80C22FAF7E0FE6A
:10612000072185F80E023046FAF7C2FE052104F574
:106130001470FAF7BDFE07210448BDE8F840FAF7ED
:10614000B7BE00BFF0030120608D01203906012099
:1061500008B5FAF75DFE48B1A1F59C53083BB3F5CD
:106160007A7F03D20846BDE80840A5E708BD2DE9BF
:10617000F0476A4E3368002B3AD0694D694C05F5FB
:10618000DE77306827F0D4FC002833D1664B1988BD
:106190001D46092909D95F8864227A43B2FBF1F2CE
:1061A000452A40F39E811880588094F84932012B8B
:1061B00000F0C281022B00F0DD8133B905215B487C
:1061C000FAF776FE012384F84932594B1D68594B82
:1061D0001B78002B00F0D881574B1B68EB1A782BEB
:1061E00040F2D281D4F89001F7F7A6FCC4F84C52E3
:1061F000BDE8F087306827F093FC94F80F328046B2
:10620000052BBED8DFE803F00309151B3543AA2888
:10621000B7D1012384F80F32B3E7552817BF424A9C
:106220000223938801331CBF9380002384F80F322C
:10623000A7E7032384F8100284F80F32A1E713289C
:1062400084F81102C4F82C0207DD374AD3880133E1
:10625000D380002384F80F3293E718B9052384F81C
:106260000F328EE70023C4F83032042384F80F3253
:1062700087E7D4F83032E218013382F81202D4F8FA
:106280002C22C4F8303293427FF47BAFE6E7D4F897
:106290002C322A4803F1020A4FFA8AF1FAF720FE5B
:1062A000804594F8109240F0148126201BF0C4FB26
:1062B000204B48B100221A701B4A53880133538087
:1062C000002384F80F325CE71A784A4519D100227E
:1062D0001A7009F1FF33102B00F2F680DFE813F09B
:1062E00030008D008D00DE008D00F400F400F4001D
:1062F0003000F400F400F400F400F400F400F400C2
:106300003000B9F1090F02D0B9F1110F01D1012A02
:10631000DDD0054A538901335381DAE7B4520120B5
:10632000F0030120608D0120E2520120400601208F
:10633000882A0120F0520120F4520120708F0120A0
:10634000BAF1060F59DDB9F1010F06D0B9F1090F05
:106350000CBF4FF002094FF0030994F8150294F8AE
:10636000161294F8142241EA002194F912E294F9E9
:1063700014C2900709B294F8133285F8BC9185F8DD
:10638000BDE185F8BFC1A5F8C01106D512F00C0F0C
:1063900014BF0122002285F8C421B9F1030F12D1E4
:1063A000BAF1090F29DD94F918220020082AA8BFA4
:1063B000082222EAE27285F8F22143B201309A42C1
:1063C0005ADC94F817320020D4F81CA09BB2024685
:1063D0005245904658DB7C4B85F8BE011B78232B39
:1063E0000BD109EB8903794A03EB8303A2F802E09E
:1063F00091800CEB8303D08013800A227449754886
:1064000046F09AFD10B1002384F83E32704B3A6892
:106410001A607A685A603A891A8194F83E3233BB1E
:1064200095F8C4316C4A002B117814BF0223012364
:1064300084F8401284F83E3295F8BF3113F001031E
:1064400018BFB1FA81F3517818BF5B0984F8411283
:106450009188D8B29278A4F8421284F83F0284F866
:10646000442213B109B1A4F8461284F848020EF090
:1064700011F80EF00FF81FE704EB4308234493F8DC
:106480001A32A8F87E3198E7013204EB480852B27C
:10649000B8F82080984508BF104699E7BAF1040F74
:1064A000ABDD94F8122294F8133243EA0223590424
:1064B0001AB204D5C3F30D03A5F8C2319DE7002A33
:1064C000F8DBA5F8C03198E7444A938901339381FA
:1064D000F2E619F0010F01BF404A1389013313811D
:1064E000EEE63F4BD3F85822B3F85C12012A1AD1DA
:1064F00041F25632914203D14FF0FF32C3F8582295
:10650000D3F85822306802EB820202EB820201EBE0
:10651000420189B2A3F85C1203681B699847002303
:106520002B806B8041E60132EAD1B1F5965F04BF62
:106530000122C3F85822E3E7294D95F9BC61002EEA
:106540003FF443AE022E11D14FF48040FFF7B4FD6B
:1065500084F8496295F9BC31012B7FF736AE95F886
:10656000BF31C3F3400385F8C4312EE6032384F81A
:106570004932EFE71A4BB3F8C231002B3FF425AE96
:10658000032384F8493220E694F8342094F8353017
:106590009A4204D0FBF7F4FAC4F84C5228E6D4F837
:1065A0004C32EB1AB3F57A7FBFF422AE0D4B1B6869
:1065B000ED1A952D7FF61CAE05210B48FAF778FCF5
:1065C000BDE8F047FBF7DCBAF0480120F4480120B1
:1065D000948F0120AC050120B8520120E252012025
:1065E000F0030120F452012040060120104BD3F8A3
:1065F000780110B5D8B10F4C217841B162780DF017
:10660000A5F9A388834216BF01210021A080E2885A
:106610005AB141F288339342B8BF13469A4204D02C
:10662000E380BDE8104039F081BD0029F9D110BDEB
:10663000608D0120B85201200023014410B410F8ED
:10664000014B0822634013F0800F4FEA43042346B6
:1066500016BF84F00703E3B2DBB2013AF3D18842FC
:10666000EDD118465DF8044B704700BF30B54FF4CC
:10667000806085B021F086FD48B3164C00230121CF
:106680004FF4E13294F8505290F904009D42019188
:1066900000924FF4806118BF08250F4A029521F03F
:1066A000D0FD206700384FF0FF0318BF012084F8A9
:1066B0008C3084F89C3084F8AC3084F8BC3084F89A
:1066C000CC3084F8DC3084F8EC3084F8FC3005B051
:1066D00030BD00BF608D012095110108364B1B684D
:1066E00013F0006359D0354B2DE9F0471F78B842BD
:1066F0004ED3FF2853D1DFF8D8A09AF8CC31002B25
:1067000043D0DFF8D0800022C8E99522C8F85C2287
:10671000A8F86022002F4BD008F18C0310461446D5
:1067200011461546164603EB0719B3F802E010337D
:1067300033F804CC714413F810EC624413F90FCC15
:10674000764509B212B238BF7646654553F80CEC6F
:10675000B8BF654653F808CC994574446044E4D109
:1067600088F8546288F8555291FBF7F192FBF7F2E2
:10677000C8E99640124B0020A8F856121B78A8F8DA
:106780006022092B8AF8CC010CD00E48BDE8F087B6
:106790000D4A02EB0010BDE8F08718467047002054
:1067A000BDE8F08798F85422084B0648DA80F2E7F3
:1067B0003A463946DEE700BFB85101207007002095
:1067C000F0480120B48F0120EC8D0120F448012015
:1067D000F0030120608D012070B40478A51E15F02F
:1067E000FF061DD0451E02464FF6FF73354401E0FB
:1067F00012F8014F1B1BAA429BB2F9D11C0A084494
:1068000010F8012CA24205BF10F8020CDBB20020E8
:10681000C01A08BFB0FA80F070BC08BF40097047CA
:10682000FF244FF6FF73EAE72DE9F8434378434C22
:10683000190703F00F0594F8642200D072B100210B
:10684000AA4284F8681204D94FF000084046BDE817
:10685000F883AA1AD1B20E29F6D803E084F864525C
:1068600084F86822224492F8AC110029ECD003F09D
:10687000F003802B40D0902B49D0A02BE4D10846C8
:1068800065F05F05FAF7C6FC02462D48131D84F833
:10689000695284F86832FBF705FB94F86882B8F116
:1068A000000FD1D0A8F1020313F0FF0641D0254A12
:1068B0004FF6FF71901912F8015B491B904289B2A3
:1068C000F9D15FFA81F90D0A4BB11E4FFE1817F886
:1068D000011BD4F88C0227F051F9BE42F7D149468A
:1068E000D4F88C0227F04AF9D4F88C02294627F014
:1068F00045F94046BDE8F883042365F07F0502268C
:10690000984684F8683284F869523346CFE70846DF
:1069100065F06F05FAF77EFC0426062284F86B0208
:10692000334684F86952904684F86A1284F86822E3
:10693000BDE7FF254FF00208A946C5E7608D01209D
:10694000CA8F0120C88F0120C21D2DE9F04F02F42B
:10695000FC7285B0524C064600AFD4F89032ADEBD5
:10696000020D04F5287A89460DEB0002E8465345EE
:10697000FA602FD094F8E0130DF1010C94F8E103C4
:1069800001F00F0ED4F894520131C7F808C04EEA56
:10699000401E07F1080084F8E0138DF800E0ED1ABE
:1069A000A2EB0C0B1946AB4544DD2A4638F0D0F972
:1069B000D4F89022B96840462A44C4F890A2A1EBCA
:1069C0000801C4F89422C9B2C84700201437BD4654
:1069D000BDE8F08F94F8E05394F8E10305F00F015F
:1069E000B4F99AC2013541EA4011BCF1000F84F8B4
:1069F000E05341F01001D4F89452C9B2A5EB0A0B50
:106A0000B8BF41F08001012888F8001022D1BBF105
:106A1000FE0F38DD07F10800FF2594F8982208F1F1
:106A200003031FFA8BF1786088F8015088F8022080
:106A3000BB6020E05A4638F08BF9D4F890324046DB
:106A400031465B44C4F89032C84701201437BD4634
:106A5000BDE8F08F07F1080094F89C2208F10203CA
:106A6000B4F89812786088F80120BB6038F0B4F967
:106A70001FFA8BF1786838F0AFF97868D7E902C26D
:106A8000D4E9A4358BE794F8981208F1030C07F1C8
:106A9000080088F801B088F80210C7F808C07EE73F
:106AA000608D012010B5062982B004464FF03203F4
:106AB0000A460DF1010028BF062221468DF800305C
:106AC00046F0F0F9024B68461B68984702B010BDCB
:106AD000889101205E2810B50ED05D2804D00B4BA4
:106AE000BDE810405B681847084C636898476368C6
:106AF0003D20BDE810401847044C5D20636898476E
:106B000063683E20BDE81040184700BF889101200F
:106B100070B5084E05460C465E20736898472846B7
:106B200073689847E0B2FFF7D5FFC4F30720BDE8CC
:106B30007040CFE7889101200368002B2DE9F041D8
:106B4000B8BF5B423A4F04463A4DA7FB03013A4EA9
:106B5000890DB27905FB0135C5EB0515AD0087FB45
:106B60000537EB17C3EBA757002A55D101EB81017D
:106B700001EB810107EB810109B2DFF8B880132036
:106B8000FFF7C6FF1B2008FB07552C4FE91787FBB3
:106B90000535C1EBA511264D09B2FFF7B9FF2368F2
:106BA0002320002BB4BF53214E21FFF7B1FF6368B0
:106BB000B279002BB8BF5B42A5FB0301890D08FB2E
:106BC0000138C8EB08184FEA880885FB08354FEAFA
:106BD000E873C3EBA5552ABB01EB810101EB8101F1
:106BE00005EB810109B21220FFF792FF114B134907
:106BF0001A2003FB058581FB0531ED17C5EBA111BB
:106C000009B2FFF785FF63682220002BBDE8F04141
:106C1000B4BF572145217BE7C1EB011107EB81018F
:106C200009B2AAE7C1EB011105EB810109B2DAE76C
:106C30006BCA5F6B806967FF008F0120D34D6210C4
:106C400000234FF4167140F2D93201814281438012
:106C50008380838130B4022515240580847130BC83
:106C60007047084B5A881B88801A9B1AC00090FBFB
:106C7000F3F00628A8BF062020EAE070C0F19600D5
:106C8000C0B270473C8F0120094B03EB40021189D1
:106C9000084A127802EAD122520707D0D3F884209A
:106CA000511CC3F88410134483F88800704700BF58
:106CB0008891012050060120164B426810B51B78C0
:106CC00003F00303032B21D1134B1B88DBB11349C2
:106CD0000A24134BB1F90410B3F9C63091FBF4F157
:106CE0005B1A4FF4B4711B0103F5B9531433B3FBB2
:106CF000F1F3C3F1080303F00F036033137043682B
:106D000000225A7010BD05231370F8E72D2313706D
:106D1000F5E700BFFC8E0120FE8E0120805201208D
:106D200088910120436872221A70732243685A7056
:106D3000742243689A7000224368DA7070470F4BE0
:106D40000A214268B3F9043093FBF1F31B014FF4BD
:106D5000B47103F5B9531433B3FBF1F310B503F079
:106D60000F03074C1919E35813604B6853600B7AF3
:106D70001372002243685A7210BD00BF8052012076
:106D8000E4620608044B93F8CD3013F0FD0F14BFF6
:106D90009E209D20704700BF88910120094B93F8E9
:106DA000CD3013F0FD0F06D142F210735843064B5D
:106DB00090FBF3F07047242358434FF47A7390FB11
:106DC000F3F070478891012040D20600064B07EE91
:106DD000900A93F8CD30B8EEE70A1BB9DFED037ADD
:106DE00020EE270A704700BF8891012048F95140E2
:106DF000104B10B593F83421012A10D1D3F8382163
:106E0000811A00290BDD0221B3F82E4183F83411D9
:106E10000949B1FBF4F142B10A44C3F8382193F8AF
:106E20003401013818BF012010BD0844C3F83801EF
:106E3000F5E700BF8891012040420F00831E00F15A
:106E40007A02EA2123F8021F9342FBD14E2243F635
:106E50004913C280CE224385CD2302812322838021
:106E6000A0F87220A0F87830704700BF30B400BBA3
:106E70001D48B0F83C3103F00103C3B990F840411C
:106E8000ACB11A4A02F1F00502E00133A3420ED080
:106E900052F8041B4904F8D590F82C1200EB81013C
:106EA000D1F8C41145F823100133A342F0D130BC0E
:106EB00070470D48B0F83C31032B4FEA530408D912
:106EC0000D6804F001030A4AA0F83C412A440A6014
:106ED000D3E70A6848F20504054BA0F83C41134487
:106EE00030BC0B60704700BF88910120CC9201201C
:106EF000A08601002DE9F04100283AD12D4A92F8F0
:106F0000400180B32C4A00242C4B92F804E092F903
:106F100005C003EB8000CEF1FF07AEF17F0692F9CA
:106F2000068003F1F002FFB2F6B203E0834202F101
:106F3000040218D053F8041B8904F7D5E1B2A1EB81
:106F40000C0181EAE175A5EBE175012D0DDC71B154
:106F5000414514BF394631468342D17004F10104E2
:106F600002F10402E6D1BDE8F0810821F4E77146A0
:106F7000F2E7114B1A79F02A09D802F10F000D4AF5
:106F80001871086844F21A1303440B60B7E7094A02
:106F90007F2593F9054092F842011D71844298794A
:106FA00001DA002C02DA4042C0B2987120445871D4
:106FB000E7E700BF8891012050060120CC92012014
:106FC000F0B5384E78B196F8B432002B46D0013B7C
:106FD000354ADBB286F8B4321378DB0741D4334B41
:106FE0000A681A440A6096F84041B4B3304B002551
:106FF0002D4F03EB840403F1F00003E09C4200F109
:1070000004002AD053F8041BC1F30322062AF5D149
:1070100097F800C0EA431CF0010F02F001020DD006
:1070200096F8B42296F843E102EB050CBCFBFEF2A5
:107030000EFB12C2012ACCBF002201220135002A18
:10704000DCD0C1F383419C4200F1040006EB8101D6
:10705000D1F8C42140F8042CD4D1F0BD96F84331C6
:10706000B5E7D6EDB17A6420124BFDEEE77A124D0A
:10707000124C17EE902AA2F57A7200FB02F283FB03
:107080000230D317C3EBA01303EB4303C3EB03138B
:1070900085FB0302DB17C3EB6213053394FBF3F3A9
:1070A0009EE700BF88910120768E0120400D0300ED
:1070B000CC920120D34D62101F85EB5140420F004E
:1070C000F0B4524C002864D194F8000300285CD03E
:1070D0004F4BB3EE097AD3ED007AF4EEC77AF1EEB6
:1070E00010FA54DCBBEE097AF4EEC77AF1EE10FA2E
:1070F0004CBF08270027B3EE097AD3ED017AF4EEEE
:10710000C77AF1EE10FA6FDD47F0010794F84051AD
:10711000002D3AD03F4ADFF80CC102EB850502F1A1
:10712000F00011E094F90363B142ACBF02210021E9
:1071300094F90463B34218DB41F004010F421CD1FF
:10714000954200F1040020D052F8043BD903F7D552
:1071500003F00F0194F90263C3F30313B142E1DCBE
:1071600094F904630121B342E6DA94F90563B3426A
:10717000D8BF41F008010F42E2D0DCF80C30954254
:1071800000F1040040F8043CDED1F0BC7047042755
:10719000B1E794F801338BB31D4B1F4ED3ED007A4A
:1071A00093ED017AF0EEE77A1C4DB0EEC77A0A68EB
:1071B00094F80003C7FE877AFDEEE77A80F00100BD
:1071C00017EE903A84F80003193B03EB4303C3EB3B
:1071D000031386FB0376DB17C3EBE6130533B5FB1E
:1071E000F3F31A440A6071E7BBEE097AF4EEC77A4A
:1071F000F1EE10FA48BF47F0020787E70A68084B2C
:1072000094F8000313440B6060E700BF88910120ED
:107210002C8F0120CC920120353AFC4440420F00D3
:10722000400D030004D80508F0B40D4F97F84061F5
:10723000A6B107F5A272054607F50D77002302E017
:107240000133B3420AD052F8044B35EA0400F7D1B7
:10725000086847F823000133B342F4D1F0BC70470B
:1072600088910120294B30B460B9294A127DBAB9FE
:1072700093F82D322749203301EB83014FF4A060AE
:1072800030BCD1E793F80603E0B10138204A83F817
:1072900006030C68204820440860127D002AE7D0CD
:1072A0001E4A12689106E3D51D4A93F80613127818
:1072B00092071AD511BB93F82F321649203301EBF0
:1072C0008301DBE7124A93F80743157DA54205D8F1
:1072D000042483F8070383F80643DAE70134012026
:1072E00083F8074383F80603D3E70029C0D193F856
:1072F0002E320849203301EB8301BFE793F82B328C
:107300000449203301EB8301B8E700BF88910120D5
:10731000D0510120CC920120801A0600708E0120ED
:10732000FC8E01201D4A10B448B91D4C92F8080388
:107330000B6823440B6098B15DF8044B704792F8DA
:10734000093303B3012B16D092F808030B68154CD0
:1073500080F00100234482F808030B600028EBD181
:1073600092F82B324FF440700F4920335DF8044BF4
:1073700001EB830158E792F808030C4C80F0010000
:1073800082F80803D4E708680124054B82F8084313
:1073900003445DF8044B0B60704700BF88910120E7
:1073A00040420F0048E80100CC92012020A10700D4
:1073B0003F4A10B4B0B992F80A336BB192F80B138C
:1073C0008A081341DB070AD501F00101032A06D818
:1073D000DFE802F0534B433B92F811335BBB5DF89F
:1073E000044B704792F80B33013303F00F0382F81C
:1073F0000B3333B192F80A330C682E4820440860EE
:10740000DBE72D4882F80A33437A002B46D12B481C
:10741000C07818B143F0040382F80A332848007892
:10742000C00732D592F810030028E5D043F00803D6
:1074300082F80A33E0E792F81E33224901EB830118
:107440004FF400305DF8044BEEE61E4B03F13002C2
:10745000002914BF19461146F2E71B4B03F118022D
:1074600000290CBF19461146EAE7164B03F1080242
:10747000002914BF19461146E2E7124B03F1180226
:10748000002914BF19461146DAE7D2F80C03002888
:10749000C8D043F0010382F80A33C3E792F80933F6
:1074A000002BB4D00220034682F80A03AFE700BFE6
:1074B00088910120A08601003C8F0120788E012058
:1074C000768E012004D8050814D8050870B432213E
:1074D000022640F203154FF4FA7446F201420023EB
:1074E000C6708580C48001814281038070BC704772
:1074F000F8B5224C94F82013621892F82423002A3D
:107500003AD000231E4D4A1C0133A5FB02614908F5
:1075100001EBC101511A621892F824230AB1092B18
:10752000F1D1CBB284F8203302680C260025571C19
:10753000076001EB41071670026801EB8701561CDA
:10754000066015700D2205680E4E6F1C31440760F1
:107550002B7037F0FDFB94F820130120084B0A181C
:107560002144A3FB025381F82403C34003EBC3036C
:10757000D31A84F82033F8BD0B46D5E78891012053
:10758000398EE338B8940120024B0146D3F8A803A2
:1075900026F0F4BA8891012008B5044BD3F8AC0367
:1075A00026F0C6FAB0FA80F0400908BD88910120A3
:1075B000044B93F831310BB11DF01ABF024B188800
:1075C000704700BF88910120248F0120084B07EEEF
:1075D000900A93F8CD304BB9F8EEE77A9FED057A33
:1075E0009FED050AA7EE870A44F0EAB9704700BF8D
:1075F000889101206766E63F0000004210B5184CF4
:10760000A379CBB194F82230C0B2DFED166A07EE51
:10761000903A154BF8EEE77A03EB8000838986EE0B
:10762000A77A07EE903AF8EEE77A67EE277AFDEE52
:10763000E77A17EE900A10BD0C4B1B6813F000633D
:107640000CD0C0B2FFF74AF86423808910FB03F026
:1076500094F822305B0890FBF3F0ECE71846EAE779
:10766000B4490120000048434C4E0020B85101208D
:1076700008B5FFF7C3FF3C2390FBF3F008BD0328D8
:1076800011D8DFE800F00A0C0206084BD3F8B40367
:107690007047074B1B78DB0701D426F06FB8034B0C
:1076A000D3F8B00370470020704700BF88910120D5
:1076B000768E0120F0B52B4F0E462B4A83B03B68E7
:1076C0002A4D82FB0312DC17B5F8DC33C4EBA204AD
:1076D0003F89A4B2A3420CD1D5F8E0332449F31A70
:1076E000B5F8E4238B4298BFBA4214BF01230023AC
:1076F00034D0036834210022019003F1010CC0F85A
:1077000000C019702146036803F1010CC0F800C0E5
:107710001A7037F061FB3946019837F05DFB47F688
:10772000FF71019837F058FB47F6FF71019837F069
:1077300053FB47F6FF71019837F04EFB47F6FF7198
:10774000019837F049FB01980221F5F765FC012308
:10775000A5F8DC43A5F8E473C5F8E063184603B068
:10776000F0BD00BF588F01206766666688910120D2
:1077700080841E0002680E2170B5561C7F250024EF
:10778000066015700268551C05601470F5F744FC1E
:10779000012070BD2DE9F0416A4F84B06A4D044666
:1077A000D7F800800E4640460CF023FB85F8E60330
:1077B000B8F1000F0AD00DF1090202A940460CF001
:1077C00048F9002840F08D8095F8E603002319461B
:1077D000ADF808308DF80A30431E0022FF208DF8E6
:1077E0000C10DBB2ADF80E208DF80B00FD2B04D988
:1077F0000023184604B0BDE8F0819DF80830042B42
:1078000000F09480052B00F09780032B00F0968009
:10781000022B00F08A80012B00F092809DF8093045
:107820000DF10E023868013B9DF80A108DF8093001
:107830000CF078F895F8E633032B74D0042B0CD1B8
:10784000424A9DF80A000121002301E012F8011FBD
:1078500081426ED20133082BF8D1D5F8E8230DF11F
:107860000808029B3A4F9A4250D023680D2100220B
:10787000581C2060204619702368591C21601A701A
:1078800023689DF80820591C21601A7023689DF810
:107890000920591C21601A7023689DF80C20591C7E
:1078A00021601A7023689DF80A20591C21601A7003
:1078B000BDF80E1037F090FA23689DF80B20204693
:1078C000591C216007211A70F5F7A6FB0123C5F8A2
:1078D000F06398E8030087E80300184604B0BDE8A9
:1078E000F08101A940460CF0ABF800283FF46CAFE2
:1078F00040460DF10A010CF0A9F800283FF464AFEE
:10790000019995F8E60301F0010165E77A68D8F876
:1079100004309A42A9D1D5F8F0330E4AF31A9342B3
:107920007FF666AFA1E70C4A8BE703228DF80820AB
:1079300074E78DF80A3090E70122F7E70222F5E7B5
:107940000422F3E7D88E012088910120185D0608F3
:107950007095012080841E00245D0608C74B1B68BB
:107960002DE9F04F814613F0800083B000F078815C
:10797000C34B187810F0020000F07281DFF820A3EA
:107980009AF81430052B40F27281DAF80030BD4CC1
:10799000002B0093BC48B8BF5B42BC49A4FB035218
:1079A000920D00FB023302EB8202C3EB031302EBE6
:1079B00082029B0084FB0354DD17C5EBA45500FB3A
:1079C000053305EB820581FB0321ADB2DB17C3EB69
:1079D000A111C5B10020AE4F0446A7FB053CC3B2C0
:1079E0002E4601304FEADC0C9A00092E0CEB8C037A
:1079F000A5EB43031FFA8CF59BB203FA02F344EAAA
:107A00000304EAD8250489B2C1B10020A04F04467E
:107A1000A7FB013CC3B20E4601304FEADC0C9A00D2
:107A2000092E0CEB8C03A1EB43031FFA8CF19BB2E4
:107A300003FA02F344EA0304EAD82543DAF804B06F
:107A4000904C8BEAEB739048904AA3EBEB73A4FB4A
:107A50000361890D00FB013301EB8101C3EB0313CB
:107A600001EB81019B0084FB0364DE17C6EBA45687
:107A700000FB063306EB810682FB0312B6B2DB176E
:107A8000C3EBA212CEB10021814F0846A7FB063EF0
:107A9000CBB2344601314FEADE0E4FEA830C092C9B
:107AA0000EEB8E03A6EB43031FFA8EF69BB203FA8E
:107AB0000CF340EA0300E9D8060492B2CAB10021EF
:107AC000734F0846A7FB023ECBB2144601314FEA82
:107AD000DE0E4FEA830C092C0EEB8E03A2EB430360
:107AE0001FFA8EF29BB203FA0CF340EA0300E9D8C6
:107AF0000643DAF80830664A002B18460193B8BFEF
:107B00005842644C6449A2FB0030030AA4FB0343BF
:107B1000DB0901FB03F1C1EBD00189B2C1B1002443
:107B200096462746AEFB013CE3B20A4601344FEAD3
:107B3000DC0C9800092A0CEB8C03A1EB43031FFA21
:107B40008CF19BB203FA00F347EA0307EAD8B9B213
:107B5000BAF81080B8F1000F1AD00024DFF830E135
:107B60002746AEFB083CE3B2424601344FEADC0C48
:107B70009800092A0CEB8C03A8EB43031FFA8CF83E
:107B80009BB203FA00F347EA0307EAD81FFA87F823
:107B9000BAF812303E4AA2FB0307FF08632F28BF42
:107BA0006327092B67D94FF0000C92466046AAFB69
:107BB000073E5FFA8CF33A460CF1010C4FEADE0EF9
:107BC0009C00092A0EEB8E03A7EB43031FFA8EF7E6
:107BD0009BB203FA04F340EA0300E8D8C4B2009B66
:107BE000019A002BCCBF39233823BBF1000F4FEA99
:107BF000226738DD27F07F07284A3B43934543F04F
:107C00000207C8BF43F00607D9F80030162000224B
:107C100003F1010CC9F800C018704846D9F80030CB
:107C200003F1010CC9F800C01A7037F0D5F82946E5
:107C3000484637F0BBF83146484637F0B7F8484673
:107C4000414637F0C9F8D9F8003001201A18C9F8B0
:107C500000201C70D9F800301A18C9F800201F70D5
:107C600003B0BDE8F08F27F07F071F43CCE700206B
:107C700003B0BDE8F08F0024B1E700BFB851012088
:107C8000FC8E01206BCA5F6B806967FFD34D621069
:107C9000CDCCCCCCC55A7C0AA0860100FFC99A3B4A
:107CA000D0510120AE4B1B682DE9F047064613F07A
:107CB000800084B000F0A180AA4B187810F0020078
:107CC00000F09B80DFF8B4E29EF81410052940F222
:107CD0009980632900F29480002089B2A24F044663
:107CE000A7FB013CC3B20D4601304FEADC0C9A0001
:107CF000092D0CEB8C03A1EB43031FFA8CF19BB213
:107D000003FA02F344EA0304EAD8E4B2DEF80830E6
:107D1000964AD91782FB0323C1EB633399B200293A
:107D200000F019810025DFF840C22846ACFB01387D
:107D3000EBB20F4601354FEAD8089A00092F08EB3D
:107D40008803A1EB43031FFA88F19BB203FA02F305
:107D500040EA0300EAD8C7B2BEF80E304FF4F3652C
:107D6000834942F20F7005FB03F5A1FB0535C5F30E
:107D70008F1585424AD8D5B10021DFF8ECE10846DD
:107D8000AEFB0538CBB2AC4601314FEAD8089A00B9
:107D9000BCF1090F08EB8803A5EB43031FFA88F534
:107DA0009BB203FA02F340EA0300E9D885B2714BB3
:107DB000D3E9FE2313433ED14FF0FF383368294601
:107DC000172000225D1C35601870304633685D1C3A
:107DD00035601A7037F000F84146304636F0E6FF5D
:107DE0003368304606215A1C32601C7033685A1CB6
:107DF00032601F70F5F710F9012004B0BDE8F0877C
:107E0000992483E7002004B0BDE8F0870021DFF863
:107E100058C10D46ACFB0032D20802EB8203A0EB46
:107E2000430390B29BB28B400431102945EA03050D
:107E3000F0D1ADB2BBE701A837F0DEF99DF808102C
:107E4000002900F08A800020DFF81CE18046AEFBAC
:107E50000139C3B28C4601304FEAD9099A00BCF10E
:107E6000090F09EB8903A1EB43031FFA89F19BB2C8
:107E700003FA02F348EA0308E9D84FEA08289DF814
:107E80000920E2B10021DFF8E0E00846AEFB023A4B
:107E9000CBB2944601314FEADA0A4FEA8309BCF1CA
:107EA000090F0AEB8A03A2EB43031FFA8AF29BB283
:107EB00003FA09F340EA0300E8D848EA00089DF80D
:107EC0000A204FEA0828E2B10021DFF89CE00846CA
:107ED000AEFB023ACBB2944601314FEADA0A4FEADE
:107EE0008309BCF1090F0AEB8A03A2EB43031FFAD3
:107EF0008AF29BB203FA09F340EA0300E8D848EAA1
:107F00000008BDF80C304FEA08181B4A632BA2FB8F
:107F100003124FEA52127FF651AF0021DFF848E01A
:107F20000846AEFB023ACBB2944601314FEADA0A78
:107F30004FEA8309BCF1090F0AEB8A03A2EB430362
:107F40001FFA8AF29BB203FA09F340EA0300E8D869
:107F500048EA000832E70F46FEE688468FE700BF92
:107F6000B8510120FC8E0120CDCCCCCC89B5F814C1
:107F7000D34D6210889101201F85EB51D051012013
:107F8000F8B53B4B054601687E27B3F9003400265F
:107F9000384A481C03EBC3032860FF2082FB0342DE
:107FA000DC170F702B68C4EB62045A1C20342A6063
:107FB000A4B21E70FEF792FB2F4B00284DD01B7809
:107FC000B0F90C1023BBA1F57A722C4B9A4246D81B
:107FD0002B48B0FBF1F189B2284636F0D9FE294B87
:107FE000DB7A7BB11DF004FA0146284636F0D0FE5C
:107FF0002146284636F0CCFE28460821F5F70CF835
:108000000120F8BD204B2846198836F0C1FEEFE765
:108010001E4B1E78002ED6D000231D4800EB830295
:1080200001339289B3421144F8DB1A4B07EE901AE0
:108030009FED196A93F82230F8EE676A07EE103A5E
:10804000B8EEC77AC6EE077A67EEA67AFCEEE77A54
:1080500017EE901AB1FBF6F1B5E71B7813B94EF69F
:108060009C21B9E7094B1E78002EF8D00146D3E7D2
:1080700088910120676666660C15002017839303BC
:1080800000879303008F0120248F012070070020B8
:108090004C4E0020B449012000004843244A0023EC
:1080A0004361D2F8DC1041F45C5130B541F02C0151
:1080B0000124C2F8DC104471D2F8D41004FA03F59C
:1080C0000133112B41EA0501F8D121F4F0314FF4CD
:1080D00020634FF0A064C2F8D4105022C38040F651
:1080E000012314490381144BA0F856206FF07E42FF
:1080F0000360142303718023037642F61403038282
:108100004FF6FF73438303F58C03C36140F20123F1
:10811000C0E9161203840023084A80F8223080F850
:10812000333080F84430A0F86830C0E9184230BDE0
:1081300088910120C4FF00FF98086400180B0C0010
:1081400008B5A0F101030228B3FA83F34FEA5313F1
:1081500001D0184608BD0F2019F0E4FB28B9054BE3
:108160001B7803F00103184608BD0F20BDE8084046
:1081700019F062BC768E012038B5054680220021B8
:1081800005F1800444F000FF00213822204644F02D
:10819000FBFE00230B4951F8232044F82320013330
:1081A0000E2BF8D11E22084905F1C00044F07AFEDA
:1081B0000B22064905F1E40044F074FE032385F820
:1081C000EF3038BD04D805083CD805085CD8050850
:1081D000034B01220349B3F90830406836F066BD0D
:1081E00050060120DC5C060837B504462A4800EB3F
:1081F0004303B3F8CE5005F00F0049B1022804F153
:1082000001011DD8002814BF9C239B2323700C461A
:108210000AB3C5F30315FFF732FA204B3C21012DB9
:10822000B0FBF3F3B3FBF1F201FB123315D0022DD7
:1082300023D01B49204603B0BDE8304036F036BDA0
:10824000032806D1174B1B7803F00103653BDBB213
:10825000DCE72023DAE71546DDE742F210716425FA
:10826000B0FBF1F1B1FBF5F005FB10100E490090E9
:10827000204636F01BFD03B030BD0C490A25B0FB8B
:10828000F1F1B1FBF5F005FB101009490090204613
:1082900036F00CFDEFE700BF8891012040420F004F
:1082A000365D0608768E0120405D0608A086010036
:1082B0004F5D0608037801224068053B114693E7AD
:1082C0001D4B1E499A68B1F8C83007EE902A9FED01
:1082D0001C7A4068F8EEE76A07EE903AF8EEE77A23
:1082E00067EE877AF4EEE76AF1EE10FA02D81549E4
:1082F00036F0DCBC934202DA134936F0D7BC9B1A45
:10830000124A07EE903AB8EEE77AD1EDEC7A3C21CA
:10831000F8EE677A67EE277A87EEA67AFDEEC77ADF
:1083200017EE903AB3FBF2F3B3FBF1F201FB123319
:10833000074936F0BBBC00BF588F0120889101204F
:10834000CDCCCC3D5E5D0608645D060840420F0062
:10835000365D0608064B07491A88074B40681B68BC
:10836000534342F2107293FBF2F236F09FBC00BF0F
:10837000248F01206A5D0608588F0120054A0649AE
:1083800092F8053492F8042401334068013236F043
:108390008DBC00BF889101206F5D06080B4B0A223F
:1083A0004FF4B4714068B3F9043093FBF2F31A014F
:1083B00002F5B9521432B2FBF1F2C2F108020449DB
:1083C00002F00F02603236F071BC00BF8052012013
:1083D000755D0608034A072303499268406836F032
:1083E00065BC00BF588F01207C5D060807B5144AA4
:1083F000406892F81414B2F81634012909D1009398
:10840000104992F818347B2236F050FC03B05DF826
:1084100004FB022906D17B220B4903B05DF804EB73
:1084200036F044BC0A220949534340F2FF32B3FB01
:10843000F2F39BB27B22092B28BF0923EDE700BF93
:1084400088910120825D0608375E06088C5D06086B
:1084500013B54468FEF796FC0F4B02461B789B074A
:1084600012D50E4B93F823140D4B59B19889FEF792
:1084700095FC0C49034600922046702236F016FC0B
:1084800002B010BDD889F2E700902D237022064972
:10849000204636F00BFCF3E7FC8E0120889101208A
:1084A000D0510120EA5D0608925D06082DE9F041F1
:1084B000404F86B090F800C006463C78BCF1170FDC
:1084C000416890F803E00CBF4FF098084FF089081E
:1084D00014F0040405D0BCF1170F374B0CBF5C68D7
:1084E0001C6884EAE473354DBEF1010F01F101000F
:1084F000A3EBE473B3FBF5F205FB123345D0BEF1F9
:10850000020F46D181F800803C21BCF1170F01FB1E
:1085100003F3B3FBF5FE05FB1E3301FB03F3B3FBD3
:10852000F5F105FB1135264BB5FBF3F528D1002CF1
:10853000B4BF572345230593222302912149CDE956
:1085400003532723CDE900E3082336F0AFFB33784C
:108550001D495A0903F01F0301EB8201012202FAAF
:1085600003F33A78D1F8280402F00602042A0CBF7B
:10857000034320EA0303C1F8283406B0BDE8F081C4
:10858000002CB4BF53234E23D5E74FF47A75B3FBC9
:10859000F5F3002C81F8008002DA2D24881C4C7041
:1085A0000A4C0B49BEF1000F08BF214636F07EFB96
:1085B000CDE700BFFC8E0120D051012080969800AD
:1085C00040420F00A95D060888910120995D0608C8
:1085D000A15D06080D4B1B681B0137B514D50C4C6B
:1085E0004568D4F8303493F90100FEF7EFFF94F8B2
:1085F000CD2003460749002A28460CBF0D220E2233
:1086000000927A2236F052FB03B030BDB8510120FF
:1086100088910120BF5D0608034B0449D3F8342438
:10862000406836F043BB00BF88910120C85D060852
:10863000044B1B78DB0703D40349406836F036BB94
:10864000704700BF768E0120CC5D060807B5094A49
:108650000949B2F906300193B2F904300093B2F936
:108660000230B2F90020406836F020FB03B05DF81C
:1086700004FB00BFF4480120D55D060837B50A4C5D
:108680004568B4F90004FEF7A1FF94F8CD20034635
:108690000649002A28460CBF0D220E2200927A229B
:1086A00036F004FB03B030BD88910120E95D060877
:1086B000084BD3F84424002A0ADD074B03EB82035E
:1086C0001A6E2AB1054B0649DB68406836F0EEBAEF
:1086D000704700BF8891012004D80508500601208A
:1086E000F25D06081FB5938802939378019353783F
:1086F000009313780A46034936F0D8FA05B05DF8BE
:1087000004FB00BFFA5D0608034B0449D3F8482474
:1087100040681432E6E700BF889101200D5E06082C
:10872000034B0449D3F8482440680832DAE700BF15
:1087300088910120115E0608034B0449D3F84824B0
:1087400040680E32CEE700BF88910120155E060812
:108750002DE9F0472DED028B82B0924607460C467C
:108760009DF8302099469DF83480002B52D0022B82
:1087700014BF0A25642507EE905AF8EEE77A27EE33
:10878000808A002A48D0B0EE480A43F019F907EE73
:10879000900AF8EEE77AF0EEE77AFDEEE77A17EE68
:1087A000906AB6FBF5F205FB12660CB13C70012431
:1087B000B5EEC08AF1EE10FA05D552EA060302D0F2
:1087C0002D233B5501349AF800103819144B002919
:1087D00014BF5146194636F069FA2518B9F1000F51
:1087E0000AD04A460F49684636F060FA7819324690
:1087F000694636F05BFA0544B8F1000F02D007F87D
:1088000005800135002328467B5502B0BDEC028B64
:10881000BDE8F0870125AEE7F0EE487ABBE700BF80
:10882000195E06081E5E06081A4B1A6812F0200F21
:1088300002F0040313B5446825D0174A1278920752
:1088400021D5164BB3F90000FEF7C0FADFED147A1C
:10885000144B204620EE270A134A93F8CD30B5EE8C
:10886000C00AB0EEC00AF1EE10FA4CBF76217521B5
:10887000002B0CBF99239F23019301230093FFF743
:1088800067FF02B010BD002BDBD12D2222704268A1
:108890005370F6E7708E0120FC8E0120648F01205A
:1088A0000AD7233C8891012082AB06081FB5184BDC
:1088B0009FED187A1B88184A07EE903A9FED170A29
:1088C00092F80923F8EEE77A4468F4EEC77A27EEC7
:1088D000800AF1EE10FAACBF01230223022A14D061
:1088E0008DED030A02931CF083FDFEF7BAF9029B9B
:1088F00001469DED030A01220620CDE90020084A29
:108900002046FFF725FF04B010BD9721F3E700BF15
:10891000248F012000007A44889101200AD7233C4B
:1089200082AB0608114BB3F84C34B3F57A7F07B528
:10893000406806D201220E4903B05DF804EB36F020
:10894000B5B907EE903A572200239FED0A0AF8EED8
:10895000E77ACDE90032012327EE800A064A19465C
:10896000FFF7F6FE03B05DF804FB00BF889101201D
:10897000265E06086F12833A82AB060873B5194E5D
:108980000546406896F86834052B07D01F231E2241
:10899000154902B0BDE8704036F088B9134C1E226C
:1089A0001349237D00931F2336F080F996F8223176
:1089B000ABB16B6820220021DFED0E7A1A54638A76
:1089C000441C686800EE103A01230B4A2044B8EEBC
:1089D000C00ACDE9003120EE270AFFF7B9FE02B048
:1089E00070BD00BF889101202E5E0608D051012085
:1089F000355E06080AD7233C82AB060807B501237B
:108A000047220649CDE90032054A91ED000A0021CE
:108A10004068FFF79DFE03B05DF804FBF895012068
:108A200082AB06080B4BDFED0C7A93ED000A9A231C
:108A3000B8EEC00A07B520EE270A0021074AB0EEBB
:108A4000C00ACDE9001302234068FFF781FE03B09E
:108A50005DF804FB588F01200AD7233C3D5E0608D1
:108A600013B504461CF0C4FC0E4B00EE100A6468FB
:108A700093F80933022B13D0FEF7F3F80146B8EE52
:108A8000C00ADFED097A00230622204620EE270ADD
:108A9000CDE900320223054AFFF75AFE02B010BDAD
:108AA0009721ECE7889101200AD7233C82AB060886
:108AB00013B50378134A1A2BDFED137A134C0CBF4E
:108AC000B2F90220B2F900201A2B4FF0010300EE98
:108AD000102A0CBF152114210022B8EEC00ACDE9DE
:108AE000003220EE270A0A4A4068B5EEC00AB0EE0E
:108AF000C00AF1EE10FA48BF2246FFF729FE02B085
:108B000010BD00BF80520120CDCCCC3D415E060897
:108B1000475E0608194B37B51A68446812F0200FF3
:108B200002F0040320D0164A127892071CD5154A89
:108B3000C17892F8CD30D2F87404002B0CBF0F2509
:108B40000C25FEF743F90123DFED0F7A2046009351
:108B5000CB1A20EE270A0D4A18BF01237F21019569
:108B6000FFF7F6FD03B030BD002BE0D17F222D21B1
:108B700022704268517042689370F3E7708E012052
:108B8000FC8E0120889101200AD7233C82AB060885
:108B900013B5044608461146FEF718F9164B93F82C
:108BA000CD30002B0BBF4FF4A5534FF47A737E22C8
:108BB0007D2207EE903A0CBF0F230C23F8EEE77AE4
:108BC000F4EEC07AF1EE10FA13DC80EE270AF2EE32
:108BD000047AB4EEE70AF1EE10FAACBF01230223E7
:108BE0000192002220460092044AFFF7B1FD02B034
:108BF00010BD1A460023F3E78891012082AB0608D6
:108C00000C4B10B41B78446803F00303032B06D10C
:108C1000094B204611225DF8044B1988B8E711234F
:108C20002D22237043685A70002243689A705DF8C1
:108C3000044B7047FC8E0120FE8E0120094B4068DA
:108C40001B7803F00303032B07D1074B7122D3F8E2
:108C500078146423B1FBF3F19AE72D2371220349C1
:108C600036F024B8FC8E012088910120945D06081E
:108C7000224B1B885A0510B5446805D5204620496B
:108C8000BDE8104044F05EBA180505D520461D49E0
:108C9000BDE8104044F056BA590605D520461A4999
:108CA000BDE8104044F04EBADA0705D52046174912
:108CB000BDE8104044F046BA9B0705D5204614494C
:108CC000BDE8104044F03EBA252018F0B5FE28B1AA
:108CD00020461049BDE8104044F034BA0E4B93F8DA
:108CE0007C342BB120460D49BDE8104044F02ABA2F
:108CF00020460B49BDE8104044F024BAA45201209C
:108D00004D5E0608525E0608575E06085C5E060861
:108D1000615E0608665E0608889101206B5E0608A3
:108D2000705E0608074B93ED6E7AD3ED6B7AB4EE66
:108D3000E77AF1EE10FA03DD0349406844F002BA25
:108D4000704700BF08310020755E060810B50C465C
:108D5000A0B9174A174892F87D142368034423608A
:108D600001B110BD92F82B324FF4806012492033CC
:108D7000BDE8104001EB8301FEF756BA11F008FF81
:108D8000322808DD206801210A4B094A034482F891
:108D90007D14236010BD064A142892F87D14C8BFC4
:108DA000064881F00101D8BF054882F87D14D4E758
:108DB0008891012040420F00CC92012020A10700A1
:108DC00048E8010010B504461AF036FE04220346B6
:108DD00002496068BDE8104035F068BFDC5C0608F9
:108DE0002B4BF0B51C6887B02A4E074620463178D9
:108DF0000AF014FE7178054620460AF0FBFD0022B9
:108E000003460592B2788DF813206CB1039005A942
:108E100020460AF015FE327A039B2AB10DF11301A8
:108E200020460AF013FE039B9DF81310ECB1E1B14C
:108E3000194A1268914218DC184A02EB8102D2F8F2
:108E400080442620039318F0F7FD0599039B70B921
:108E500011F0010F14BF502200228907786808D54D
:108E60000F4935F023FF07B0F0BD0E4CE9E744226F
:108E7000F3E732B10C49CDE900422A4635F016FF3E
:108E8000F1E72A460949009435F010FFEBE700BFEF
:108E9000D88E0120B85201207C8D012088910120BC
:108EA000785E0608BD640608805E06088C5E0608CB
:108EB000F8B50446417882782C48237890F8E95038
:108EC000302B2B4B05F1FF354FEA85052B4448D15C
:108ED00093F8E85093F8E96000EB85054FF47A7752
:108EE00000EB86004FF0030CD5EDAE7A40F2CF7563
:108EF000FDEEE77A17EE903AD0EDAE7AAB42FDEE9A
:108F0000E77AA8BF2B4617EE900AB3F57A7FB8BF71
:108F10004FF47A73A842A3F57A73A8BF2846C3EB2F
:108F20000313B842B3FBF7F3C3F10E03B8BF3846DF
:108F3000DBB2A0F57A70B3FBFCFCC0EBC00062446E
:108F40000CEB4C0ED2B2A3EB0E03B0FBF7F70833D9
:108F500039442046DBB2C9B2F4F7E2FD00232373A3
:108F6000F8BD93F8EA5093F8EB60B5E788910120DB
:108F700004D805082DE9F04790F80290044690F8CF
:108F80000180002609F10207FFB2002508EB060A5E
:108F9000032E1BD108F10301022DC9B20ED10B2300
:108FA0003A462046F4F7BCFD0135052DF0D10136D7
:108FB000072EEAD100232373BDE8F08709EB0502F1
:108FC00016232046D2B2F4F7ABFDEDE7022DEBD12C
:108FD00017233A465FFA8AF12046F4F7A1FDE3E74A
:108FE00070B504466FF00205A2781323617820461D
:108FF00052FA85F2EEB207390135D2B2C9B2F4F7AE
:109000008FFDA27861781323324420460731D2B213
:10901000C9B2F4F785FD042DE6D161780323A27867
:1090200020460639C9B2F4F77BFD61780223A278A5
:1090300006312046C9B2F4F773FD0023237370BDD7
:109040002D492DE9F84391F8D830054691F8D920FB
:1090500091F8E71003EB830302EB82022748002913
:109060004FEA43034FEA4202B0F9004014BF4FF009
:10907000FF310121C2F100084C43444503DB944217
:10908000A8BF1446A046B0F902205C424A43A2425F
:1090900003DB9A42A8BF1A4614461BB11922544357
:1090A00094FBF3F4293C4FEA88066FF003074FF076
:1090B0000909002E3346B8BF06F13F03C4EBA313E2
:1090C000512B0FD8284693FBF9F101EBC1029B1AF3
:1090D000AA780A446978803B3944D2B2DBB2C9B27B
:1090E000F4F71EFD0137A6EB0806052FE1D100239A
:1090F0002B73BDE8F88300BF8891012080520120C6
:1091000010B5044611F080FD6422074902FB00F30C
:1091100060680122C3F38F23632BBDE8104028BF92
:10912000632335F0C3BD00BF375E06082DE9F84361
:109130000546002415F0FCF81C4E07464FF0880841
:10914000DFF86C9033786968A342214403DC002384
:109150000B70BDE8F88337B3D6ED427A09EB840390
:10916000FDEEE77A17EE900AD3ED007AFDEEE77A8E
:1091700017EE902AD6ED437AFDEEE77A121AD20066
:1091800017EE903A1B1A204692FBF3F3C3F18803C3
:109190000B70FEF733FAB0F57A7F02DA6B68532270
:1091A0001A550134CEE781F80080FAE770070020F5
:1091B00060300020374B13B5C17804469A68022905
:1091C000354B9B8941D0032945D0012905D19A1AF5
:1091D0009A42A8BF1A4622EAE272D3B19A1A0B2029
:1091E0009A42A8BF1A46B3FBF0F322EAE27207EEF6
:1091F000902AB8EEE77A07EE903AF8EEE77AC7EEF3
